:100000000C941D190C9456190C9456190C945619ED
:100010000C9456190C9456190C9456190C945619A4
:100020000C9456190C9456190C9456190C94561994
:100030000C9456190C9432890C9456190C94561938
:100040000C9456190C9497830C9419BD0C94561962
:100050000C94FC4D0C94F24D0C9456190C945619BA
:100060000C9456190C9456190C9456190C94561954
:100070000C9456190C9456190C9456190C94561944
:100080000C9456190C9456190C9456194E414E491D
:100090004E495459494E46CDCCCC3D0AD7233C1746
:1000A000B7D13877CC2B329595E6241FB14F0A0093
:1000B0000020410000C84200401C4620BCBE4CCA83
:1000C0001B0E5AAEC59D7400407A10F35A00A07200
:1000D0004E18090010A5D4E80000E8764817000083
:1000E000E40B54020000CA9A3B000000E1F5050051
:1000F0000080969800000040420F000000A086019A
:10010000000000102700000000E803000000006469
:1001100000000000000A00000000000100000000D4
:10012000002C76D888DC674F0823DFC1DFAE59E1A9
:10013000B1B796E5E3E453C63AE651997696E8E618
:10014000C28426EB898C9B62ED407C6FFCEFBC9CEB
:100150009F40F2BAA56FA5F490055A2AF75C936BFD
:100160006CF9676DC11BFCE0E40D47FEF520E6B5B8
:1001700000D0ED902E0300943577050080841E0892
:100180000000204E0A000000C80C333333330F98B0
:100190006E12831141EF8D2114893BE65516CFFE77
:1001A000E6DB18D1844B381BF77C1D901DA4BBE403
:1001B00024203284725E228100C9F124ECA1E53D45
:1001C00027434F4D4D554E49434154494F4E0044EE
:1001D000525952554E004552524F525300494E46C5
:1001E0004F004543484F00506C6561736520526570
:1001F000736574005052494E5445522048414C5446
:1002000045440025533A202553004B494C4C454466
:100210002E20005072696E7465722068616C74657E
:10022000642E206B696C6C28292063616C6C65649A
:10023000210A006563686F3A004572726F723A0076
:100240004F4646004F4E000A4D65617375726564F6
:1002500020706F696E74733A0A00337833206D65CD
:1002600073682E205A206F66667365743A20004FBB
:1002700046460A00466164652048656967687420DF
:1002800000426564204C6576656C696E67200046A7
:1002900061696C656420746F20656E61626C6520B5
:1002A000426564204C6576656C696E670A004D6531
:1002B000736820426564204C6576656C20646174C7
:1002C000613A0A00496E76616C6964206D657368F5
:1002D0002E0A00206E6F7420656E74657265642E40
:1002E0000A0020204D3230312058004D61782041E5
:1002F0006363656C65726174696F6E2028756E69E1
:1003000074732F7332290020204D3230332058006F
:100310004D61782066656564726174657320287527
:100320006E6974732F73290020520020204D3230E3
:1003300034205000416363656C65726174696F6E4F
:100340002028756E6974732F7332292028503C70F1
:1003500072696E742D616363656C3E20523C7265F8
:1003600074726163742D616363656C3E20543C74E8
:10037000726176656C2D616363656C3E2900204A6D
:100380000020540020530020204D32303520420000
:10039000416476616E6365642028423C6D696E5FDE
:1003A0007365676D656E745F74696D655F75733EC7
:1003B00020533C6D696E5F66656564726174653E6D
:1003C00020543C6D696E5F74726176656C5F666522
:1003D0006564726174653E204A3C6A756E635F6451
:1003E00065763E290020440020490020204D33300E
:1003F00031205000486F74656E64205049440020DD
:10040000440020490020204D333034205000426504
:100410006420504944002E0A00206E6F74206469E5
:100420007361626C65642E20536861726564207725
:100430006974680020496E76616C6964206578741F
:1004400072756465722000536C6565702E2E2E00E7
:1004500050726F62696E6720506F696E7400255329
:100460002025692F256900206F6620004D424C2011
:1004700047323920706F696E742000290A004A20C3
:100480006F7574206F662072616E67652028302D4D
:1004900000290A0049206F7574206F662072616E12
:1004A00067652028302D004732384C30004D657389
:1004B000682070726F62696E6720646F6E65004DB0
:1004C0006573682070726F62696E6720646F6E6515
:1004D0002E0A005374617274206D65736820707207
:1004E0006F62696E6720776974682022473239200D
:1004F0005331222066697273742E0A0047323953D1
:1005000032004732384C300A473239533200686182
:1005100073206E6F20646174612E0A004D657368EC
:1005200020426564204C6576656C696E67200053D7
:10053000206F7574206F662072616E6765202830A9
:100540002D35292E0A004D65736820706F696E7411
:10055000206F7574206F662072616E67650A0043B4
:100560006C69636B20746F20526573756D652E2EF8
:100570002E00616C736F20656E61626C6564290A80
:10058000004E6F204D6F76652E004E6F206D6564B6
:1005900069610A00456E642066696C65206C697348
:1005A000740A00426567696E2066696C65206C6933
:1005B00073740A00286E6F2066696C6529004E6F9F
:1005C00074205344207072696E74696E670A005318
:1005D00044207072696E74696E6720627974652058
:1005E0000043757272656E742066696C653A20000E
:1005F0002E0A0044656C6574696F6E206661696CD3
:1006000065642C2046696C653A200046696C65205B
:1006100064656C657465643A002569730025696DCD
:1006200020256973002569682025696D2025697377
:1006300000256964202569682025696D2025697376
:100640000025697920256964202569682025696D60
:1006500020256973005072696E742074696D653A63
:1006600020006F6B006F666600E201DD01D601CFEE
:1006700001C10144454255473A004D3131332053C1
:10068000004D656761205A65726F204F46462E0007
:10069000434F4E4649475F4558504F5254004D45D1
:1006A00041545041434B00434F4F4C45525F5445DA
:1006B0004D5045524154555245004348414D4245E5
:1006C000525F54454D5045524154555245004241A8
:1006D00042595354455050494E47004152435300EC
:1006E0004D4F54494F4E5F4D4F444553005448457C
:1006F000524D414C5F50524F54454354494F4E0068
:10070000455854454E4445445F4D3230004C4F4EA1
:10071000475F46494C454E414D45004155544F5267
:1007200045504F52545F53445F5354415455530006
:1007300053445F5752495445005245504541540077
:100740005344434152440050524F4D50545F53550F
:1007500050504F525400484F53545F414354494FF7
:100760004E5F434F4D4D414E445300454D4552471A
:10077000454E43595F504152534552004341534502
:100780005F4C494748545F4252494748544E45538D
:100790005300544F47474C455F4C4947485453001A
:1007A000534F4654574152455F504F5745520042B0
:1007B00055494C445F50455243454E54004C4556B4
:1007C000454C494E475F44415441005A5F50524F97
:1007D00042450052554E4F5554004155544F4C45DB
:1007E00056454C005052494E545F4A4F42005052B9
:1007F0004F4752455353004155544F5245504F5265
:10080000545F54454D50004155544F5245504F523E
:10081000545F504F5300564F4C554D455452494329
:1008200000454550524F4D0042494E4152595F4696
:10083000494C455F5452414E534645520053455230
:1008400049414C5F584F4E5F584F4646004649520B
:100850004D574152455F4E414D453A4D61726C696D
:100860006E20322E302E392E332D6B6164312028CC
:1008700044656320323720323032312031333A340C
:10088000373A30392920534F555243455F434F443F
:10089000455F55524C3A6769746875622E636F6D97
:1008A0002F6B61642F4D61726C696E2050524F54F2
:1008B0004F434F4C5F56455253494F4E3A312E30BD
:1008C000204D414348494E455F545950453A4D6586
:1008D0006761205A65726F204558545255444552FD
:1008E0005F434F554E543A3120555549443A64625E
:1008F0006663636435352D656262612D343631354A
:100900002D616264372D3139366161343338663395
:1009100030340A002F2F004D31343520533C696E9E
:100920006465783E206F7574206F662072616E6713
:10093000652028302D31290A003F4A206F75742028
:100940006F662072616E67652028302E303120740A
:100950006F20302E33290A0020580020204D617866
:100960003A2000200020204D696E3A2000203B20D4
:100970000020204D323131205300536F66742065C2
:100980006E6473746F70730046523A0020466C6F49
:10099000773A20004D424C2041646A757374205AA6
:1009A0000064697300656E0043290A0061626C652A
:1009B0006420286D696E2074656D702000436F6C33
:1009C00064206578747275646573206172652000B7
:1009D0004D65736820706F696E74206F7574206F39
:1009E000662072616E67650A004D34323120696E8F
:1009F000636F727265637420706172616D65746596
:100A0000722075736167650A0020286D6D290020CA
:100A10003B204C6576656C696E67200020204D3464
:100A200032302053004D65736820426564204C6568
:100A300076656C696E670020460020420020480001
:100A400020204D3134352053004D61746572696149
:100A50006C2068656174757020706172616D657479
:100A6000657273002020473239205334205A002009
:100A70004A00202047323920533320490020204D9E
:100A80003134392043203B20556E69747320696EE0
:100A90002043656C736975730A0054656D706572E7
:100AA000617475726520556E697473002020473239
:100AB00031203B004C696E65617220556E6974731C
:100AC00000454550524F4D204F4B0A004D383400E1
:100AD000446F6E65207072696E74696E6720666916
:100AE0006C650A004D3737004D333100496E766131
:100AF0006C69642065787472756465720A0043617C
:100B0000703A00436F6F6C696E672E2E2E00486539
:100B10006174696E672E2E2E00453120255300200A
:100B2000573A0020573A0042656420436F6F6C6962
:100B30006E672E2E2E004265642048656174696ED2
:100B4000672E2E2E0023646566696E652044454637
:100B500041554C545F00626564004B6420004B6952
:100B600020004B702000504944204175746F74750B
:100B70006E652066696E69736865642120507574BE
:100B800020746865206C617374204B702C204B6955
:100B900020616E64204B6420636F6E7374616E74A9
:100BA000732066726F6D2062656C6F7720696E745A
:100BB0006F20436F6E66696775726174696F6E2E20
:100BC000680A00504944204175746F74756E652041
:100BD0006661696C6564212074696D656F75740A5E
:100BE00000504944204175746F74756E65206661CC
:100BF000696C6564212054656D70657261747572ED
:100C00006520746F6F20686967680A005049442046
:100C10004379636C65730025532025692F2569008E
:100C2000204B643A2000204B693A2000204B703A58
:100C3000200020436C617373696320504944200A8B
:100C400000204E6F206F76657273686F6F740A00B4
:100C50002054753A2000204B753A2000206D6178B1
:100C60003A2000206D696E3A200020643A2000206E
:100C7000626961733A20005761697420666F72205F
:100C8000686561742075702E2E2E005049442041F5
:100C900075746F74756E652073746172740A005098
:100CA0004944204175746F74756E65206661696C86
:100CB0006564212054656D7065726174757265207C
:100CC000746F6F20686967680A0050494420417555
:100CD000746F74756E6500504944204175746F746B
:100CE000756E65206661696C6564212042616420CF
:100CF0006865617465722069640A004572723A2001
:100D00007574663820666F6E74206E6F7420696E1D
:100D1000697469616C697A65642E004572723A2063
:100D20007574663820666F6E74206E6F7420696EFD
:100D3000697469616C697A65642E004572723A2043
:100D40007574663820666F6E74206E6F7420696EDD
:100D5000697469616C697A65642E00426564004556
:100D60006E636C6F73757265002568753A25303255
:100D700068750025303268753A253032687500256F
:100D800030326875272530326875002020202020F9
:100D90002020002020202000657272001FE020101B
:100DA000201020101020102020102010303008407B
:100DB000048003001FE03FF03FF03FF01FE01FE022
:100DC0003FF03FF03FF00FC0078003003FFFF038D7
:100DD000007030FC3020FC102078102030102C00E7
:100DE000D02E31D02F7BD02F7BD02E31D02C00D0E5
:100DF00020301020781020FC1030FC303800703F7C
:100E0000FFF03FFFF03800703186302387102787CE
:100E1000902F87D02F03D02030102078102078100A
:100E20002030102F03D02F87D027879023871031B1
:100E300086303800703FFFF01FFFF81FFFF80410E6
:100E400040020820020820041040082080104100C1
:100E50001041000820800410400000001FFFF81F10
:100E6000FFF8001DC43F0000000C86198000000D33
:100E70000E198000000F0B198000000D9F198000D3
:100E8000000DD3998000001CFBFF00000000000053
:100E90000000000000000000F380001F80007700C9
:100EA000001980005B1CF6131DAE5B35AB0635FBED
:100EB0005B3DA70CBD9B4B30EB19B19BE39D8E9F17
:100EC0009D8E0001E00000000001200000000001F4
:100ED000E00000005072696E742041626F727465A8
:100EE00064004D32350050617573696E672E2E2E89
:100EF000004D323400454550524F4D2056657273B7
:100F0000696F6E204572726F7200454550524F4DA9
:100F100020496E646578204572726F7200454550B5
:100F2000524F4D20435243204572726F72003F0072
:100F300049676E6F726500526573657400496E692A
:100F40007469616C697A6520454550524F4D00487F
:100F50006F6D696E672058595A004D3330332055F4
:100F600031204525692053256900504944204175A9
:100F7000746F74756E65202A005049442D44202AF0
:100F8000005049442D49202A005049442D50202A20
:100F90000020082046616374002008204D6178001D
:100FA0002008204D696E004F6666004F6E00417547
:100FB000746F74656D7000452073746570732F6D68
:100FC0006D005A2053746570732F6D6D0059205356
:100FD000746570732F6D6D00582053746570732F96
:100FE0006D6D00416476616E636564205365747451
:100FF000696E67730054656D7065726174757265B2
:101000000053746570732F6D6D00436F6E66696772
:1010100075726174696F6E003F004E65787420438D
:101020006F726E657200446F6E65004E6578740075
:101030004C6576656C696E6720446F6E6521004D66
:101040006F7665205A00473239533200000C0F008A
:10105000FE07022503BB017FFE08FE08FE05080807
:1010600006000040F0C88888987810050808060037
:1010700000C0F88888888888F805050506000120E2
:1010800030F830200508080600002070F8202020E5
:1010900020E00509090600FF2070A8A8B88888701C
:1010A00020070505070001D86C366CD8050909062C
:1010B00000FFF8A88888888888A8F8050A0A06002A
:1010C000FE205050505088A8A888700303030600E3
:1010D0000340A040FFFFFFFFFFFFFFFFFFFFFFFFF9
:1010E000FFFFFFFFFFFFFFFFFFFF0000000605FF00
:1010F00001070706020080808080800080030303D0
:10110000060105A0A0A005060606000050F85050F4
:10111000F8500509090600FF2070A8A07028A870E3
:1011200020050707060000C8C8102040989805074A
:101130000706000040A0A040A89068010303060233
:10114000058080800309090601FF204040808080DF
:101150004040200309090601FF8040402020204034
:10116000408005070706000020A8702070A8200511
:1011700005050600012020F820200203030601FFD8
:10118000C04080050101060003F8020202060100CA
:10119000C0C0050707060000081010204040800569
:1011A0000707060000708898A8C88870030707061C
:1011B000010040C040404040E005070706000070C5
:1011C0008808102040F8050707060000F8081030CE
:1011D00008887005070706000010305090F81010BE
:1011E000050707060000F880F00808887005070763
:1011F000060000304080F088887005070706000070
:10120000F8081010202020050707060000708888C5
:1012100070888870050707060000708888780810B5
:1012200060020505060100C0C000C0C00206060637
:1012300001FFC0C000C04080030505060101204039
:10124000804020050303060002F800F803050506A8
:1012500001018040204080050707060000708810CB
:10126000202000200507070600007088B8A8B88075
:1012700070050707060000708888F88888880507C9
:1012800007060000F04848704848F00507070600C8
:101290000070888080808870050707060000F0488D
:1012A00048484848F0050707060000F88080F080AD
:1012B00080F8050707060000F88080F08080800530
:1012C0000707060000708880809888700507070669
:1012D0000000888888F8888888030707060100E0EE
:1012E0004040404040E0050707060000381010105D
:1012F0001090600507070600008890A0C0A09088A5
:10130000050707060000808080808080F8050707B9
:1013100006000088D8A88888888805070706000086
:101320008888C8A8988888050707060000708888FC
:1013300088888870050707060000F08888F080809C
:101340008005070706000070888888A89068050750
:1013500007060000F08888F0A090880507070600BF
:101360000070888070088870050707060000F82064
:10137000202020202005070706000088888888880C
:101380008870050707060000888888885050200567
:10139000070706000088888888A8A8500507070660
:1013A00000008888502050888805070706000088BC
:1013B000885020202020050707060000F80810208C
:1013C0004080F80309090601FFE08080808080806A
:1013D00080E0050707060000804040201010080349
:1013E00009090601FFE020202020202020E005033D
:1013F000030600052050880501010600FEF80303DE
:1014000003060105804020050505060000700878E8
:1014100088780507070600008080F0888888F00536
:10142000050506000070808088700507070600002B
:10143000080878888888780505050600007088F017
:101440008070050707060000304840E04040400536
:1014500007070600FE708888887808700507070669
:1014600000008080F0888888880307070601004014
:1014700000C0404040E00409090601FE10003010A1
:10148000101010906005070706000080808890E02B
:101490009088030707060100C04040404040E00537
:1014A0000505060000D0A8A8A8A8050505060000A7
:1014B000B0C888888805050506000070888888708F
:1014C0000507070600FEF0888888F080800507077A
:1014D0000600FE788888887808080505050600005B
:1014E000B0C880808005050506000078807008F08F
:1014F0000507070600002020F82020201805050514
:101500000600008888889868050505060000888818
:101510008850200505050600008888A8A850050504
:101520000506000088502050880507070600FE8841
:10153000888850204080050505060000F8102040EE
:10154000F80309090601FF20404040804040402048
:101550000109090602FF80808080808080808003EE
:1015600009090601FF8040404020404040800503BB
:101570000306000248A890FF5045544700504C41D4
:10158000004E65787420506F696E74002569202FB5
:101590002025750047323953310047323953320024
:1015A000436C69636B20746F20426567696E005AF3
:1015B0002056616C756500496E6465782059004954
:1015C0006E64657820580053746F7265205365749B
:1015D00074696E6773004C6F61642053657474693D
:1015E0006E677300426564205472616D6D696E6749
:1015F00000426564205A0046616465204865696759
:101600006874004F6666004F6E00426564204C654A
:1016100076656C696E670045646974204D65736812
:10162000004C6576656C20426564004D6F74696F8F
:101630006E00526573746F72652044656661756CE7
:101640007473004C6F61642053657474696E6773C2
:101650000053746F72652053657474696E6773000C
:10166000416476616E6365642053657474696E6766
:1016700073004D61696E00313235003500424544DA
:101680003A204550434F53203130304B0052756E55
:10169000617761792057617463683A204F4E004D3D
:1016A00061782054656D7000323630004D696E20CF
:1016B00054656D7000350045313A204550434F5315
:1016C000203130304B005053550047656E657269CC
:1016D000630050726F746F636F6C00312E30004284
:1016E00061756400313135323030004D656C7A6996
:1016F0002028437265616C69747929004D657368AF
:10170000204C6576656C696E670045787472756407
:101710006572730031006769746875622E636F6D5E
:101720002F6B61642F4D61726C696E2F77696B69E5
:10173000004D656761205A65726F00323032312D7D
:1017400030392D303300322E302E392E332D6B614F
:101750006431004D61726C696E00546865726D6928
:1017600073746F727300426F61726420496E666FAA
:10177000005072696E74657220496E666F004D612B
:10178000696E003F004261636B0053746F70004DDF
:10179000323200417474616368204D656469610090
:1017A0004D3231005072696E742066726F6D204D3B
:1017B000656469610052656C65617365204D65649F
:1017C00069610041626F7574205072696E74657250
:1017D00000436F6E66696775726174696F6E00545D
:1017E000656D7065726174757265004D6F74696FB7
:1017F0006E00526573756D65205072696E74005489
:10180000756E650053746F70205072696E7400506D
:1018100061757365205072696E7400496E666F2041
:1018200053637265656E000A4D3234004D323320C9
:101830002573003F005374617274205072696E7496
:101840000043616E63656C005072696E74004361A1
:101850006E6E6F7420656E74657220737562646954
:10186000723A200002202E2E0001526566726573C6
:1018700068004D61696E002100486F74656E6420D8
:10188000746F6F20636F6C64004261636B00507211
:101890006F63656564004D6F74696F6E00446973B2
:1018A00061626C65205374657070657273004D38A9
:1018B0003400426564204C6576656C696E6700474C
:1018C00032385A004732385900486F6D6520400061
:1018D00047323858004175746F20486F6D65004776
:1018E0003238004D61696E00507265686561742020
:1018F000242042656400507265686561742024206C
:10190000456E640054656D70657261747572650032
:101910007D157815436F6F6C646F776E005072653C
:101920006865617420240046616E205370656564AB
:1019300000426564004E6F7A7A6C65004D61696E95
:10194000004261627973746570205A00466C6F774B
:101950000046616E20537065656400426564004E08
:101960006F7A7A6C6500426564205A005370656531
:1019700064004D61696E00486F6D696E6720466155
:10198000696C6564006F70656E0054524947474545
:10199000524544003A20007A5F6D696E00795F6DB0
:1019A000696E00785F6D696E005265706F72746960
:1019B0006E6720656E6473746F70207374617475E4
:1019C000730A0020746F6F206C6F6E6720657874E7
:1019D000727573696F6E2070726576656E7465647A
:1019E0000A0020636F6C6420657874727573696F88
:1019F0006E2070726576656E7465640A0057617258
:101A00006E696E673A20486F6D696E672042756D2A
:101A1000702044697669736F72203C20310A00029D
:101A20000204000040C10000E0C00000000000000F
:101A300068430000634300007A430000A0400000B8
:101A4000A04000000040FFFDFCFAF8F6F4F2F0EED2
:101A5000ECEAE9E7E5E3E1E0DEDCDAD9D7D5D4D298
:101A6000D0CFCDCBCAC8C7C5C3C2C0BFBDBCBAB931
:101A7000B7B6B4B3B2B0AFADACAAA9A8A6A5A4A29C
:101A8000A1A09E9D9C9A99989795949392908F8EE1
:101A90008D8B8A8988878684838281807F7E7D7B07
:101AA0007A797877767574737271706F6E6D6C6B0E
:101AB0006A696867666564636261605F5E5D5C5BFE
:101AC0005A5958585756555453525150504F4E4DDD
:101AD0004C4B4A4A494847464645444342424140A6
:101AE0003F3E3E3D3C3B3B3A39383837363535345E
:101AF0003332323130302F2E2E2D2C2B2B2A292908
:101B000028272726252524232322212120201F1EA4
:101B10001E1D1C1C1B1B1A19191818171616151533
:101B200014131312121111100F0F0E0E0D0D0C0CB9
:101B30000B0A0A0909080807070606050504040335
:101B4000030202010000000000010000000100008B
:101B50008000555555000000400033333300AAAAD9
:101B60002A004992240000002000C7711C009999A6
:101B70001900D1451700555515003BB113002449F4
:101B8000120011111100000010000F0F0F00E338B8
:101B90000E0043790D00CCCC0C00C3300C00E8A241
:101BA0000B0064210B00AAAA0A00703D0A009DD810
:101BB0000900427B090092240900DCD308008888D0
:101BC00008001042080000000800F0C107008787E5
:101BD000070075500700711C07003EEB0600A1BC12
:101BE00006006990060066660600703E06006118F1
:101BF000060017F4050074D105005BB00500B29033
:101C00000500627205005555050078390500B81EBB
:101C10000500050505004EEC040087D40400A1BDB5
:101C2000040090A7040049920400C17D0400EE69FD
:101C30000400C7560400444404005C320400082138
:101C4000040041100400000004003FF00300F8E02D
:101C5000030026D20300C3C30300CCB503003AA897
:101C600003000A9B0300388E0300C08103009F75A8
:101C70000300D0690300505E03001D530300344885
:101C80000300913D03003333030016290300381F7E
:101C9000030097150300300C0300030303000BFA45
:101CA000020049F10200BAE802005CE002002DD80F
:101CB00002002DD0020059C80200B0C0020031B9A4
:101CC0000200DAB10200AAAA0200A0A30200BC9C92
:101CD0000200FA9502005C8F0200DF880200828217
:101CE0000200457C02002776020027700200436A4A
:101CF00002007C640200D05E02003F590200C8531B
:101D0000020000005C4300005C4300007A430000D6
:101D100040C10000E0C00000000053657474696EAB
:101D200067732053746F726564000000FA4300000B
:101D3000FA430000A0400000C8410000A04200009B
:101D4000A0420000C8430080C043F4010000F40139
:101D50000000640000008813000024F4D43050C355
:101D60008E20C2A24017828B7011127A910D816C65
:101D7000D90AA861E108C7586607615143061E4B9E
:101D80005D05C145A7041A411104093D9803713945
:101D900031034036DB0265339102D4305402802E89
:101DA0001D02632CEE01752AC501B028A001102781
:101DB00081018F2564012B244B01E0223401AC21E9
:101DC0001F018D200D01801FFC00841EED00971D5A
:101DD000DF00B81CD200E61BC600201BBC00641A42
:101DE000B200B219A8000A19A0006A189900D11708
:101DF000910040178B00B516840031167E00B31594
:101E000079003A157300C7146F0058146A00EE1376
:101E100066008813630025135E00C7125B006C1216
:101E2000570015125400C111510070114F002111BB
:101E30004B00D61049008D10470046104400021098
:101E40004200C00F4000800F3E00420F3C00060FD2
:101E50003B00CB0E3800930E37005C0E3500270E8A
:101E60003400F30D3200C10D3100900D3000600DD3
:101E70002E00320D2D00050D2C00D90C2B00AE0CC0
:101E80002900850C29005C0C2700350C27000E0C5E
:101E90002600E80B2400C40B2400A00B23007D0BBC
:101EA00023005A0B2100390B2100180B2000F80ADF
:101EB0001F00D90A1E00BB0A1E009D0A1D00800AD1
:101EC0001D00630A1C00470A1B002C0A1B00110A94
:101ED0001A00F7091A00DD091900C4091900AB0935
:101EE0001900920917007B091800630917004C09B3
:101EF000160036091600200916000A091500F50813
:101F00001500E0081400CC081400B8081400A40858
:101F10001400900813007D0812006B081300580885
:101F2000120046081200340811002308110012089C
:101F3000110001081100F0071000E0071000D007A1
:101F40001000C0071000B0070F00A1071000910794
:101F50000E0083070F0074070F0065070E00570778
:101F60000E0049070E003B070D002E070E0020074C
:101F70000D0013070D0006070D00F9060C00ED0615
:101F80000D00E0060C00D4060C00C8060C00BC06D0
:101F90000C00B0060C00A4060B0099060C008D0680
:101FA0000B0082060B0077060B006C060B00610627
:101FB0000A0057060B004C060A0042060A003806C3
:101FC0000A002E060A0024060A001A060A00100655
:101FD000090007060A00FD050900F4050900EB05E4
:101FE0000900E2050900D9050900D0050900C70567
:101FF0000900BE050900B5050800AD050800A505E6
:1020000009009C050800940508008C05080084055B
:1020100008007C050800740508006C0507006505CC
:1020200008005D050700560508004E050700470536
:1020300007004005080038050700310507002A059C
:102040000700230507001C050600160507000F05FD
:1020500007000805060002050700FB040600F5045A
:102060000700EE040600E8040600E2040700DB04B3
:102070000600D5040600CF040600C9040600C30408
:102080000600BD040600B7040600B1040500AC0458
:102090000600A6040600A00405009B0406009504A3
:1020A0000500900406008A040500850405008004EC
:1020B00006007A04050075040500700405006B0431
:1020C000050066040500610405005C040500570472
:1020D0000500520405004D040500480405004304B2
:1020E00005003E0404003A040500350405003004F0
:1020F00004002C04050027040400230405001E042A
:1021000004001A04040016040500110404000D0460
:102110000400090405000404040000040400FC0396
:102120000400F8030400F4030400F0030400EC03CB
:102130000400E8030400E4030400E0030400DC03FB
:102140000400D8030400D4030400D0030400CC032B
:102150000400C8030300C503030024F404D9201BB2
:10216000C40C5C0E9804C4095F0265077101F40594
:10217000F900FB04B30048048700C1036900580359
:10218000550003034500BE023A00840231005302A9
:102190002A002902250004022000E4011C00C801D5
:1021A0001900AF0117009801140084011300710198
:1021B00010006101100051010E0043010D003601B5
:1021C0000B002B010B0020010B00150109000C0175
:1021D000090003010800FB000800F3000800EB0001
:1021E0000700E4000600DE000600D8000600D2006A
:1021F0000600CC000500C7000500C2000500BD00B8
:102200000400B9000400B5000400B1000400AD00F2
:102210000400A9000400A5000300A20003009F0021
:1022200004009B0003009800030095000200930047
:102230000300900003008D0002008B000300880063
:1022400002008600020084000300810002007F007B
:1022500002007D0002007B0002007900020077008E
:10226000010076000200740002007200010071009B
:1022700002006F0002006D0001006C0002006A00A5
:1022800001006900020067000100660001006500AE
:1022900001006400020062000100610001006000B2
:1022A00001005F0002005D0001005C0001005B00B6
:1022B00001005A00010059000100580001005700B8
:1022C00001005600010055000100540001005300B8
:1022D00000005300010052000100510001005000B5
:1022E00001004F0001004E0000004E0001004D00B3
:1022F00001004C0001004B0000004B0001004A00AF
:1023000001004900010048000000480001004700AA
:1023100001004600000046000100450000004500A5
:10232000010044000100430000004300010042009E
:102330000000420001004100000041000100400097
:1023400001003F0000003F0001003E0000003E0091
:1023500001003D0000003D0001003C0000003C0089
:1023600000003C0001003B0000003B0001003A007F
:1023700000003A0001003900000039000100380077
:10238000000038000000380001003700000037006E
:102390000100360000003600000036000100350064
:1023A000000035000000350001003400000034005A
:1023B000000034000100330000003300000033004F
:1023C0000100320000003200000032000100310044
:1023D000000031000000310001003000000030003A
:1023E0000000300001002F0000002F0000002F002F
:1023F00000002F0001002E0000002E0000002E0023
:1024000001002D0000002D0000002D0000002D0017
:1024100001002C0000002C0000002C0000002C000B
:1024200001002B0000002B0000002B0000002B00FF
:1024300001002A0000002A0000002A0000002A00F3
:1024400001002900000029000000290000002900E7
:1024500000002900010028000000280000002800DA
:1024600000002800000028000100270000002700CD
:1024700000002700000027000000270001002600C0
:1024800000002600000026000000260000002600B4
:1024900001002500000025000000250000002500A7
:1024A0000000250000002500010024000000240099
:1024B000000024000000240000002400010023008C
:1024C0000000230000002300000023000000230080
:1024D0000000230000002300010022000000220071
:1024E0000000220000002200000022000000220064
:1024F0000100210000002100000021000000210057
:102500000000210000002100000021000100200047
:10251000000020000000200000002000000020003B
:1025200000002000000020000000200001001F002B
:1025300000001F0000001F0000001F0000001F001F
:1025400000001F0000001F0001001E0000001E0010
:1025500000001E0000001E0000003930000033257E
:10256000000087190000B00F0000DB080000BD0468
:102570000000740200003F01000020436F756E747C
:1025800020583A00426564004531004500626564A8
:10259000002C2073797374656D2073746F7070658F
:1025A0006421204865617465725F49443A200045A2
:1025B00072723A204D415854454D50004D41585487
:1025C000454D50207472696767657265640048659F
:1025D0006174696E67204661696C65640048656175
:1025E00074696E67206661696C6564004572723A51
:1025F000204D494E54454D50004D494E54454D5087
:102600002074726967676572656400544845524D6D
:10261000414C2052554E4157415900546865726DE6
:10262000616C2052756E6177617900202F00204225
:10263000403A0020403A007C3C3E5E2B3D3F2F5B01
:102640005D3B2C2A225C0043616E6E6F74206F70BC
:10265000656E207375626469722000534420636163
:102660007264206F6B0A006F70656E526F6F74201A
:102670006661696C65640A00766F6C756D652E69BC
:102680006E6974206661696C65640A004E6F205340
:102690004420636172640A002E0A006F70656E2028
:1026A0006661696C65642C2046696C653A20004659
:1026B000696C652073656C65637465640A002053FA
:1026C000697A653A200046696C65206F70656E65B1
:1026D000643A2000454E4420535542524F555449C8
:1026E0004E450A002220706F7300222070617265CF
:1026F0006E743A2200535542524F5554494E45206C
:1027000043414C4C207461726765743A22005375E2
:102710006263616C6C204F766572666C6F77004502
:1027200078636565646564206D6178205355425215
:102730004F5554494E452064657074683A0066727E
:1027400065736800646F696E67002066696C653A3E
:1027500020004E6F77200057726974696E6720748D
:102760006F2066696C653A200000200000000000C0
:1027700000000000000000000000DC00000000007D
:1027800000000000000000000000EF00000000005A
:1027900000000000000000000001F7E00000000061
:1027A00000000000000000000003FBF0000000003B
:1027B00000000000000000000003FCFC000000001E
:1027C00000000000000000000007FF7E0000000085
:1027D00000000000000000000007FFBF0000808034
:1027E000EE0E1B070E338303B00FFFDF8000C0C067
:1027F000E71C7BC70E33C307B80FFFEFC001C0E073
:10280000E73CFBC70E33E30F3C1FFFF7E000E07827
:10281000E338E0870E30E30C001FFFFBF002E03CE2
:10282000E071C0070E30E31C003FFFF43002709EE1
:10283000E0E1C0070E33C31C007FFFEFC00770CF7D
:10284000E0E1C0070E33C31C003FFFEFF00638E79E
:10285000E0C1C0070E30231C001FFFDFE00EF8E3CD
:10286000E0C0E0070E30E31C001FFFBFC00CFCE01F
:10287000E0C0F1C79C33E30F1C0FFF7F801C0CE00E
:1028800060C07BC39C33C307BC07FF7F00180EE00A
:1028900020C03B8190338303B007FEFE00000000A0
:1028A00000000000000000000003FDFC000000002C
:1028B00000000000000000000001FBF80000000024
:1028C00000000000000000000001F7F00000000020
:1028D00000000000000000000000F7C00000000041
:1028E000000000000000000000006E00000000007A
:1028F0000000000000000000000050000000000088
:1029000000000000000000000000000000000000C7
:1029100000000000000000000000000000000000B7
:1029200000000000000000000000000000000FFF99
:1029300003C1FF000000000000000000000008616B
:1029400006410180000000000000000000000CE7CC
:1029500004619CC00000000000000000000004CCE6
:102960000C209640000000000000000000000498C9
:1029700009B0926000000000000000000000043078
:1029800019909320000000000000000000000430B7
:1029900013D89120000000000000000000000498FF
:1029A000300893200000000000000000000004CC6C
:1029B00027EC92600000000000000000000004E628
:1029C00064249640000000000000000000000CF3AA
:1029D000CC379CC00000000000000000000008612F
:1029E00084230180000000000000000000000FFFB1
:1029F000FC3FFF000000000000000000000000009D
:102A000000000000000000000000000000000000C6
:102A10000000000000000000000000FC7E0000003C
:102A2000000FFE000000000000000086C200000051
:102A30000008020000000000000000C38600000043
:102A40000009F2000000000000000043840001F0D3
:102A5000000B62000000000000000049247F1F17E7
:102A6000F80EC67F7FE3F8000000004924C1B07C67
:102A70000C018CC1C4360C000000004C659CE73989
:102A8000E403199CE19CE6000000004C653CCD9FEE
:102A9000E406313CA399B2000000004EE501CD9C54
:102AA000040C6F01A6F912000000004FE53FE77922
:102AB000E408DB3FA409B200000000CC679CB0E949
:102AC000C609F39CE60CE6000000008442C1EF3C1E
:102AD000120802C1C2060C00000000FC7E7F4D9768
:102AE000FE0FFE7F7E03F80000000000000047108C
:102AF00000000000000000000000000000007070F6
:102B000000000000000000000000000000001FC0E6
:102B10000000000000000000006D61726C696E66CC
:102B2000772E6F726700322E302E392E332D6B6167
:102B30006431001FFFFFFFFFFFFF60000000000186
:102B4000FF400000000000FF8000000000007F83C5
:102B5000CF00000C303F87FF80000C301F8679804B
:102B6000000C000F8C30C7838C30E78C30CFC7CC83
:102B700031F38C30DCECEC33B98C30D86C6C33191D
:102B80008C30D06C0C33198C30D86C0C33198C30E1
:102B9000DC6C0E3B198C30CF7C079F198C30C77CC6
:102BA000038F1940000000000002600000000000D8
:102BB000061FFFFFFFFFFFF870012C0190012701A6
:102BC000B0012201C0011D01F00118011002130122
:102BD00030020E016002090190020401C002FF00F0
:102BE0000003FA004003F5008003F000D003EB007F
:102BF0002004E6007004E100E004DC004005D7009A
:102C0000C005D2004006CD00D006C8008007C30032
:102C10003008BE00F008B900C009B400B00AAF0027
:102C2000B00BAA00D00CA500000EA000500F9B0016
:102C3000C01096005012910000148C00C01587003F
:102C4000B0178200B0197D00D01B7800001E730001
:102C500040206E0090226900F024640040275F004D
:102C600090295A00E02B5500102E500020304B00C8
:102C700010324600E033410090353C0010373700F9
:102C800070383200A0392D00B03A2800A03B230054
:102C9000603C1E00103D1900903D1400103E0F00D6
:102CA000703E0A00C03E0500003F0000403FFBFFB1
:102CB000803FF6FFC03FF1FF2020506C616E6E65D3
:102CC0007242756666657242797465733A200020B7
:102CD00046726565204D656D6F72793A200020431C
:102CE0006F6D70696C65643A2044656320323720EB
:102CF000323032310A00204C6173742055706461A7
:102D00007465643A20323032312D30392D30332021
:102D10007C20417574686F723A20286B61642C20A6
:102D2000416E796375626963204D656761205A65FC
:102D3000726F204D424C20313256290A004D61728B
:102D40006C696E20322E302E392E332D6B6164313A
:102D50000A0020536F66747761726520526573654F
:102D6000740A00205761746368646F67205265734A
:102D700065740A002042726F776E206F757420525E
:102D8000657365740A002045787465726E616C2005
:102D900052657365740A00506F77657255700A004A
:102DA00073746172740A004732385859004D3130DB
:102DB0003031006572726F722077726974696E6764
:102DC00020746F2066696C650A00446F6E6520731D
:102DD0006176696E672066696C652E0A00456E64CF
:102DE00073746F707300255320256320256320259D
:102DF0006320256300205A3A0020593A0020583AAF
:102E000000656E6473746F7073206869743A200093
:102E1000004D6F76652025736D6D004D6F766520D2
:102E2000302E316D6D004D6F766520316D6D004D2A
:102E30006F76652031306D6D004D6F76652041787D
:102E40006973004D6F76652045787472756465729C
:102E5000004D6F7665205A004D6F76652059004D04
:102E60006F76652058005072696E742066726F6DBF
:102E7000204D6564696100FFFFFF4D656761205A61
:102E800065726F2052656164792E005072696E74AC
:102E9000696E672E2E2E005072696E742050617517
:102EA00073656400204500205A0020590020204D01
:102EB0003932205800537465707320706572207524
:102EC0006E6974003B2000220A00556E6B6E6F77AE
:102ED0006E20636F6D6D616E643A2022006F6B002F
:102EE000627573793A2070617573656420666F72DC
:102EF00020696E7075740A00627573793A2070618A
:102F00007573656420666F7220757365720A00625E
:102F10007573793A2070726F63657373696E670AAF
:102F2000004D6564696120496E7365727465640063
:102F3000000000010200090A000000000403080765
:102F40000000000000000000000000000000000081
:102F50004D3131322053687574646F776E0053546D
:102F60004F505045442E20005072696E7465722097
:102F700073746F707065642064756520746F20656C
:102F800072726F72732E20466978207468652065AE
:102F900072726F7220616E6420757365204D3939CD
:102FA0003920746F20726573746172742E202854F6
:102FB000656D7065726174757265206973207265E4
:102FC0007365742E2053657420697420616674657E
:102FD000722072657374617274696E67290A004E9B
:102FE0006F20436865636B73756D20776974682023
:102FF0006C696E65206E756D6265722C204C617314
:1030000074204C696E653A20004D3239004E6F20B5
:10301000436865636B73756D2077697468206C69AC
:103020006E65206E756D6265722C204C6173742024
:103030004C696E653A2000636865636B73756D203B
:103040006D69736D617463682C204C617374204CDE
:10305000696E653A20004C696E65204E756D62653B
:1030600072206973206E6F74204C617374204C69F8
:103070006E65204E756D6265722B312C204C61732C
:1030800074204C696E653A20004D31313000536533
:103090007269616C20737461747573206D69736DEE
:1030A000617463680A00534420726561642065722C
:1030B000726F720A002121204B494C4C20636175CC
:1030C00073656420627920746F6F206D756368206A
:1030D000696E6163746976652074696D65202D2061
:1030E00063757272656E7420636F6D6D616E643AA4
:1030F0002000DB0FC93F45BCDA3F8FB30240FCF034
:10310000274056946140FE4B9B4084A5D840E02365
:103110001841346A5641E859974164DBD5416E271E
:103120001742B4B75542CE1A9742C8AED542B588B9
:103130005A43D40684BFA65FA7BF7443E0BF10B153
:103140001AC01C2C58C0E8F697C0B849D6C04E4EDD
:1031500017C124D355C1802497C1A0B5D5C1121A77
:1031600017C244AE55C2781797C26CACD5C26788F7
:103170005AC320746F6F206C6F6E6720657874720D
:103180007573696F6E2070726576656E7465640A1A
:103190000020636F6C6420657874727573696F6E5C
:1031A0002070726576656E7465640A006F6B0A0044
:1031B000526573656E643A200020453A00205A3A01
:1031C0000020593A00583A0000002200250028004B
:1031D0002B0000002100240027002A000202020226
:1031E00002020202040404040404040403030303AB
:1031F00003030303010101010101010101020408AC
:1032000010204080010204081020408001020408C0
:103210001020408080402010080402014572726F27
:10322000722077726974696E6720746F204545500B
:10323000524F4D210A001FDCCCE211241FBECFEFFC
:10324000D0E4DEBFCDBF84B780939D1414BE0FB60B
:10325000F894A89580916000886180936000109236
:1032600060000FBE12E0A0E0B1E0E6ECF1EE01E09C
:103270000BBF02C007900D92A036B107D9F724E129
:10328000A0E6B2E001C01D92AD39B207E1F719E145
:10329000CCE1D9E104C02197FE010E942BEECB3195
:1032A000D107C9F70E9410DD0C94D7F00C940000F0
:1032B000CF93DF93EC01CB01BA010E946CE72DECB8
:1032C0003CEC4CEC5DE30E94CBE7688379838A8316
:1032D0009B83DF91CF910895CF93DF93EC01CB01D6
:1032E000BA010E946CE72DEC3CEC4CEC5DE30E94D3
:1032F000CBE7688379838A839B83DF91CF9108959D
:10330000CF93DF93EC01CB01BA010E946CE72AE076
:1033100037ED43E25CE30E94CBE7688379838A83DD
:103320009B83DF91CF910895CF93DF93EC01CB0185
:10333000BA010E946CE72AE037ED43E25CE30E94A9
:10334000CBE7688379838A839B83DF91CF9108954C
:10335000CF93DF93EC01CB01BA010E946CE70E948E
:1033600063EF79836883DF91CF91089520E030E5A2
:1033700043EC50E46091290470912A0480912B045D
:1033800090912C040E94CBE76093641170936511B7
:10339000809366119093671108952CEA35EC47E20B
:1033A0005EE360912D0470912E0480912F04909122
:1033B00030040E94CBE76093601170936111809399
:1033C000621190936311089520E030E543EC50E4DE
:1033D0006091290470912A0480912B0490912C040F
:1033E0000E94CBE76093641170936511809366111E
:1033F0009093671108952CEA35EC47E25EE3609103
:103400002D0470912E0480912F04909130040E941D
:10341000CBE7609360117093611180936211909378
:10342000631108958F929F92AF92BF92CF92DF92D5
:10343000EF92FF92FC01C080D180E280F38020E017
:1034400030E0A901C701B6010E9466E787FD99C077
:103450006DEB77E386E095E3A70196010E9484EE89
:103460006B017C0120E030E04AE754E40E94CBE7A6
:103470004B015C0120E030E0A901C701B6010E94C8
:1034800066E720E030E040EA50E487FF04C020E037
:1034900030E040EA50ECC501B4010E9484EE2DEC0E
:1034A0003CEC4CEC5DE30E94CBE70E9463EF6B01C8
:1034B0007C018BE2F7FE09C0F094E094D094C094B4
:1034C000C11CD11CE11CF11C8DE280933D04C7019D
:1034D000B60120E137E240E050E00E940FEE8AE0C2
:1034E000882E912CA12CB12CCA01B901A5019401FF
:1034F0000E940FEE605D60933E04C701B60128EEA6
:1035000033E040E050E00E940FEECA01B901A5018E
:1035100094010E940FEE605D60933F04C701B60105
:1035200024E630E040E050E00E940FEECA01B9010D
:10353000A50194010E940FEE605D609340048EE24D
:1035400080934104C701B601A50194010E940FEECA
:103550006B01CA01B901A50194010E940FEE605DE3
:1035600060934204F0E3CF0EC09243048DE394E0F5
:10357000FF90EF90DF90CF90BF90AF909F908F9093
:1035800008956DEB77E386E095EB66CFA4E0B0E0BD
:10359000ECECFAE10C945CEE0E946CE72AE037ED6B
:1035A00043E25CE30E94CBE769837A838B839C834D
:1035B000CE01019637DF2496E2E00C9478EE8F92EC
:1035C0009F92AF92BF92CF92DF92EF92FF92FC0157
:1035D000C080D180E280F38020E030E0A901C70103
:1035E000B6010E9466E787FD99C06DEB77E386E040
:1035F00095E3A70196010E9484EE9F7720E030E0DA
:1036000048EC52E40E94CBE720E030E040EA50E48E
:103610000E9484EE2DEC3CEC4CEC5DE30E94CBE789
:103620000E9463EF6B017C0180E280933D0460E2C5
:10363000F0E1CF16F7E2DF06E104F1048CF0C701F8
:10364000B60120E137E240E050E00E940FEECA01EF
:10365000B9012AE030E040E050E00E940FEE605DEA
:1036600060933E0460E288EEC81683E0D806E10469
:10367000F1048CF0C701B60128EE33E040E050E0E1
:103680000E940FEECA01B9012AE030E040E050E0AC
:103690000E940FEE605D60933F0460E2E4E6CE16A8
:1036A000D104E104F1048CF0C701B60124E630E056
:1036B00040E050E00E940FEECA01B9012AE030E07C
:1036C00040E050E00E940FEE605D609340048AE0AD
:1036D000882E912CA12CB12CC701B601A501940113
:1036E0000E940FEE6B01CA01B901A50194010E946D
:1036F0000FEE605D609341048EE280934204F0E33C
:10370000CF0EC09243048DE394E0FF90EF90DF90E2
:10371000CF90BF90AF909F908F9008956DEB77E31F
:1037200086E095EB66CFA4E0B0E0E9E9FBE10C941C
:103730005CEE0E946CE72DEC3CEC4CEC5DE30E94EF
:10374000CBE769837A838B839C83CE01019637DF35
:103750002496E2E00C9478EEFC0184910895FC013B
:1037600080810895FC01A081B1811C92A281B38166
:103770008C918F5F8C930280F381E02D90818CE09F
:10378000989F800D1124E8EFF1E113AE84AF089506
:10379000119800C087FD43C0419800C0119A00C035
:1037A00000C0119800C086FD46C0419800C0119A23
:1037B00000C000C0119800C085FD3BC0419800C00A
:1037C000119A00C000C0119800C084FD30C041981B
:1037D00000C0119A00C000C0119800C083FD25C030
:1037E000419800C0119A00C000C0119800C082FD2D
:1037F0001AC0419800C0119A00C000C0119800C0C2
:1038000081FD0FC0419800C0119A00C000C01198FE
:1038100000C0419800C0119A00C000C00895419AAC
:10382000BCCF419AF0CF419AE5CF419ADACF419A85
:10383000CFCF419AC4CF419AB9CF90E080E00895AC
:1038400090E080E0089520917803833021F425FDF5
:103850000CC024FD0CC030E0A90102C0559547956D
:103860008A95E2F7CA018170089581E0089580E0A9
:1038700008958091930384FD0BC08091950387FD8B
:1038800007C090919603937081E019F480E0089549
:1038900081E008952FEB280F2A3108F047C0E22F6E
:1038A000F0E08091930390919403A0919503B091DF
:1038B000960304C0B695A795979587952A95D2F754
:1038C00080FD02C081700895E758FC4FE081EE232F
:1038D00041F18091F6059091F705E80FF92FF11D60
:1038E000808190ED980F9A3030F08E3251F48181C2
:1038F00080538A3098F4F0937103E093700381E071
:1039000008958D3211F08B3249F4818190ED980F3A
:103910009A3088F38E3211F48281EACFF0E0E0E051
:10392000EACF1092710310927003E9CF80E00895FE
:10393000CF93DF9385E4AEDF882309F188E04091DF
:103940009303509194036091950370919603972F80
:103950009170C92F90E0D92FCC0FDD1F71FB22276A
:1039600020F930E0220F331F220F331FC22B67FBD9
:10397000442740F9C42B8C2BDF91CF91089580E030
:10398000DECF88DF882341F081E020917003309101
:103990007103232B09F480E0089580E090E0A0E813
:1039A000B0E48093750190937601A0937701B09372
:1039B000780189EB91E00E94549F80E090E0A0EFB5
:1039C000B1E480936D0190936E01A0936F01B09369
:1039D00070018093710190937201A0937301B09371
:1039E0007401E0913204EE0FFF0BE756FE4F808129
:1039F00091818330910549F184309105D9F1029785
:103A000061F480E090E0AEE3B3E480936D019093C5
:103A10006E01A0936F01B093700181EA91E00E9462
:103A2000549F1092750110927601109277011092B6
:103A3000780189EB91E00E94549F809132048F5F5E
:103A40008430ECF480933204089580E090E0AEE39B
:103A5000B3E480936D0190936E01A0936F01B093D6
:103A600070018093710190937201A0937301B093E0
:103A70007401D3CF80E090E0AEE3B3E4F2CF1092D4
:103A8000320408950C94F68C0C94F68C0C94F68CFD
:103A90000C94F68CCF92DF92EF92FF92CF93DF934C
:103AA00000D000D0CDB7DEB7FC01C080D180E2806D
:103AB000F38020E030E0A901C701B6010E9466E76B
:103AC00087FD1BC06DEB77E386E095E3A7019601C8
:103AD0000E9484EE69837A838B839C83CE01019656
:103AE0000E946BA70F900F900F900F90DF91CF91D6
:103AF000FF90EF90DF90CF9008956DEB77E386E035
:103B000095EBE4CFA4E0B0E0E8E8FDE10C945CEED6
:103B10000E946CE72DEC3CEC4CEC5DE30E94CBE7A3
:103B200069837A838B839C83CE010196B3DF2496CD
:103B3000E2E00C9478EE882361F063E972E084E6B9
:103B400090E00E947FAC6AEB72E084E690E00C9417
:103B50007FAC68EB71E084E190E0F9CFCF93DF9325
:103B6000C0919805D0919905209729F1609194050D
:103B70007091950580919605909197050E9463EF4D
:103B80006E5F7F4F24976C177D07ACF4709396049B
:103B9000609395040E9465BC605A75418F4F9F4F9A
:103BA00060939704709398048093990490939A0477
:103BB000DF91CF910895109297041092980410927B
:103BC000990410929A04F4CF0E94048AB4CF0E9400
:103BD0001AA581E0B0CF0E940AA6ADCFB0E0A0E068
:103BE000E4EFFDE10C9455EE6B01E9014A3009F474
:103BF000D5C0453109F081C0DB011296ED91FC91F1
:103C0000F28096818781139A00C00000E6E2F0E01E
:103C10003197F0F7092F182FEF2CE29420EFE222D2
:103C200030E1B32EBF0CE80188EFB2DD00C0000028
:103C300086E290E00197F0F7BFE1BF1508F49BC062
:103C40008F2D80778068A4DD8E2DA2DD00C000005E
:103C500086E290E00197F0F780E89ADD80E098DD59
:103C600000C0000086E290E00197F0F78AEF90DD57
:103C700000C0000086E290E00197F0F7005F1F4F60
:103C80008881807F85DD89918295807F81DDC01765
:103C9000D107B1F700C0000086E290E00197F0F78D
:103CA000F394E0E1EE0EFB10BECF1398D60112960E
:103CB000ED91FC9180819281980F928321819217DE
:103CC00008F09FC194819F5F94839381890F82172D
:103CD00010F08FEF820F8383458150E0440F551F12
:103CE00070E060E0868197810E9483F081E0CDB72B
:103CF000DEB7E9E00C9471EEDEC1FB0102811381B5
:103D0000423309F485C108F48DC1463409F475C104
:103D1000473409F482C14B3349F789812B81D8019B
:103D200012967C91129713963C91213009F4BFC1F1
:103D3000233009F0A0C148EF480F582F91E0341705
:103D400008F490E031E0541708F030E0492F432B9D
:103D500061E0571708F460E0462311F4932331F231
:103D6000FA8030E0F901EB57FE4FD0802F573E4FDD
:103D7000F901E08099C180EE8F0D8068807F08DDB9
:103D80008F2D8295807F04DD00C0000086E290E0E8
:103D90000197F0F780E8FCDC80E861CF0B9A13987C
:103DA000399A4198099A119A139A00C0000086E244
:103DB00090E00197F0F788E790E0CEE9DFE0FE01C0
:103DC0003197F1F70197D9F788EFE2DC00C00000E6
:103DD00086E290E00197F0F780E2DADC80E0D8DC60
:103DE00000C0000086E290E00197F0F780E0D0DCB0
:103DF00080E8CEDC00C0000086E290E00197F0F79A
:103E000080E0C6DC80E1C4DC00C0000086E290E017
:103E10000197F0F7CE010197F1F7CE010197F1F785
:103E2000CE010197F1F7CE010197F1F7CE0101978D
:103E3000F1F7CE010197F1F7CE010197F1F7CE012D
:103E40000197F1F7CE010197F1F7CE010197F1F754
:103E5000CE010197F1F7CE010197F1F7CE0101975D
:103E6000F1F7CE010197F1F72197F1F780E290DCAD
:103E700080E48EDC00C0000086E290E00197F0F75D
:103E800080E286DC80E684DC00C0000086E290E010
:103E90000197F0F7D0E0C0E08C2F8077806878DC65
:103EA0008D2F76DC00C0000086E290E00197F0F7ED
:103EB00080E86EDC80E06CDC00C0000086E290E010
:103EC0000197F0F78AEF64DC00C0000086E290E022
:103ED0000197F0F780E2119800C0419800C0119A54
:103EE00000C000C0119800C0419800C0119A00C0E5
:103EF00000C0119800C0419800C0119A00C000C0D5
:103F0000119800C0419800C0119A00C000C01198DB
:103F100000C0419800C0119A00C000C0119800C0B4
:103F2000419800C0119A00C000C0119800C041988B
:103F300000C0119A00C000C0119800C0419800C094
:103F4000119A00C000C0119800C0419800C0119A99
:103F500000C000C0119800C0419800C0119A00C074
:103F600000C0119800C0419800C0119A00C000C064
:103F7000119800C0419800C0119A00C000C011986B
:103F800000C0419800C0119A00C000C0119800C044
:103F9000419800C0119A00C000C0119800C041981B
:103FA00000C0119A00C000C0119800C0419800C024
:103FB000119A00C000C000C00000E6E2F0E03197B6
:103FC000F0F7815009F087CF88EFE2DB00C00000F6
:103FD00086E290E00197F0F7CF5FD05FC03209F042
:103FE0005BCF80E0D5DB80ECD3DB00C0000086E255
:103FF00090E00197F0F7139879CEF80185818883D6
:1040000075CE80E0CDB7DEB7E9E00C9471EE53C019
:10401000B901C8010E9463BD69CED80111968C9187
:10402000888364CE443191F0473109F05FCE188225
:10403000D80112968C911297898315968C911597B9
:1040400081508A8313968C918B8350CED80115961C
:104050004C91159750E0440F551F70E060E01696A4
:104060008D919C910E9483F0F80112828081815091
:10407000838314823BCE381708F438CE871708F4B0
:1040800035CEFA80E12CD12C243070F46ACEBE01FA
:10409000C8010E9463BD898198819D0D98838E0D12
:1040A0008983FF0C09F422CEF7FEF6CFF0CF58E05B
:1040B000580F482F43CEEF92FF920F931F93CF9349
:1040C000DF93EC018B017A018A859B858617970720
:1040D00031F0888199810E9450BF1B870A87B70100
:1040E000888199810E941EB82E813F81820F932F73
:1040F000911D9F838E8390E080E0CDB7DEB7E6E030
:104100000C9474EEB0E0A0E0E8E8F0E20C9454EE19
:10411000EC017B018A018A859B858617970731F020
:10412000888199810E9450BFFB86EA86888599859F
:10413000019609F5CC80DA808E81D80EA880B980EE
:10414000D5015596ED91FC91C5010995C80E7801F0
:1041500010E0F70121917F0121111FC08E819F8105
:10416000810F911D9F838E8390E080E0CDB7DEB7F5
:10417000EAE00C9470EEEE80FF80B80188819981AE
:104180000E941EB88E0D9F2D911D288539852817F8
:10419000390780F681E090E0E9CF4C2D6D2DC50107
:1041A0000E94A8BFD80E180FD4CFB0E0A0E0EBED6E
:1041B000F0E20C9457EEEC01D62E1CAD0BAD7C0159
:1041C00084E0E80EF11CE98DFA8DC7010995412FB5
:1041D000480F2D2D602FC7010E94A8BF9BAD890FEE
:1041E0008BAF81E090E0CDB7DEB7E7E00C9473EEE3
:1041F000682F70E090E080E00C94DBB08091700359
:1042000090917103009731F04AE050E070E060E077
:104210000C9487E560E070E0CB0108958091700315
:1042200090917103009731F04AE050E070E060E057
:104230000C945AE460E070E0CB010895EFDF97FD45
:104240000AC0ECDF6F3F71058105910509F02CF480
:10425000E5DF862F089580E008958FEF089580911F
:10426000700390917103892B39F0E8DF91E081119F
:1042700001C090E0892F089591E0FCCFCF93DF93A8
:10428000C82FD62F7EDB882321F0E9DFDF91CF9185
:1042900008958C2FFFDA8111F9CF8D2FF7CFBEDF74
:1042A000CB010895CF93DF93EB016BDB882311F0F3
:1042B000F6DFEC01CE01DF91CF9108950F931F93AC
:1042C000CF9380917003909171030097D9F0FC0116
:1042D0008F01C1912C2F2F7D81F0C53411F0C5368F
:1042E000B9F7F801108270E060E00E9404E3F80181
:1042F000C083CF911F910F91089570E060E00E94FC
:1043000004E3F7CF60E070E0CB01F3CFCF92DF9210
:10431000EF92FF92CF93DF9300D000D0CDB7DEB7FE
:10432000FC01C080D180E280F38020E030E0A90170
:10433000C701B6010E9466E787FD1CC06DEB77E3FD
:1043400086E095E3A70196010E9484EE69837A8353
:104350008B839C8360E2CE0101960E94D4A60F90CD
:104360000F900F900F90DF91CF91FF90EF90DF9023
:10437000CF9008956DEB77E386E095EBE3CFCF9296
:10438000DF92EF92FF92FC01C080D180E280F38047
:1043900020E030E0A901C701B6010E9466E787FD71
:1043A00027C06DEB77E386E095E3A70196010E94B5
:1043B00084EE6B017C0120E030E0A9010E9466E7F9
:1043C00020E030E040E05FE387FF04C020E030E021
:1043D00040E05FEBC701B6010E9484EE0E9463EFEC
:1043E000CB010E9482AAFF90EF90DF90CF900895BA
:1043F0006DEB77E386E095EBD8CFB0E0A0E0E3E0AB
:10440000F2E20C945CEE20E24F8158856E818D8142
:104410000E947AB7E2E00C9478EE4F925F926F922E
:104420007F928F929F92AF92BF92CF92DF92EF9244
:10443000FF92FC01C080D180E280F38020E030E078
:10444000A901C701B6010E9466E787FFA1C06DEB15
:1044500077E386E095EBA70196010E9484EE6B015D
:104460007C0120E030E04AE754E40E94CBE74B01B6
:104470005C0120E030E040E251ECC701B6010E944F
:1044800066E7181654F420E030E048EC52E4C70127
:10449000B6010E94E7EF87FD8FC020E030E0A90160
:1044A000C701B6010E9466E787FF77C060E070E051
:1044B00080EA90ECA50194010E9484EE2DEC3CEC86
:1044C0004CEC5DE30E94CBE70E9463EF6B017C0143
:1044D000F7FC68C020E137E240E050E00E940FEEB8
:1044E000CA01B9012AE030E040E050E00E940FEE3E
:1044F000605D60933E04C701B60128EE33E040E002
:1045000050E00E940FEE9AE0892E912CA12CB12C44
:10451000CA01B901A50194010E940FEE605D60938C
:104520003F04C701B60124E630E040E050E00E94BD
:104530000FEECA01B901A50194010E940FEE605D62
:10454000609340048EE280934104C701B601A50147
:1045500094010E940FEE6B01CA01B901A5019401FB
:104560000E940FEE605D60934204F0E3CF0EC092B4
:1045700043048EE394E0FF90EF90DF90CF90BF90E4
:10458000AF909F908F907F906F905F904F90089525
:104590006DEB77E386E095E35ECF60E070E080EA64
:1045A00090E488CFF094E094D094C094C11CD11CC6
:1045B000E11CF11C6DE29DCF20E030E0A901C701B4
:1045C000B6010E9466E787FF6BC060E070E080EA9A
:1045D00090ECA50194010E9484EE2DEC3CEC4CEC97
:1045E0005DE30E94CBE70E9463EF4B015C0120E09A
:1045F00030E0A901C701B6010E9466E787FD0BC044
:1046000020E030E040E251E4C701B6010E94E7EF4C
:1046100060E287FD13C0B7FC48C0C501B40128EEB5
:1046200033E040E050E00E940FEECA01B9012AE0F9
:1046300030E040E050E00E940FEE605D60933F0488
:10464000C501B40124E630E040E050E00E940FEEE6
:104650008AE0482E512C612C712CCA01B901A301AA
:1046600092010E940FEE605D609340048EE28093A1
:104670004104C501B401A30192010E940FEE6B0138
:10468000CA01B901A30192010E940FEE605D60931F
:10469000420480E3C80EC09243048FE394E06BCFE2
:1046A00060E070E080EA90E494CFB094A09490949D
:1046B0008094811C911CA11CB11C6DE2BFCFA4E0B1
:1046C000B0E0E5E6F3E20C945CEE0E946CE72AE0D1
:1046D00037ED43E25CE30E94CBE769837A838B8307
:1046E0009C83CE01019699DE2496E2E00C9478EE4C
:1046F000FC0160817181828193810E9463EFCB0113
:104700000C9482AAA4E0B0E0E8E8F3E20C945CEE3A
:104710000E946CE769837A838B839C83CE01019628
:10472000E7DF2496E2E00C9478EE4FE350E0BC0122
:104730008FE495E00C94BDF0282F1092D505809160
:10474000C0059091C105A091C205B091C305B7FF06
:1047500008C01092C0051092C1051092C2051092B7
:10476000C30580913704882331F08091C005809380
:10477000B9051092D0058091B3051816FCF4082EE7
:10478000000C990B821B91092091B905022E000C97
:10479000330B2817390794F097FF02C090E080E0B0
:1047A0008093B905092E000CAA0BBB0B8093C005A2
:1047B0009093C105A093C205B093C3058091B9053C
:1047C0006623A9F09091BA05891714F48093BA056D
:1047D0002091BA05022E000C330B2C5F3F4F482F5F
:1047E000082E000C550B241735071CF484508093B9
:1047F000BA050895E0912204E63028F581E08E0F95
:10480000809322044091C0055091C1056091C2057A
:104810007091C3052091BA059091B3058091380439
:1048200039E0E39FF0011124E551FC4FA091F6110E
:10483000B091F711B183A08342835383648375835E
:104840002683978380870895B0E0A0E0EAE2F4E24F
:104850000C945CEE8D8190913B0F891778F08093DA
:104860003B0F9E01285F3F4F4E815F8164E570E002
:1048700086EE9EE00E942EE71092E50EE2E00C9498
:1048800078EE0F931F93CF93DF936F3F11F4109245
:104890003B0F20913B0F21111EC08C010E94B5E6F9
:1048A000800F911FEC01C01BD10BC535D1053CF029
:1048B0000197FC012491207C2038D1F3F3CFDD2730
:1048C000AE01B80186EE9EE00E94D6E6CA51D14FF5
:1048D00018821092E50EDF91CF911F910F910895EC
:1048E0000F931F930E9465BC0091DF031091E003BA
:1048F0002091E1033091E203601B710B820B930B5B
:1049000097FD0CC089B183FB882780F991E0892746
:104910004A9B8260309B84608093DE038091DE033B
:1049200081709091DE0391FD82609091DD03981774
:1049300049F0813009F148F0823079F0833091F00C
:104940008093DD031F910F910895913079F092309B
:10495000B9F79091DC0391500CC0992339F0933052
:10496000C1F3EECF9130A9F3923051F79091DC036F
:104970009F5F9093DC03E4CF992359F3933001F7C1
:10498000F5CFCF92DF92EF92FF92CF93C82F0E9484
:1049900065BC6B017C0124EA30E74DE75FE3609181
:1049A000190170911A0180911B0190911C010E94C4
:1049B00066E787FD18C08AEF90E0A0E0B0E08C0DBC
:1049C0009D1DAE1DBF1D8093D0039093D103A09376
:1049D000D203B093D303C0931401CF91FF90EF9013
:1049E000DF90CF90089580E090E0DC01E8CFCF9396
:1049F00080919F03811154C010923312109234128F
:104A0000109235121092011210920012109203129D
:104A1000109202121092051281E08093041282E239
:104A20008093061210920B1210920A12EFE1F2E13B
:104A30002DE232E18FEF81932E173F07E1F7C1E0BE
:104A4000C0931C122FE03FEA3093121220931112F0
:104A5000C0931312109214121092151290E49093B6
:104A60001612109217122EE03FEA30932E12209366
:104A70002D122CE031E03093FF112093FE119EE1C6
:104A80009093231291E1909324129CE19093211230
:104A90008093201280931F120E94A2BDC0939F0397
:104AA00081E080939E0389E69DE090934811809376
:104AB000471110924A111092491153985B9A5298DB
:104AC0005A9A3898409A0CDF1092DC03CF910895DF
:104AD000FC0180E0309749F09491992331F0907C6B
:104AE000903809F08F5F3196F7CF0895009751F015
:104AF000FC0180E09191992331F0907C9038D1F3C2
:104B00008F5FF8CF80E00895B0E0A0E0EAE8F5E23A
:104B10000C9454EEEC015B018A01FB01099587FDC1
:104B200010C0C82ED12CF12CE12C2196F801C082A6
:104B3000D182E282F382CE01CDB7DEB7EAE00C94F7
:104B400070EE982F907E903CA9F48F7190E0B0E0C9
:104B5000A0E06C017D0156E0CC0CDD1CEE1CFF1CBE
:104B60005A95D1F7CE010196F50109958F73C82AA0
:104B70002296DCCF982F907F903E11F58F7090E0B9
:104B8000B0E0A0E06C017D0136E0CC0CDD1CEE1C39
:104B9000FF1C3A95D1F7CE010196F50109958F7367
:104BA000C82A46E0CC0CDD1CEE1CFF1C4A95D1F750
:104BB000CE010296F50109958F73C82A2396B6CFC8
:104BC000982F987F903F79F5877090E0B0E0A0E053
:104BD0006C017D0186E0CC0CDD1CEE1CFF1C8A956F
:104BE000D1F7CE010196F50109958F73C82A96E099
:104BF000CC0CDD1CEE1CFF1C9A95D1F7CE01029661
:104C0000F50109958F73C82A26E0CC0CDD1CEE1C3B
:104C1000FF1C2A95D1F7CE010396F50109958F73F4
:104C2000C82A249683CF982F907C903841F4807CBA
:104C3000803869F42196CE01F5010995F8CF8E7F71
:104C40008D3F28F02196CE01F5010995F8CFC12CB2
:104C5000D12C76016BCF9CE0899F802D112491E0AF
:104C6000980F90939D032CE0280F2093D80530E0F7
:104C70002E5F3F4F409130124217130619F014F087
:104C800080E00895209132129217D0F7662341F008
:104C90008E5F0E9487BE8091D8058E5F0E9487BE7E
:104CA0008091D80590913012891750F320913212DB
:104CB00090919D03291720F31092331280933412A0
:104CC00081E0089520919C03022E000C330B821783
:104CD000130641F080939C036CE470E18CEF91E14A
:104CE0000C9450BF0895ACE0B0E0E9E7F6E20C9414
:104CF00056EE6F3F71058105910509F070F488EF5C
:104D000091E153DAE0910012F09101123196849111
:104D100090E02C96E8E00C9472EEF0903312E09064
:104D2000341220919E0321110FC04BE35DE06E2DE4
:104D30008F2D0E9401C090E080E0F80EF0923312B7
:104D4000E09234129927E5CFC0900012D090011262
:104D50002CEF31E13A8329832F2D30E03C832B83E4
:104D60002E2D30E03E832D8318861F822FEF3FEFDC
:104D70003A8729871C861B8602E810E29E012F5F76
:104D80003F4FAB01BC01C6010E941DB0B6018CEFC4
:104D900091E10E9450BF8F819885CFCF4F925F9253
:104DA0006F927F928F929F92BF92CF92DF92EF92FB
:104DB000FF920F931F93CF93DF93CDB7DEB7289762
:104DC0000FB6F894DEBF0FBECDBF7C016A0149016A
:104DD000FB0190818CE0989F800D1124982FF701A2
:104DE0002081822F880F820F880F80933312909337
:104DF00034124115510561F1FA82E9827C836B839B
:104E000001111FC0AE014B5F5F4FB401C6017CDED4
:104E10006C016D817E818F81988561157105810599
:104E20009105B1F060DFF70180818F5F808385316C
:104E300048F3CE0101960E94B21BE4CFB12C86014B
:104E400029C08A01B12C26C0452846284728B1F739
:104E500028960FB6F894DEBF0FBECDBFDF91CF917D
:104E60001F910F91FF90EF90DF90CF90BF909F9098
:104E70008F907F906F905F904F900895B39407C08C
:104E8000B1102DC001151105C9F20F5F1F4F01159B
:104E90001105A9F2AE014B5F5F4FB401C60134DECC
:104EA0006C014D805E806F807884411451046104F0
:104EB0007104A9F0F0E24F1651046104710401F38A
:104EC000D301C2018D97A109B1090297A105B105CE
:104ED00030F04BE2441651046104710479F6F70195
:104EE0008081482F4B0D5527551F4631510534F011
:104EF000853020F0CE0101960E94B21B81E0411462
:104F000051046104710409F480E0B80EF701808156
:104F10008B0D8083BB2009F497CFBA94AE014B5F11
:104F20005F4FB401C801F0DD8C016D817E818F81FE
:104F30009885D9DEEFCFCF93DF93FC0125AD21110A
:104F400004C021E025AF0E94A2BDC091FE11D09106
:104F5000FF11E0912D12F0912E1282E00995E0915F
:104F60002D12F0912E1281E0099530E020E044E10D
:104F7000BE018CEF91E10E949DBD2FE232E147E13D
:104F8000BE018CEF91E10E949DBDE0912D12F09148
:104F90002E1280E00995DF91CF910895ACE0B0E04A
:104FA000E4EDF7E20C9456EEF0903312E0903412F8
:104FB00020919E03211112C04BE15DE06E2D8F2DDB
:104FC0000E9401C090E080E0F80EF0923312E0926F
:104FD000341299272C96E8E00C9472EEC0900012DF
:104FE000D09001122CEF31E13A8329832F2D30E04C
:104FF0003C832B832E2D30E03E832D8318861F8229
:105000007A8769871C861B8602E810E29E012F5F63
:105010003F4F4CEA5BE1BC01C6010E94B2B0B60151
:105020008CEF91E10E9450BF8F819885CDCFA4E095
:10503000B0E0EDE1F8E20C9452EE7C01062F5A014B
:10504000122F862F660F990B9C0123583E4F690142
:1050500086E0882E912C11160CF03DC0AE014F5FFA
:105060005F4F6CEA7BE1C7014FDD7C0169817A818A
:105070008B819C81611571058105910561F16D330D
:1050800071058105910509F450C06E3771058105E0
:10509000910509F44AC06A3271058105910501F54F
:1050A00007FF11C08FE59DE00E3F11F08BE59DE0FD
:1050B00036E01302B001112471DF66E070E00E9457
:1050C000FCED161B60C065E470E080E090E00BDE54
:1050D000115069F510E0812F2496ECE00C946EEEEF
:1050E000643271058105910571F4A114B104D1F008
:1050F000E6E01E02B0011124C50150DFB4010E9498
:10510000FCED161BA8CF603471058105910551F4A3
:105110001150F6016081062E000C770B880B990B5D
:10512000E2DD99CFE0DD115096CF07FDBBCF61E006
:1051300089819A81AB81BC81CD97A105B10509F424
:1051400060E0600F6A30A4F01150862F6AE00E9480
:10515000DBED092F682F880F770B605D7F4F072EDF
:10516000000C880B990BBFDD112309F4B3CF602F1E
:10517000062E000C770B605D7F4F072E000C880B0E
:10518000990BB1DD1150112309F4A4CF86E0180268
:10519000B0011124C70102DF66E070E00E94FCED5F
:1051A000161B99CFE8EFF1E183AF64AF6FEF7FEFAC
:1051B000CA01F4CEACE0B0E0E0EEF8E20C9456EEBA
:1051C000F0903312E090341220919E03211112C00E
:1051D0004BEF5CE06E2D8F2D0E9401C090E080E0CF
:1051E000F80EF0923312E092341299272C96E8E0F0
:1051F0000C9472EEC0900012D09001122CEF31E1AD
:105200003A8329832F2D30E03C832B832E2D30E0F1
:105210003E832D8318861F827A8769871C861B86AA
:1052200002E810E29E012F5F3F4F4FEA5BE1BC01B5
:10523000C6010E94B2B0B6018CEF91E10E9450BF4E
:105240008F819885CDCFB0E0A0E0E9E2F9E20C943F
:1052500052EE5B01C42F790141FB662760F9FBDC4C
:10526000882309F45EC0D12CC12CA114B10431F003
:10527000C5012EDC96E0899F6001112410E000E05A
:10528000E114F10421F0C70131DC082F10E0C0FF68
:1052900020C080E890E08C199D094AEF40039001FE
:1052A000419F300D1124820F931F6CE070E00E942B
:1052B000FCED4B01C0E8D0E081E0881A910897FC32
:1052C0000AC060E270E080E090E00DDDC81BD90B01
:1052D000F3CFC0E8D0E0C114D10491F0CE0166E074
:1052E00070E00E94E8ED4091DA055091DB05262F31
:1052F0006091D905C5019BDE96E0899FE0011124EC
:105300000115110529F0BE01C70154DFC81BD90BD7
:10531000C730D10530F060E270E080E090E0E3DC7F
:10532000F5CFCDB7DEB7ECE00C946EEE809157016F
:10533000882339F030E020E041E06FE47FE082E054
:1053400082CF089580915701882349F06091270406
:105350007091280430E020E041E081E074CF0895AE
:105360006FEF7FEF27CFB0E0A0E0E9EBF9E20C941C
:1053700054EE5C016B01ACDBE82EC601B7DBF12C0F
:1053800003E110E0081B1109C5E20E151F050CF41E
:10539000CFE18C2F90E09C012E5F3F4F4091301267
:1053A0004217130609F08CF509972091321228173D
:1053B00019065CF14091DA055091DB056091D90541
:1053C00010923312C093341225E1C50130DED1E0D2
:1053D000C114D104A9F06AE370E080E090E083DCBE
:1053E0000E151F05A4F4C45F80913012C81740F059
:1053F000209132124C2F4950550B241715064CF4AE
:10540000CDB7DEB7EAE00C9470EED0E0E1CFDD235B
:10541000B9F3802F880F080F000F00933312C09349
:10542000341260E270E080E090E05DDCC60198DF5D
:10543000E7CFACE0B0E0EFE1FAE20C9452EE982F47
:10544000862F6A017901B02E692F05DC882309F4C3
:1054500086C010919E03C701002371F139DBA82E8D
:105460008090001290900112111141C02FEF3FEF78
:10547000122F23E12A194091DA055091DB05609142
:10548000D905C601D4DDAA2009F469C0B6E08B9F16
:10549000600111246AE370E080E090E024DC57E0D2
:1054A000C516D10408F441C060E270E080E090E0ED
:1054B0001ADCC81AD90AF3CF19DBA82E8090001283
:1054C00090900112112391F2FE0133968AE0DF01E0
:1054D0001D928A95E9F78CEF91E19A8389830BE518
:1054E00010E29E012F5F3F4F4FEA5BE112C0FE01C9
:1054F00033968AE0DF011D928A95E9F78CEF91E1FE
:105500009A8389830BE510E29E012F5F3F4F4CEA9F
:105510005BE1B701C4010E94B2B0B4018CEF91E12C
:105520000E9450BF2F813885A3CF4091D805212FED
:1055300030E0A6E0AA9EC00111242E5F3F4F28173D
:1055400039070CF49C0180E8821B8093331240934E
:105550003412BB2041F06FEF7FEFC7011FDD2C96A7
:10556000ECE00C946EEEC701FBDEF9CFE8EFF1E161
:1055700083AF64AFCA01F4CE0C9438B1CF93DF93FC
:10558000DB01F9019C919130C1F0943080F094508E
:105590009C938830D1F480819181009771F00197BC
:1055A00091838083480F591FEA01188206C08C3509
:1055B00039F49C5F9C93943041F4DF91CF9108952E
:1055C0008B3339F781E08C93F8CF20813181B90199
:1055D0006F5F7F4F71836083420F531FEA0188839F
:1055E000808191818F3591056CF7E7CF0F931F93E1
:1055F00081E0009161131091621320916313309147
:10560000641340915D1350915E1360915F1370912C
:105610006013041715072607370708F480E01F9169
:105620000F9108954F925F926F927F928F929F9207
:10563000BF92CF92DF92EF92FF920F931F93CF937F
:10564000DF9310929803109297032FE320939B030C
:1056500010929A031092990310929303109294035C
:1056600010929503109296039C01F90190812F5F8F
:105670003F4F9032D1F39E34C9F4818190ED980F61
:105680009A3020F08D3211F08B3281F432969F01E6
:105690002F5F3F4F808180538A3008F46DC09F0197
:1056A0002F5F3F4F8081803209F468C0F093F70587
:1056B000E093F6058F010F5F1F4FC0816AE270E033
:1056C000C8010E949DF0009731F0FC013197808164
:1056D0008032E1F31182CD3421F0C43511F0C734AA
:1056E000D9F5F80180810F5F1F4F8032D1F38053CD
:1056F0008A3090F5C0939B0390E080E06AE0AF01B0
:105700004F5F5F4F689F9001699F300D1124C90161
:10571000C0972081820F911D27FD9A95FA01208163
:1057200020532A3060F390939A0380939903DF010A
:1057300031962C912032D9F3CD3461F58E3191051B
:1057400039F0F0F48731910519F08C31910511F59C
:10575000B0939803A0939703DF91CF911F910F917E
:10576000FF90EF90DF90CF90BF909F908F907F90B1
:105770006F905F904F900895F90189CFF9018FCF15
:105780008537910538F08737910510F3803A13E09B
:105790009107F1F28090F6059090F70540E050E017
:1057A000BA0130E020E0C12CD12C7601C394FD0178
:1057B0003196DC91DD2309F484C0D132F1F4CD348B
:1057C000E1F480329105C9F440939303509394031C
:1057D0006093950370939603F0939803E093970377
:1057E00063E270E0CF010E949DF0009709F4B4CF0E
:1057F000FC011082B1CFDF01DACFD154DA3108F0E9
:105800005BC0DF011D91103291F0A0EDA10FAA3015
:10581000E8F01E3271F4A181A053AA30B8F021152E
:10582000310519F49F0121503109B12C13C0FD013C
:10583000E8CF1D3211F01B3291F7A181B0EDBA0F04
:10584000BA3020F0AE3259F7A281E6CFBE2EB8189A
:10585000309759F3AD2FB0E02601370104C0440C56
:10586000551C661C771CDA95D2F744295529662900
:105870007729A758BC4FBC92A081A154AA3108F443
:10588000BACFDF01D191DD2309F491CF00EDB02E25
:10589000BD0E19E01B15A8F713EDB12EBD0E11E0DA
:1058A0001B1578F7DB3269F3FD013196DC91D032BC
:1058B00009F07DCFDF01F8CF21153105E9F69D0113
:1058C000DBCF309398032093970340939303509337
:1058D000940360939503709396033ECF10928704D0
:1058E000109288041092890410928A04E3E6F4E08E
:1058F00084E2DF011D928A95E9F7089590915E0494
:10590000981771F00E941A8D80915E04882349F0E7
:105910008DE691E00E94648D10925E040C9404A0C8
:10592000089581E080935E048DE691E00E943A8DB7
:10593000F5CF90915E0481E08927E0CF4F925F928E
:105940006F927F928F929F92AF92BF92CF92DF928F
:10595000EF92FF921F93CF93DF93EC01162F2091CC
:105960005F04309160044091610450916204688149
:1059700079818A819B810E9466E7882309F497C018
:10598000B0905E0480E0BADFC880D980EA80FB80F6
:1059900020E030E0A901C701B6010E94E7EF87FFD0
:1059A00003C0C12CD12C7601C0925F04D092600458
:1059B000E0926104F09262042DEB37E346E855EB88
:1059C000C701B6010E9466E787FD0BC02DEB37E3E8
:1059D00046E855E3C701B6010E94E7EF18160CF040
:1059E00076C0A701960160E070E080E89FE30E9426
:1059F000FBEE609356047093570480935804909381
:105A0000590480EF9FEFA9E7B4EC80935A04909378
:105A10005B04A0935C04B0935D04BB2009F447C011
:105A200040906D0150906E0160906F017090700118
:105A30008090710190907201A0907301B0907401F8
:105A4000C0907501D0907601E0907701F0907801D8
:105A500081E054DF112359F1A301920160916D019E
:105A600070916E0180916F01909170010E9466E7C4
:105A700081111BC0A50194016091710170917201A7
:105A800080917301909174010E9466E781110DC0AD
:105A90002091750130917601409177015091780104
:105AA000C701B6010E9466E781110E9401A1DF9142
:105AB000CF911F91FF90EF90DF90CF90BF90AF906C
:105AC0009F908F907F906F905F904F90089560E0CF
:105AD00070E0CB018ECFCF93DF93C3E6D4E020E01C
:105AE00030E0A901688179818A819B810E9466E703
:105AF00081111FC020E030E0A9016C817D818E8181
:105B00009F810E9466E7811114C020E030E0A90166
:105B1000688579858A859B850E9466E7811109C021
:105B20002C9684E0C738D807D1F680E0DF91CF917A
:105B3000089581E0FBCFCF92DF92EF92FF926B014D
:105B40007C0183E3C816D104E104F10470F082E320
:105B5000C81AD108E108F10862E370E080E090E043
:105B60000E94D9BB0E94B187ECCFC701B6010E9449
:105B7000D9BB0E94B187FF90EF90DF90CF9008953E
:105B8000BC0190E080E00C94DBB08091ED058130A9
:105B900069F09091651392FB882780F992FF07C006
:105BA00097FB882780F991E08927089581E008957F
:105BB0008091D0119091D111891B8F7009F4E5CF9C
:105BC00081E008958F929F92AF92BF92EF92FF92E1
:105BD0000F931F93CF93DF93EC018B01E42EF22EF2
:105BE0008091F6119091F7118C179D0709F43EC032
:105BF0002091210427FD1092210429E7C535D20701
:105C000009F03FC0815D9A4371F40E9465BC6E51FA
:105C10007B4F8F4F9F4F6093230470932404809396
:105C2000250490932604D093F711C093F61130E029
:105C300020E00093C0051093C1052093C205309366
:105C4000C305E092BA05F092B305C15DDA4321F4D1
:105C5000109238041092220482E08093570181E070
:105C60008093D0051092360410923104DF91CF91C9
:105C70001F910F91FF90EF90BF90AF909F908F90EA
:105C800008952AE3C13DD20771F685559947D1F4AD
:105C90000E9465BC8090230490902404A090250469
:105CA000B0902604681979098A099B0997FF0AC0F0
:105CB00080914B058770873029F47ADFCDEFD1E7EB
:105CC0008111B1CFC1EDDAE3AECFCF92DF92EF9287
:105CD000FF92CF93DF9300D000D0CDB7DEB7809195
:105CE000B4051092B405882329F1809135048F5FA3
:105CF000809335048930D8F081E08093340420E02B
:105D000040E070E060E08EE597E35CDF86E490E1E0
:105D100090934E0580934D050F900F900F900F902C
:105D2000DF91CF91FF90EF90DF90CF9008950E9488
:105D3000ABACF2CF6091C0057091C1058091C205F6
:105D40009091C305611571058105910509F449C05C
:105D50000E946CE72DEC3CEC4CEC5CE30E94CBE742
:105D60009B01AC0160917501709176018091770182
:105D7000909178010E9484EE6B017C0120E030E07C
:105D800040E050E40E9466E718162CF4C12CD12C98
:105D9000E12C90E4F92E20E030E040E050ECC70127
:105DA000B6010E94E7EF87FF05C0C12CD12CE12C82
:105DB00080ECF82EC0927501D0927601E0927701C6
:105DC000F092780189EB91E00E94549F82E08093E9
:105DD00057011092C0051092C1051092C205109291
:105DE000C30580915701882309F496CFC0907501AF
:105DF000D0907601E0907701F090780120E030E0DB
:105E0000A901C701B6010E9466E787FD16C067E1D8
:105E100077EB81ED98E3A70196010E9484EE6983F8
:105E20007A838B839C836BE2CE0101960E94D4A679
:105E3000BC018FE390E197DA6FCF67E177EB81EDFB
:105E400098EBE9CF81E08093380480914B0587700F
:105E5000873051F010924B05109255048FED98E168
:105E600090934E0580934D0580915E04809333049A
:105E700080E044DD20E040E070E060E081E49FE20B
:105E8000A1CE54DA809155048770873071F4109256
:105E9000320420E040E070E060E08BE496E392DEC4
:105EA00081E0809331040C94CD1C089520E040E003
:105EB00070E060E081ED9AE385CEAEE1B0E0E3E62C
:105EC000FFE20C945AEE482F082E000C550B20913F
:105ED0001501309116018F3F39F0FA01EE0FFF1FC7
:105EE000E95EFE4F208131813F932F935F938F9323
:105EF0008AE59FE09F938F938E010F5F1F4F1F9343
:105F00000F930E94FFE6C8010E949523CFDF0FB6D2
:105F1000F894DEBF0FBECDBF6E96E4E00C9476EE33
:105F20008FEFCBCF8091D905C8CFCF93DF93E0918E
:105F30002204EE2329F1E150E0932204AE2FB0E0D9
:105F400099E0E99FF0011124E551FC4F278140E0E1
:105F500070E060E0811103C046816281738189E055
:105F60008A9FE0018B9FD00D1124C551DC4F8881A1
:105F7000998128DE888580933804DF91CF91089538
:105F800095DFFBCF81E0D1CFB0E0A0E0EAECFFE20B
:105F90000C9457EE0DDE082F61E081E00E949C23F7
:105FA000C091BA05FC2E85E0E82EEC0E11E01C1B1A
:105FB000DC2ED194C11114C08091B9058823F9F069
:105FC00080915701882309F473C081E09091B9054D
:105FD000911180E024E04AE050E16D2D0E947AB7F3
:105FE000011139C0D2E0C130B9F58091B9058130D5
:105FF000B1F080915701811121C0D2E043C080915E
:10600000B4051092B4058823D9F2BCDF8091D00585
:106010008823B1F2CDB7DEB7E7E00C9473EE809140
:10602000B4051092B405882321F38DE590E30E9416
:10603000A9B88091D0058823E1F2ECCF81E090915E
:10604000B905913009F080E023E041E050E1612F93
:106050000E947AB7D2CFD1E0DC1314C08091B90589
:106060008D17B9F080915701882361F06C2F6F195B
:1060700081E09091B9059C1380E023E045EF5FE05B
:106080000E947AB7CF5FCE1195CFDF5FD093B30573
:10609000C1CF8091B4051092B405882319F38CE622
:1060A00091E30E94A9B88091D0058823D9F2B2CF9C
:1060B000D1E0002309F4A1CFE5CFB0E0A0E0E3E612
:1060C000F0E30C9455EE61E081E00E949C23C091C6
:1060D000BA0585E0C82ECC0ED4E0DC1B13E01C1BF7
:1060E00082E0F82EFC1A81E0E82EEC1ABC2EB19466
:1060F000C1112AC08091B9058823B1F08091570160
:10610000882359F081E09091B905911180E024E055
:1061100043EE5FE06B2D0E947AB7CF5FCC12E8CFE1
:1061200085E08093B3050BC08091B4051092B4054F
:10613000882321F327DF8091D0058823F9F2CDB79A
:10614000DEB7E9E00C9471EEC13081F58091B905BC
:106150008130B9F0809157018823F9F2DD24D3947E
:106160008091B905813009F0D12C8DEF9BE00E9420
:10617000DF1A00E09C0148ED5FE06E2D8D2D59D9AE
:10618000CCCF8091B4051092B405882319F30E94F6
:1061900050B848E45DE16DEF7BE088ED9FE00E9440
:1061A000B8B88091D0058823A9F2C9CFC23009F0D0
:1061B00073C08091B9058230B1F080915701882376
:1061C00009F4ABCFDD24D3948091B905823009F076
:1061D000D12C81E09CE00E94DF1A00E09C014DEC94
:1061E0005FE06F2DCBCF8091B4051092B40588236A
:1061F00021F30E9450B846E45DE161E07CE08DEC63
:106200009FE00E94B8B88091D0058823B1F297CF63
:106210008091B9058330B1F080915701882309F44A
:106220007CCFDD24D3948091B905833009F0D12C43
:1062300085E09CE00E94DF1A00E09C0142EC5FE0F8
:10624000612F9CCF8091B4051092B405882321F36F
:106250000E9450B844E45DE165E07CE082EC9FE0A0
:106260000E94B8B88091D0058823B1F268CF8091A0
:10627000B4051092B4058823C9F00E9450B842E4D6
:106280005DE169E07CE087EB9FE00E94B8B8809117
:10629000D005882359F053CFC33009F4B9CFC430A7
:1062A00009F03BCF8091B905843009F38091570103
:1062B000882309F432CFDD24D3948091B90584304A
:1062C00009F0D12C89E09CE00E94DF1A00E09C01DB
:1062D00047EB5FE06D2F52CFA7E0B0E0E2E7F1E3DC
:1062E0000C944CEE61E081E00E949C237090BA0512
:1062F000672C85E0870D8D838CE087198E8388E07D
:1063000087198F838BE0582E57188AE0482E47183C
:1063100089E0382E371887E0282E27187110C7C05B
:106320008091B905882309F4B1C080915701882371
:1063300061F0662D619581E09091B905911180E041
:1063400024E043EE5FE00E947AB720E030E543ECC2
:1063500050E460916011709161118091621190918F
:1063600063110E94CBE760932D0470932E048093F9
:106370002F04909330042CEA35EC47E25EE3609101
:1063800064117091651180916611909167110E945E
:10639000CBE76093290470932A0480932B04909395
:1063A0002C0485E07812DFC11092D9058091B905DF
:1063B000853009F4C1C180915701882391F011E023
:1063C0008091B905853009F010E08CE591E10E94DB
:1063D0004A1D65E0661900E09C0149E85FE0812FF5
:1063E00028D820E030E543EC50E460919F0570919F
:1063F000A0058091A1059091A2050E94CBE7609332
:106400002D0470932E0480932F04909330042CEA73
:1064100035EC47E25EE36091A3057091A40580919D
:10642000A5059091A6050E94CBE76093290470937F
:106430002A0480932B0490932C0489E07812B1C233
:106440008FEF8093D9058091B905893009F492C204
:1064500080915701882391F011E08091B90589302E
:1064600009F010E08BE995E00E944A1D00E09C01D4
:1064700049E85FE0632D812F0E94192A73948D8172
:1064800078124CCF8DE08093B3050DC08091B40598
:106490001092B405882309F448CF74DD8091D005AB
:1064A000882309F442CF2796E2E10C9468EE81E05C
:1064B000781230C09091B9059130C9F080915701A0
:1064C000882309F442CF61E0661981E0913009F038
:1064D00080E09091F4052BEA3FE0911102C027EA99
:1064E0003FE001E04EEA5FE00E94192A2ECF809142
:1064F000B4051092B405882309F38091F40587252B
:106500008093F40583E0809357018091D005882320
:10651000A9F2C9CF82E07812EFC28091B90582302A
:1065200009F47EC080915701882309F111E0809120
:10653000B905823009F010E060915F01709160014F
:10654000072E000C880B990B0E946CE769837A83F5
:106550008B839C83CE0101960E94782362E06619AA
:1065600000E09C0140EA5FE0812F0E94192A20E0B0
:1065700030E543EC50E460916011709161118091BD
:106580006211909163110E94CBE760932D04709388
:106590002E0480932F04909330042CEA35EC47E2CC
:1065A0005EE3609164117091651180916611909124
:1065B00067110E94CBE76093290470932A048093AB
:1065C0002B0490932C0488E078120BCF1092D905FD
:1065D0008091B905883009F4B2C1809157018823B0
:1065E00009F4E2C011E08091B905883009F010E0AB
:1065F0006091170170911801072E000C880B990B00
:106600000E946CE769837A838B839C83CE01019619
:106610000E94782300E09C014AE65FE06F81DFCEB4
:106620008091B4051092B405882309F47BCF10E063
:1066300000E025EF30E050E040E06FE571E080EAF7
:106640009FE00E94EAB88091D005882309F46ACFC0
:106650002ACF8091B905833029F180915701882391
:1066600009F485CF11E08091B905833009F010E07D
:106670006091590170915A01072E000C880B990BFB
:106680000E946CE769837A838B839C83CE01019699
:106690000E94782363E0661900E09C0149E95FE00D
:1066A000812F22CF8091B4051092B4058823A9F2DE
:1066B00010E000E025EF30E050E040E069E571E0F7
:1066C00089E99FE00E94EAB88091D005882329F2E9
:1066D000EACE8091B4051092B405882309F418C25B
:1066E00020E030E048EC52E460915B0170915C0185
:1066F00080915D0190915E010E94CBE70E9468EF5E
:10670000912C812CE0E5AE2EE7E3BE2E6B0118EE56
:10671000E12E13E0F12E00E010E020E030E0A901CE
:106720006BE571E081E99FE00E945CB88091D00543
:10673000882309F4EDC1B7CE8091B4051092B40559
:10674000882309F438CE0E9450B850E040E06CE550
:1067500071E189E89FE00E945EB98091D0058823AD
:1067600009F429CEA0CE86E07812B6C01092D905E1
:106770008091B905863009F471C080915701882352
:1067800099F011E08091B905863009F010E08DE2B2
:1067900094E00E94121A66E0661900E09C0141E84C
:1067A0005FE0812F0E94192A20E030E543EC50E49D
:1067B00060919F057091A0058091A1059091A2051F
:1067C0000E94CBE760932D0470932E0480932F04D6
:1067D000909330042CEA35EC47E25EE36091A30528
:1067E0007091A4058091A5059091A6050E94CBE724
:1067F0006093290470932A0480932B0490932C04B3
:106800008CE078123BCE8FEF8093D9058091B9054B
:106810008C3009F456C180915701882309F42ECE9B
:1068200011E08091B9058C3009F010E060911501FC
:1068300070911601072E000C880B990B0E946CE7D3
:1068400069837A838B839C83CE0101960E9478238F
:1068500000E09C014AE65FE06E810DCE8091B405B8
:106860001092B405882309F488CF0E9450B820E024
:1068700030E048EC52E460912D0470912E04809138
:106880002F04909130040E94CBE720E030E040E8F4
:106890005FE30E9483EE0E9468EF3BEF832E39E1B5
:1068A000932E46E4A42E47E3B42E6B0117E5E12EA8
:1068B0001EE3F12E0FE010E021E030E040E050E078
:1068C0006DE274E081E89FE00E945CB88091D005A1
:1068D000882309F452CFE7CD87E0781274CE109266
:1068E000D9058091B9058730A9F080915701882397
:1068F00009F45ACF11E08091B905873009F010E012
:1069000089E294E00E944A1D00E09C0149E75FE0B3
:10691000622D65CD8091B4051092B405882329F3CA
:106920000E9450B844EE59E169E274E089E79FE0C3
:106930000E945EB98091D0058823B9F2B4CD8091D0
:10694000B4051092B405882309F447CE0E9450B8CC
:1069500002E91FE225EF30E046E950E067E171E02F
:106960008AE69FE00E94EAB88091D005882309F466
:1069700034CE99CD8091B4051092B405882309F4E2
:1069800067CD0E9450B850E040E06BE975E089E8BF
:106990009FE00E945EB98091D005882309F458CD0C
:1069A00082CD8AE0781259C08FEF8093D90580910B
:1069B000B9058A30A9F080915701882309F45ECD8A
:1069C00011E08091B9058A3009F010E08DE294E081
:1069D0000E94121A00E09C0141E85FE0642D4BCD5B
:1069E0008091B4051092B405882329F30E9450B811
:1069F00020E030E048EC52E460912D0470912E04C8
:106A000080912F04909130040E94CBE720E030E089
:106A100040E85FE30E9483EE0E9468EF8DEC882ED1
:106A200089E1982E96E4A92E97E3B92E6B0117E51C
:106A3000E12E1EE3F12E0FE010E021E030E040E017
:106A400050E06DE274E081E89FE00E945CB88091C4
:106A5000D005882309F4AFCF26CD8BE07812D0CEB5
:106A60008FEF8093D9058091B9058B30A9F0809183
:106A70005701882309F402CD11E08091B9058B30CC
:106A800009F010E089E294E00E944A1D00E09C01B8
:106A900049E75FE0652DEFCC8091B4051092B40515
:106AA000882329F30E9450B846EB59E169E274E06B
:106AB00089E79FE00E945EB98091D0058823B9F2F2
:106AC000F2CC8091B4051092B405882309F4A3CECA
:106AD0000E9450B800E91FE223E730E04CE350E0A9
:106AE00065E171E08AE69FE00E94EAB88091D005F6
:106AF000882309F490CED7CC83E0781609F4A9CD89
:106B000084E0781222CC8091B905843009F4E1CD7B
:106B100080915701882309F42ACD11E08091B905AD
:106B2000843009F010E08BE591E00E940D2264E0D2
:106B3000661900E09C0141E95FE0B2CDA3E0B0E05E
:106B4000E4EAF5E30C944CEE4C013B015A011901C7
:106B5000280181E0809338044091C0055091C1051F
:106B60006091C2057091C30541155105610571051C
:106B700071F0141615060CF080E080933104109229
:106B8000C0051092C1051092C2051092C305109164
:106B900031048091B4058B831092B405811105C036
:106BA00080915701882309F46FC0C2010E946825B3
:106BB000082F80E0C114D10419F0C6010E94682595
:106BC0001A821982E114F104B1F4402F50E0282F09
:106BD00030E0CA01820F931F46976CF485E190E084
:106BE000841B950B821B930B97FD019695958795BA
:106BF0008A8381E0898301E02CEA3BE1A201BE01A6
:106C00006F5F7F4FCE0102960E94CE26E114F10401
:106C100091F08A81882321F01A8289818F5F89838C
:106C200000E02FEA3BE1A701BE016F5F7F4FCE017D
:106C300002960E94CE26C114D10459F000E02CEA3D
:106C40003BE1A601BE016F5F7F4FCE0102960E941D
:106C5000CE2641E04127B30181E00E94EABEC40193
:106C60000E946825412FB40194E1981B892F0E944E
:106C7000EABEEB81EE2341F0111101C05101A114D4
:106C8000B10431F0F50109952396E2E10C9468EE28
:106C900080E04BD9F9CFCF92DF92EF92FF920F9322
:106CA0001F9388E1C82E80E1D82EF12CE12C0AE157
:106CB00010E126E737E34DEC5CE166E270E18BE240
:106CC00090E13CDF1F910F91FF90EF90DF90CF900C
:106CD0000895B0E0A0E0EFE6F6E30C9454EEADB614
:106CE000BEB68DE39FE00E94682590E001962DB727
:106CF0003EB7281B390B0FB6F8943EBF0FBE2DBF11
:106D00008DB79EB701967C016DE37FE00E94AEE6F1
:106D1000809139040AE01FE0813031F005EF1EE078
:106D2000823011F00DE11FE08EE2C82E8FE0D82EE8
:106D300026E53FE24BE857E360E37FE087E39FE02F
:106D4000FDDE0FB6F894BEBE0FBEADBEEAE00C94F9
:106D500070EE0F931F93CF93DF93FC01EB018091B3
:106D6000C0059091C105A091C205B091C305B7FFC0
:106D700008C01092C0051092C1051092C205109271
:106D8000C3058091C4059091C505A091C605B09139
:106D9000C7054091C0055091C1056091C205709131
:106DA000C30584179507A607B70744F48093C00569
:106DB0009093C105A093C205B093C305809157017C
:106DC0008823E1F06091C0057091C1058091C205F2
:106DD0009091C3050091C8051091C9052091CA057D
:106DE0003091CB05600F711F821F931F0995BC0165
:106DF0008091CE059091CF050E94B3298091B40572
:106E0000811108C08091BD058823B1F1809157019F
:106E1000882391F18091CC059091CD050097B1F038
:106E20004091C0055091C1056091C2057091C305A4
:106E30000091C8051091C9052091CA053091CB0574
:106E4000400F511F621F731FFE010995E091BE059F
:106E5000F091BF05309741F08091BD05811103C0CD
:106E60008091B405811109958091B4051092B40503
:106E7000882311F080E059D8DF91CF911F910F91B5
:106E800008956CE679E183E99BE163CF64E979E1F8
:106E900086EC9AE15ECF68E579E182E89DE159CF21
:106EA00060E879E18FE593E254CF68EA79E182E81E
:106EB00093E24FCF1092380480E037C880913404B9
:106EC000811104C0F7DF81E00E949B1D8091570172
:106ED000882341F030E020E041E060E370E181E0B0
:106EE0000E94232982E080935701089580E090E07A
:106EF000A0E8B0E48093750190937601A0937701A8
:106F0000B093780189EB91E00E94549F8091330403
:106F10000E947E2CCFCF0E941AA50E94048A0E9454
:106F20009B1D0C94562F4F925F926F927F928F927F
:106F30009F92AF92BF92CF92DF92EF92FF921F93F8
:106F4000CF93DF9300D000D0CDB7DEB70E9465BCF1
:106F50006B017C01809114018F3FD9F10E9465BCC7
:106F60008090D0039090D103A090D203B090D3032F
:106F7000681979098A099B0997FD2BC08091D01166
:106F80009091D1118F5F8F70891719F1E0911401E1
:106F900080E090E0A5E0B3E4E53050F424E0E29F27
:106FA000F0011124E757FE4F80819181A281B381C6
:106FB00089839A83AB83BC8320E030E0A901BE01C2
:106FC0006F5F7F4F8DE691E00E94F2D88FEF809344
:106FD00014010E9470248091DE0382FF33C08091EF
:106FE000DB03811131C091E09093DB038091F505C3
:106FF00089278093B4051092F50583E080935701AB
:107000001092DE030E9465BC6C507E4F8F4F9F4FE5
:107010006093DF037093E0038093E1039093E203B6
:1070200068E873E182E090E00E947FAC16E01150C6
:1070300059F00E9423AC62E070E080E090E00E9492
:10704000D9BBF5CF1092DB038091F0059091F1054B
:10705000A091F205B091F305A7019601281B390B09
:107060004A0B5B0BDA01C901B7FF05C080913604FA
:10707000882309F4ECC1D701C6018C599F4FAF4F4B
:10708000BF4F8093F0059093F105A093F205B09364
:10709000F3056091DC03062E000C770B77FF03C02D
:1070A0007195619571099091DC038091DA039813D1
:1070B00067C0633008F064C01092DC038091DC0389
:1070C0008093DA03643008F06BC08091B4058111BD
:1070D000E9C08091F6119091F7113AE3813D930751
:1070E00009F004C180915501882309F4EDC0815055
:1070F000809355010E94D88F80902306909024069B
:10710000A0902506B090260681110E94E58FD5013A
:10711000C4013AE0B695A795979587953A95D1F72A
:10712000009751E0A507B10520F08FEF9FEFA0E099
:10713000B0E09695879520915701211106C13091B5
:1071400036043111B1C18091F6119091F711815D32
:107150009A4309F490C18091380481118CC18091C7
:10716000D6039091D703A091D803B091D903C81A40
:10717000D90AEA0AFB0AF7FC8CC10E94562F89C182
:10718000633009F09BCF8091DC0387FD07C081E06D
:10719000880F880F8093DC0364E090CF8FEFF8CFE7
:1071A0008091D50521E030E040E050E0882309F4EB
:1071B00056C08090D1059090D205A090D305B09094
:1071C000D40581149104A104B104E9F170E090E0C8
:1071D00080E00E946AE720E030E040E85EE30E9441
:1071E000CBE72B013C01C701B601681979098A096F
:1071F0009B090E946AE79B01AC01C301B2010E9496
:10720000FBEE20E030E04AE754E40E94CBE74B017C
:107210005C0120E030E040EA52E40E94E7EF24E61F
:1072200030E040E050E087FF12C020E030E040EF67
:1072300051E4C501B4010E94E7EF2AE030E040E0EC
:1072400050E087FF04C021E030E040E050E0C09211
:10725000D105D092D205E092D305F092D405A09149
:10726000DC030A2E000CBB0B0E9446EE24E030E04B
:1072700040E050E00E940FEE8091C0059091C10562
:10728000A091C205B091C305820F931FA41FB51F23
:107290008093C0059093C105A093C205B093C30528
:1072A0001092DC03D701C6018856954CAF4FBF4FF3
:1072B0008093D6039093D703A093D803B093D903B8
:1072C00081E08093570105CF8CE080935501809138
:1072D000D4039091D503009729F001979093D5039B
:1072E0008093D40381E08093570104CF8A5D9C4A48
:1072F00009F000CF809155019FEF980F90935501B1
:107300008111F8CE8091D6058F5F8093D60590913C
:10731000D70524E0891708F02CE020935501981731
:1073200010F41092D60581E080935701D701C60171
:107330008856954CAF4FBF4F8093D6039093D70399
:10734000A093D803B093D903D5CE009741F04091D4
:10735000D4035091D5034817590708F0F4CE809113
:107360003604811112C0223038F0243008F441C0B4
:10737000243011F41092570188EF91E10E949B276D
:1073800081E0809337048093360483E00E94622674
:1073900081E080931C12E091F611F091F7110995AC
:1073A0001092370480913604811127C01092B405E1
:1073B0008091F6119091F711815D9A4309F0CBCE3F
:1073C0000E9465BCDC01CB018C199D09AE09BF0987
:1073D0008090D4039090D503B12CA12C88169906E7
:1073E000AA06BB0608F0AFCE9093D5038093D403D2
:1073F000AACE81E080935701BFCF8CEF91E10E942C
:1074000020BF91E0811101C090E090933604882361
:1074100069F28091F6119091F711815D9A43B9F468
:107420000E9465BCDC01CB018C199D09AE09BF0926
:10743000C090D403D090D503F12CE12CC816D90606
:10744000EA06FB0620F49093D5038093D4030F90B3
:107450000F900F900F90DF91CF911F91FF90EF90C1
:10746000DF90CF90BF90AF909F908F907F906F9064
:107470005F904F90089558E9C50E5AE3D51EE11C60
:10748000F11CC092D603D092D703E092D803F092B9
:10749000D903809136048111DACF80915701813070
:1074A000B1F610925701D3CF009709F46ECF4FCFAA
:1074B0008093390420E040E070E060E089E696E3E4
:1074C0000C94E22DCF938091E303811109C086EEE5
:1074D0009EE0909328048093270481E08093E30347
:1074E0000E94FA2320E040E070E060E082EA99E246
:1074F0000E94E22DC1E0C09338040E941A8DDADCAC
:10750000C093380460E087E99EE20E94412482EE45
:107510009EE090934E0580934D05CF9108959091F4
:10752000651394FB882780F994FF06C081E0909151
:107530006D11911101C080E008958091ED058230B8
:1075400059F0EDDF882349F08091651382FB88278D
:1075500080F991E08927089581E008950E9438B765
:10756000DEDF882351F08091651382FD06C081EF34
:107570009EE090934E0580934D050C9471A6109259
:10758000F50510926201CBDF9091651380FB97F9AE
:107590009093651360E084ED9EE00E9441240C947A
:1075A000562FA4E0B0E0E7EDFAE30C944EEE109213
:1075B000D5058091B4051092B405882361F020E0D0
:1075C00040E070E060E085E599E70E94E22D2496B6
:1075D000E0E10C946AEE209121013091220140916A
:1075E000C0055091C105CA01820F931F2436310591
:1075F00009F021C44730510544F006978A309105BF
:107600000CF028C48AE090E02FC406964A3F5F4FF2
:10761000ACF380913704882309F4CCC160915911EF
:1076200070915A11072E000C880B990B0E946CE781
:10763000B1E0B98320915511309156114091571105
:10764000509158110E94E7EF18160CF019826091C2
:10765000980570919905072E000C880B990B0E94D4
:107660006CE72091940530919505409196055091D5
:1076700097050E94E7EF18161CF4E981E260E983A0
:10768000C980C092CF03C0906D01D0906E01E09090
:107690006F01F09070018091710190917201A09141
:1076A0007301B091740189839A83AB83BC8380900A
:1076B000750190907601A0907701B090780120E05C
:1076C00030E04AE754E4C501B4010E94CBE72B0146
:1076D0003C0120E030E0A901C501B4010E9466E749
:1076E00020E030E040EA50EC87FD04C020E030E0CC
:1076F00040EA50E4C301B2010E9484EE2DEC3CEC60
:107700004CEC5DE30E94CBE70E9463EF4B015C0110
:1077100080E2B7FE09C0B094A09490948094811C3C
:10772000911CA11CB11C8DE280933D0460E290E1AC
:10773000891697E29906A104B1048CF0C501B40141
:1077400020E137E240E050E00E940FEECA01B901AB
:107750002AE030E040E050E00E940FEE605D609370
:107760003E0460E2A8EE8A16A3E09A06A104B104E2
:107770008CF0C501B40128EE33E040E050E00E94F7
:107780000FEECA01B9012AE030E040E050E00E946B
:107790000FEE605D60933F04C501B40124E630E064
:1077A00040E050E00E940FEE6AE0462E512C612C22
:1077B000712CCA01B901A30192010E940FEE605D14
:1077C00060934004C501B401A30192010E940FEE31
:1077D0004B01CA01B901A30192010E940FEE88205A
:1077E00009F452C32EE220934104605D6093420489
:1077F000B0E38B0E809243046DE374E087EC93E07A
:107800000E94A8F020E030E0A901C701B6010E9463
:1078100066E720E030E040E05FEB87FD04C020E059
:1078200030E040E05FE3C701B6010E9484EE0E94B1
:1078300063EFCB010E9403AABC0182EC93E00E949B
:10784000A8F020E030E0A90169817A818B819C81D8
:107850000E9466E720E030E040E05FEB87FD04C077
:1078600020E030E040E05FE369817A818B819C8198
:107870000E9484EE0E9463EFCB010E9403AABC0128
:107880008DEB93E00E94A8F0E0912104EF77E9836B
:10789000E1112AC08091651383FD08C340DE88236F
:1078A00019F180915D1390915E13A0915F13B091D7
:1078B00060130097A105B105B9F0BC01CD016D5968
:1078C0007F4F8F4F9F4F24E630E040E050E00E9412
:1078D00094ED6091611370916213809163139091A4
:1078E00064130E9494ED29830E9424A64B015C013D
:1078F000162F80911301C9808C15C1F0C09213011D
:1079000028E4C29EB001112490E080E00E946AE762
:107910002AE037ED43E25CE30E94CBE70E9468EF88
:107920006093BC03C110C5C21092B70380911201CD
:10793000181709F43FC080921201C501B40120E17B
:107940003EE040E050E00E9494ED690189019CE333
:10795000492E512C612C712CC501B401A301920157
:107960000E9494ED4B015C01CA01B901A30192018F
:107970000E9494EDC114D10409F0A4C29F928F9289
:107980007F936F938FE79DE09F938F9387EA93E0B8
:107990009F938F930E94FFE60FB6F894DEBF0FBE51
:1079A000CDBF85E0982F990F990F891B880F8058BC
:1079B0008093A6030E9465BC0091A1031091A203CD
:1079C0002091A3033091A4036B017C01C01AD10A5A
:1079D000E20AF30A9701860137FD11C02091A00346
:1079E00020952093A0036A547C4F8F4F9F4F609344
:1079F000A1037093A2038093A3039093A403D09058
:107A0000A003D98281E00E946226809130128731E2
:107A100080F480913212843060F082E6E82E8EE0AD
:107A2000F82E03E126E044E064E08CEF91E10E944F
:107A300026C08091CF03982F927042E102E081FF2F
:107A400002C048E00CE080913012843180F48091D3
:107A50003212841760F0992309F453C28EE39EE03A
:107A60007C0123E060E58CEF91E10E9426C08091CB
:107A700030128431C0F4809132128230A0F0C9807B
:107A8000CC2009F441C280912706882309F43CC226
:107A900082E09EE07C0102E123E042E068E68CEFB8
:107AA00091E10E9426C0809130128C3108F09DC077
:107AB0008090551190905611A0905711B090581188
:107AC000C0905911D0905A11843198F4809132129B
:107AD000883078F08091CF0380FF19C284EB9DE05D
:107AE0007C010CE022E048E069E38CEF91E10E9428
:107AF00026C080913012883040F4D7FE0BC248E98E
:107B00005DE067E087E30E94D228809130128C31DB
:107B1000B0F480913212843190F020E030E040E007
:107B20005FE3C501B4010E9484EE0E9463EF77FF1A
:107B300014C248E95DE06CE187E30E94D228C0905E
:107B40009405D0909505E0909605F090970580916A
:107B50003012883060F4809198059091990597FFD4
:107B60001FC248E95DE067E081E50E94D22880916C
:107B700030128C31B0F480913212843190F020E0D8
:107B800030E040E05FE3C701B6010E9484EE0E944E
:107B900063EF77FF27C248E95DE06CE181E50E9471
:107BA000D228809130128C3100F5809132128431CC
:107BB000E0F0809127068823C1F024E6829FC0016F
:107BC000112481589F4F6FEF70E00E94FCEDCB01B4
:107BD0000E9482AAAC016CE187E60E94B62A65E2A7
:107BE00070E080E090E00E94732699DC882379F1B0
:107BF00080913012843358F5809132128A3238F1F4
:107C000007E028E04AE26AE28CEF91E10E94CDBEF3
:107C100005E022E04CE262E38CEF91E10E94CDBEF0
:107C200024E04AE061E38AE20E949DBE6091FE1179
:107C30007091FF1182E3809318128BE280931912E6
:107C400028E132E142E38CEF91E10E949DBD8091F9
:107C50003012853350F480913212813330F024E0B9
:107C60004AE461E386E30E949DBE80913012843332
:107C700068F480913212823348F002E02091BC0314
:107C800042E367E38CEF91E10E94CDBE8091301218
:107C90008033D8F4809132128832B8F08091B703E3
:107CA000882361F047EB53E060E387E30E94B62A44
:107CB00065E270E080E090E00E94732647EA53E0BE
:107CC00060E38091A6030E94B62A80913012883228
:107CD00008F060C0809132128D3108F45BC02BE057
:107CE00040E86DE180E00E949DBE809130128732B5
:107CF00008F050C0809132128F3108F44BC083E0FD
:107D00008093331216E21093341268E570E080E03D
:107D100090E00E9473268BE080933312109334120C
:107D2000C980CC2009F481C182EC93E00E94B02983
:107D300088E28093331216E21093341269E570E002
:107D400080E090E00E94732680E3809333121093CA
:107D50003412C980CC2009F48BC18DEB93E00E94D2
:107D6000B0298DE48093331216E2109334126AE541
:107D700070E080E090E00E94732685E580933312E6
:107D800010933412C980CC2009F495C187EC93E09C
:107D90000E94B02980913012833338F580913212DD
:107DA0008B3218F183E00E94622683E080933312C5
:107DB00083E38093341266E070E080E090E00E94FC
:107DC000732681E00E946226809121019091220118
:107DD0000E9482AAAC0163E38CE00E94B62A65E2AD
:107DE00070E080E090E00E94732680913012813430
:107DF00008F0EDCB80913212863308F4E8CB109274
:107E000033128EE38093341286EE9EE00E94762534
:107E1000182F863108F072C186EE9EE00E94B029CC
:107E2000153109F4D4CB60E270E080E090E00E946C
:107E300073261F5FF5CF243631054CF48536910546
:107E400004F58A30910534F48AE090E009C0843664
:107E50009105BCF0883EA3E09A0714F087EE93E00A
:107E60002817390709F4D5CB90932201809321017B
:107E70001092C0051092C1051092C2051092C30560
:107E8000C8CB84E690E0F0CF662351F02EE2209339
:107E90004104605D6093420480E280934304ACCC73
:107EA00080E28093420480934104F6CFF4E6F983A4
:107EB0001BCD89810E94B7AABC0187EB93E00E9489
:107EC000A8F034CD0436110538F47F936F93DF9218
:107ED000CF9283E79DE058CD7F936F93DF92CF924F
:107EE00089E69DE09F938F9387EA93E09F938F931A
:107EF0000E94FFE60FB6F894DEBF0FBECDBF86E04E
:107F000051CD88E39EE0ACCD8CEC9DE0C3CD8CE9F7
:107F10009DE0E6CDC6010E9482AAFC01808193E02B
:107F2000803229F4818192E0803209F491E043E0CB
:107F300050E0491B51094E0F5F1F892F880F880F92
:107F4000981B892F67E0805C0E94B62A69E070E088
:107F500080E090E00E947326D8CDCB010E9482AAD7
:107F6000FC01808193E0803229F4818192E08032AB
:107F700009F491E043E050E0491B51094E0F5F1FA7
:107F8000892F880F880F981B892F6CE1805C0E94D5
:107F9000B62A69E070E080E090E00E947326CFCDC1
:107FA0000E9482AAFC01808193E0803229F48181C1
:107FB00092E0803209F491E043E050E0491B51091E
:107FC0004E0F5F1F892F880F880F981B892F67E03E
:107FD000865A0E94B62A69E070E080E090E00E9434
:107FE0007326C5CDCB010E9482AAFC01808193E05B
:107FF000803229F4818192E0803209F491E043E0FB
:1080000050E0491B51094E0F5F1F892F880F880FC1
:10801000981B892F6CE1865A0E94B62A69E070E0AD
:1080200080E090E00E947326BCCD87E00E942B9CEC
:1080300080FF13C002EC13E0D8016D918D0166231F
:1080400009F476CE6F320CF06FE3062E000C770B3E
:10805000880B990B0E947326EFCF80914B0580FD12
:1080600063CE6FEF7FEF83E99DE00E94CE2760CE65
:1080700087E00E942B9C81FF13C00DEB13E0D80119
:108080006D918D01662309F46CCE6F320CF06FE3B5
:10809000062E000C770B880B990B0E947326EFCFEE
:1080A00080914B0581FD59CE6FEF7FEF83E99DE015
:1080B0000E94CE2756CE87E00E942B9C82FF13C0E1
:1080C00007EC13E0D8016D918D01662309F462CEAF
:1080D0006F320CF06FE3062E000C770B880B990BB8
:1080E0000E947326EFCF80914B0582FD4FCE6FEF3C
:1080F0007FEF8BE89DE00E94CE274CCE81E0C980C7
:10810000C11001C080E09091A5038917C9F0D090FB
:10811000E50ED9828093A50386EE9EE00E94762527
:10812000D81608F054C029812F5F2983E22FF0E090
:10813000EA51F14F8081807C8038A9F32093E50ECD
:108140000091E50E10E00A51114FC8010E947625FA
:10815000898360E870E0C8010E94DA2849814531CE
:1081600008F035CA60E270E080E090E00E9473267B
:108170006981643109F42BCA60E270E080E090E02C
:108180000E9473268981833109F421CA60E270E07C
:1081900080E090E00E9473269981923109F417CA19
:1081A000292F30E02E5F3F4F4AEF4203B001439F3B
:1081B000700D112460587F4F86EE9EE00E94DA28F1
:1081C00060E270E080E090E00E94732600CA1092A6
:1081D000E50EB6CF81E008959091C00095FFFCCFE9
:1081E0008093C6000895CF93DF93EC018991882393
:1081F00011F0F2DFFBCFDF91CF910895CF93DF93A2
:10820000EC018991882311F0E7DFFBCF8DE0E4DFFB
:108210008AE0E2DFDF91CF910895CF93DF93EC0105
:10822000FE0184912196882311F0D6DFF9CFDF91EA
:10823000CF9108954F925F926F927F928F929F920B
:10824000AF92BF92CF92DF92EF92FF921F93CF93A4
:10825000DF93CDB7DEB762970FB6F894DEBF0FBEDF
:10826000CDBF9091E80B93FD67C1F82E89E40E9481
:10827000C11C882309F489C10E941E2190E01816B0
:10828000190614F481E090E026E0289FF001299F70
:10829000F00D1124E955FA4F82819381198A8337B1
:1082A000910514F083E790E09093990580939805E9
:1082B0000E94AE1D6091980570919905072E000CE3
:1082C000880B990B0E946CE72091940530919505DD
:1082D00040919605509197050E94E7EF18160CF40F
:1082E0001AC187E29BE060E00E94412461E06F25B3
:1082F0008F2D0E94BDA6FF2009F41EC121E020930E
:1083000062011D821E821F82188619861A861B86AC
:108310001C8680E09CE3ACE1B6E48D879E87AF8746
:10832000B88B812C912C90E8A92E9FEBB92E1A8A3C
:1083300011E0412C512C3201609198057091990502
:10834000072E000C880B990B0E946CE76B017C01D7
:10835000A50194010E9466E78823A9F02091940565
:108360003091950540919605509197059989911105
:10837000D5C0C701B6010E9466E7881F8827881FFD
:108380008A8B460157010E9465BC6B017C01DC01B0
:10839000CB0129853A854B855C85821B930BA40B09
:1083A000B50BB7FD2CC0D701C60188519C4FAF4F0C
:1083B000BF4F89879A87AB87BC8780E00E94248360
:1083C00083E29BE02ADF411451046104710409F443
:1083D000CDC0C301B201605F784D8F4F9F4F6C19C4
:1083E0007D098E099F0928EE33E040E050E00E94AD
:1083F00094EDCA01B9010E94BC2A8AE0EDDE0E9418
:1084000059C50E9465BC6093FC057093FD0580937F
:10841000FE059093FF0520919405309195054091BC
:1084200096055091970529833A834B835C83C50158
:10843000B4010E9483EE9F774114510461047104DA
:1084400009F097C020E030E040E85FE30E9466E773
:1084500087FF0FC0412C512C3201112331F085E0F0
:10846000482E8DE0582E612C712C4C0C5D1C6E1C1E
:108470007F1C3A893323C1F18D819E81AF81B885FC
:10848000892B8A2B8B2B61F0D701C6012D813E8170
:108490004F815885821B930BA40BB50BB7FD24C0ED
:1084A00029813A814B815C816D857E858F85988994
:1084B0000E9483EE20E030E040E85FE30E9466E740
:1084C00087FD32C0D701C601805A9541AF4FBF4FDB
:1084D0008D839E83AF83B88729813A814B815C81EC
:1084E0002D873E874F87588B809162018823E1F06A
:1084F000411451046104710461F030E1C31A37E2A0
:10850000D30AE108F108C418D508E608F708F7FE11
:108510000BC010E011CF86E39BE0E5CEC701B601AA
:108520000E9466E787FF1EC080916201882321F0C8
:10853000109262010E9438B762960FB6F894DEBFBF
:108540000FBECDBFDF91CF911F91FF90EF90DF90D5
:10855000CF90BF90AF909F908F907F906F905F90E3
:108560004F900895460157011A8A0DCF8FE334DEEC
:1085700044CF20E030E040E450E40E94E7EF1816DA
:108580000CF077CF2601370174CF83E50E94C11C20
:10859000898B811107C0FF2079F282E50E94C11CFE
:1085A000882351F20E944F217ACE0F931F93CF93CD
:1085B0008C01C62F8EEF9AE030DEC8012EDE8AE3F2
:1085C0000BDE80E38C0F08DE8AE006DECF911F9180
:1085D0000F910895CF92DF92EF92FF926A017B0193
:1085E0001CDE42E0C701B6010E9482B3FF90EF900B
:1085F000DF90CF900895EEDF8AE0EECDADE5B0E0FC
:10860000E4E0F3E40C944CEE70E060E085E40E945A
:1086100052217C01182F8F3FB1F1882341F087ED63
:108620009CE0FBDDC35ADF4FE2E10C9468EE6EEB99
:1086300070E083E50E9452215C0165E070E083E414
:108640000E9452216C0160E085E50E943E212C963B
:108650008FAF2C9760E08AEC9CE00E9441240E943E
:1086600065BC69877A878B879C871F3F09F067C441
:1086700034E7A316B1040CF489C18FE99CE0CDDD89
:108680000E9438B7CFCF6CE370E0D3CF20E030E06A
:1086900040E05EE32BAF3CAF4DAF5EAFABC12AE92C
:1086A00039E949E15FE323962CAF3DAF4EAF5FAFB1
:1086B0002397ADC1409055115090561160905711BD
:1086C0007090581151C22B96EEADFFAD2B974083A1
:1086D000A4C24BEEC42ED12CE12CF12C22C384E198
:1086E00090E0A0E0B0E08D879E87AF87B88B34E143
:1086F000C32ED12CE12CF12C24C3CD86DE86EF864F
:10870000F88A1FC32B96EEADFFAD2B978083E9C38C
:10871000D501C4012EA53FA548A959A9821B930BD9
:10872000A40BB50BB7FD47C02D968FAD2D970E94BA
:1087300024838AE051DDD501C4018053984FAF4FA7
:10874000BF4F8EA79FA7A8ABB9AB9AA991116FC0D5
:108750002BA93CA94DA95EA9C301B2010E94E7EF74
:1087600018160CF050C020E030E040E050E4C301A7
:10877000B2010E9484EE6BAB7CAB8DAB9EAB2AA5A5
:108780003BA54CA55DA5280D391D4A1D5B1D2FABD2
:1087900038AF49AF5AAF6D966CAD7DAD8EAD9FAD24
:1087A0006D970E946CE7A30192010E9466E7881F03
:1087B0008827881F8AAB89859A85AB85BC85898F78
:1087C0009A8FAB8FBC8F29893A894B895C8928178E
:1087D00039074A075B0720F4298F3A8F4B8F5C8F4C
:1087E000898D9A8DAB8DBC8D881A990AAA0ABB0A0D
:1087F00091E889169FE4990692E1A906B10460F117
:1088000083EC9BE02DC2D501C4012FA938AD49AD41
:108810005AAD821B930BA40BB50B4EEC55E26DEDDC
:1088200075E2B7FDC8CF812F0E945486C4CF6996E8
:108830006CAD7DAD8EAD9FAD69970E946CE79B01DD
:10884000AC01C301B2010E9466E787FFB4CF4BE0E1
:1088500056E26BE176E2E7CF2996AEADBFAD299740
:10886000A215B3050CF08FC0B3E02B1631040CF445
:108870008AC086E69BE0D1DC1F3F09F066C0E6E5D2
:10888000FBE0FE83ED8385E49BE0C7DC8D819E8168
:10889000C4DC49815A816B817C8182E69BE0ABDE3E
:1088A00085E49BE0BADC8D819E81B7DC4D8D5E8DC9
:1088B0006F8D78A18EE59BE09EDE85E49BE0ADDCCC
:1088C0008D819E81AADC49A15AA16BA17CA18AE578
:1088D0009BE091DE2C963FAD2C97332309F4D0CE4C
:1088E0002CEA35EC47E25EE36D8D7E8D8F8D98A18D
:1088F0000E94CBE76B017C0120E030E543EC50E4C3
:1089000069A17AA18BA19CA10E94CBE729813A8120
:108910004B815C811F3FF1F420939B0530939C05B4
:1089200040939D0550939E05C0929F05D092A0054F
:10893000E092A105F092A2056093A3057093A405AF
:108940008093A5059093A6059BCE20E13EE23E8351
:108950002D8399CF20935C1130935D1140935E116C
:1089600050935F11C0926011D0926111E092621138
:10897000F092631160936411709365118093661196
:10898000909367117DCE0E949337CEC08BE89CE018
:1089900044DC0E94CF838FE780939A052CE330E07C
:1089A000C9A6A8EEB3E00E94C0ED6AA77BA78CA77A
:1089B0009DA729853A854B855C85260F371F481F63
:1089C000591F2FAB38AF49AF5AAF81E08093620196
:1089D00060E087E79CE00E94412402E00E0D023037
:1089E00008F054CE8BEA9AEAAAEABEE38BAF9CAFBA
:1089F000ADAFBEAF023008F052CE8DEC9CECACE4D3
:108A0000BEE323968CAF9DAFAEAFBFAF23970230CE
:108A100008F4E12C2D96EFAE2D9789859A85AB85CC
:108A2000BC85898B9A8BAB8BBC8B8EA79FA7A8AB81
:108A3000B9AB19A21AA21BA21CA21D8E1E8E1F8EDC
:108A400018A219821A821B821C822FE730E040E0B4
:108A500050E02D873E874F87588B80E090E4ACE153
:108A6000B6E48D839E83AF83B8871D8A1E8A1F8AD2
:108A7000188EFFE7CF2ED12CE12CF12C1AAA1BAABD
:108A80001CAA1DAA1EAA1DA21EA21FA218A691E022
:108A900024969FAF2497312C212C412C512C32014C
:108AA00095010B2C000C440B550B61962CAF3DAF80
:108AB0004EAF5FAF619749A5042E000C550B299668
:108AC0005FAF4EAF299757E11502C0011124DC01B9
:108AD000A55ABE4E2B96BFAFAEAF2B97C5014E9693
:108AE0009C01092E000C440B550B65962CAF3DAF35
:108AF0004EAF5FAF6597CC979C01990F440B550B18
:108B000069962CAF3DAF4EAF5FAF699736E0A31AC1
:108B1000B108C5010B2C000CAA0BBB0B6D968CAFDA
:108B20009DAFAEAFBFAF6D9780916201882309F40E
:108B300098C00E9465BC4B015C0190919B046E96AD
:108B40009FAF6E97992309F47BC00E944A871092C9
:108B50009B041F3F09F0AECD4090940550909505C1
:108B60006090960570909705A30192016D897E89AA
:108B70008F89988D0E94E7EF87FF04C04D8A5E8A37
:108B80006F8A788EA30192016D817E818F81988595
:108B90000E9466E7181624F44D825E826F82788602
:108BA00061966CAD7DAD8EAD9FAD61970E946CE717
:108BB000698F7A8F8B8F9C8F2496AFAD2497AA23D1
:108BC00009F454C09B01AC01C301B2010E94E7EF5C
:108BD0001816B4F5D501C40129893A894B895C89F5
:108BE000821B930BA40BB50BAC01BD01485853413C
:108BF0006109710977FD24C04D855E856F8578898F
:108C00004C195D096E097F097595679557954795CC
:108C10001F3F09F058CD40939A058DA39EA3AFA3A3
:108C2000B8A7298D3A8D4B8D5C8D2D8B3E8B4F8B4C
:108C3000588F89869A86AB86BC8624961FAE249769
:108C400065966CAD7DAD8EAD9FAD65970E946CE76E
:108C5000A30192010E9466E787FF5ACD81EE9BE057
:108C6000DCDA109262010E94CF830ACD298D3A8D01
:108C70004B8D5C8DC301B2010E9466E787FFE0CF98
:108C8000D501C40129853A854B855C85821B930BF0
:108C9000A40BB50BAC01BD014858534161097109E2
:108CA00077FDCECF2114310409F40AC12DA13EA1D4
:108CB0004FA158A5280F391F4A1F5B1F298B3A8BDC
:108CC0004B8B5C8B2DA13EA14FA158A5281B390BC6
:108CD0004A0B5B0BC701B6010E9485ED29893A89D1
:108CE0004B895C890E940FEECD84DE84EF84F88886
:108CF000C20ED31EE41EF51E34E1C316D104E104F6
:108D0000F1040CF4ECCC4CEEC416D104E104F104F3
:108D10000CF0DFCC50E8C516D104E104F1040CF4EA
:108D2000ECCCCD86DE86EF86F88A8EEF90E0A0E070
:108D3000B0E09C01AD012C193D094E095F096901A4
:108D40007A018FE69CE069DA6D857E858F8598894A
:108D50000E94BC2A8AE69CE060DAC701B6010E9444
:108D6000BC2A4D815E816F81788583E69CE032DC90
:108D70004D895E896F89788D8CE59CE02BDC93E0D2
:108D8000291631040CF49CC0C701B6010E946CE79F
:108D900020E030E040E850E40E94CBE769837A832A
:108DA0008B839C832D813E814F8158856D897E897F
:108DB0008F89988D0E9483EE2BED3FE049EC5FE3B5
:108DC0000E94CBE79B01AC0169817A818B819C81F8
:108DD0000E94FBEE27966CAF7DAF8EAF9FAF2797BB
:108DE00069897A898B899C890E946CE72FE632E138
:108DF00043E85AE30E94CBE76D837E838F83988795
:108E000023962CAD3DAD4EAD5FAD239727966CAD4F
:108E10007DAD8EAD9FAD27970E94CBE769837A83A6
:108E20008B839C839B01AC010E9484EE2D813E814B
:108E30004F8158850E94FBEE6D8F7E8F8F8F98A398
:108E40002BAD3CAD4DAD5EAD6D817E818F81988542
:108E50000E94CBE729813A814B815C810E94CBE75C
:108E600069A37AA38BA39CA327964CAD5DAD6EAD91
:108E70007FAD279786E59CE0ADDB4D815E816F81FC
:108E8000788580E59CE0B7DB81E49CE0023010F05F
:108E900082E39CE0C2D949815A816B817C818CE25A
:108EA0009CE098DB4D8D5E8D6F8D78A186E29CE015
:108EB00091DB49A15AA16BA17CA180E29CE09BDBE4
:108EC0008D859E85AF85B8898C0D9D1DAE1DBF1DFE
:108ED000B595A795979587951F3F09F013CC80937B
:108EE0009A052996FFAD2997FF9329A52F933F92C5
:108EF0002F928CE09CE09F938F9387E19CE09F935F
:108F00008F931F920E9424243FEF231A330A0FB637
:108F1000F894DEBF0FBECDBF898D9A8DAB8DBC8D11
:108F20008D839E83AF83B887898A9A8AAB8ABC8AED
:108F30006E969FAD6E9724969FAF249781CE8E2C10
:108F40000E2C000C9908F40183E0EE0FFF1F8A95A8
:108F5000E1F7E35BFE4F868197810F978A159B05AA
:108F60000CF48BCB8BE89CE058D90E94CF8387E12F
:108F7000889DF001899DF00D1124EF5AFE4E8FE778
:108F8000828724E130E00CCDCF93DF936EE074E074
:108F90000E9403B7C0E9D5E04B855C856D857E8571
:108FA00085E094E017DB20E030E543EC50E46F858A
:108FB000788989899A890E94CBE7AB01BC0182E05C
:108FC00094E008DB2CEA35EC47E25EE36B897C89B0
:108FD0008D899E890E94CBE7AB01BC018FEF93E0A6
:108FE0000ADBDF91CF91089560E973E00E9403B737
:108FF0006091F90B7091FA0B8091FB0B9091FC0B37
:109000000E946AE7AB01BC0187E893E0E3DA409194
:10901000290C50912A0C60912B0C70912C0C84E837
:1090200093E0D8DA40912D0C50912E0C60912F0CCA
:109030007091300C81E893E0CDDA40910B065091AD
:109040000C0660910D0670910E068EE793E0D3CA70
:10905000CF93DF9364E373E00E9403B7C9EEDBE0D4
:109060004CA95DA96EA97FA98BE293E0B3DA48AD64
:1090700059AD6AAD7BAD88E293E0ACDA4CAD5DAD45
:109080006EAD7FAD81E893E0B6DADF91CF910895C0
:10909000CF93DF9360E173E00E9403B7C9EEDBE09A
:1090A0004CA15DA16EA17FA187E093E093DA48A572
:1090B00059A56AA57BA58AEA9EE28CDA4CA55DA536
:1090C0006EA57FA587EA9EE285DA48A959A96AA913
:1090D0007BA984EA9EE28FDADF91CF910895CF9346
:1090E000DF936BEE72E00E9403B7C9EEDBE06881AC
:1090F00079818A819B810E946AE7AB01BC0182EE83
:1091000092E068DA6C817D818E819F810E946AE79E
:10911000AB01BC018AEA9EE25DDA688579858A85C1
:109120009B850E946AE7AB01BC0187EA9EE252DAA6
:109130006C857D858E859F850E946AE7AB01BC01A9
:1091400084EA9EE258DADF91CF91089545D883ED05
:1091500092E063C88F929F92AF92BF92EF92FF927C
:109160000F931F93CF93DF938AE592E056D86091D7
:109170008704709188048091890490918A0445E065
:109180000E9482B387E492E048D8C0E0D9E0D15091
:1091900019F080E221D8FBCF8C2F0E94F820CF5FFE
:1091A000C330A1F78AE018D803E614E0C0E080E2FB
:1091B00013D88C2F0E94F8207801D3E080E20CD8DD
:1091C000F70180809180A280B38020E030E0A90187
:1091D000C501B4010E94E7EF87FD03C08BE20E9446
:1091E000EC4045E0C501B4010E9482B3D150FCE0DF
:1091F000EF0EF11CD111E2CF8AE00E94EC40CF5F6C
:109200000C5F1F4FC33099F68AE00E94EC40DF915B
:10921000CF911F910F91FF90EF90BF90AF909F90D3
:109220008F900895811107C080E492E00E940D4163
:109230008AE00C94EC4084E492E0F8CF89E392E079
:109240000C940D4183E392E00C940D41811101C017
:10925000F9CF0895CF93DF93C82F64EF73E00E9496
:10926000ECB68C2FF3DFC1E5D1E14B855C856D85D4
:109270007E858BEE93E0AED920E030E543EC50E400
:109280006F85788989899A890E94CBE7AB01BC01F7
:1092900088EE93E09FD92CEA35EC47E25EE36B89D8
:1092A0007C898D899E890E94CBE7AB01BC0185EE4C
:1092B00093E090D98AE00E94EC40DF91CF9108952D
:1092C000CF9384E50E94C11CC0E08823F1F00E9486
:1092D0001E21C82F1816CCF4B5DF8DE40E94EC4097
:1092E0008091990390919A030E94C02D84E394E0A9
:1092F0000E940D416C2FCC0F770B880B990B0E94AD
:1093000038B18AE00E94EC40CFEF8C2FCF910895C6
:10931000A2E1B0E0EEE8F9E40C944DEE9091E80B98
:1093200093FD72C0082FCCDF182F87FD6DC089E434
:109330000E94C11C882309F47FC00E941E2190E076
:109340001816190614F481E090E026E0289FF00139
:10935000299FF00D1124E955FA4F80819181198AD6
:109360000E94A6BC61E0802F0E94BDA660915911A9
:1093700070915A11072E000C880B990B0E946CE714
:10938000209155113091561140915711509158111B
:109390000E94E7EF1816E4F48EE09BE09F938F9312
:1093A00089E19BE09F938F931F920E9424240F904A
:1093B0000F900F900F900F9031E03A8B46C082E5EE
:1093C0000E94C11C882309F43FC00E944F21C8CFCE
:1093D000298983E09BE0222309F349894A8B35C020
:1093E00060E070E0CB014FC0C701B6010E9466E7A4
:1093F00087FF0EC080916201882321F010926201E4
:109400000E9438B73092F4056296E1E10C9469EE5F
:109410004601570100E098C08FE30E94EC40CFC0A6
:1094200020E030E040E450E40E94E7EF18160CF032
:1094300004C12601370101C183E50E94C11C898B4B
:109440008111C3CF0111BBCF1A8A83E50E94C11CD1
:10945000882331F00E944F219093600180935F0137
:1094600082E40E94C11C882331F00E944F21909316
:109470005A018093590186E40E944A1C882309F40A
:10948000AFCF0E945E2160935B0170935C0180937B
:109490005D0190935E013324339420E030E0A90114
:1094A0000E9466E7811101C0312C3092F40500233F
:1094B00009F4AACF5A89552309F4A6CF1092F405CE
:1094C00081E0809362011D821E821F8218861986A8
:1094D0001A861B861C8680E09CE3ACE1B6E48D878F
:1094E0009E87AF87B88B812C912C90E8A92E9FEB9B
:1094F000B92E00E0412C512C32016091591170912C
:109500005A11072E000C880B990B0E946CE76B0117
:109510007C01A50194010E9466E78823A9F02091AF
:109520005511309156114091571150915811998908
:1095300091115ACFC701B6010E9466E7082F001F9C
:109540000027001F460157010E9465BC6B017C018A
:10955000DC01CB0129853A854B855C85821B930B09
:10956000A40BB50BB7FD2EC0D701C60188519C4F87
:10957000AF4FBF4F89879A87AB87BC87812F0E94E7
:1095800024838FE19BE00E940D414114510461044A
:10959000710409F441CFC301B201605F784D8F4F70
:1095A0009F4F6C197D098E099F0928EE33E040E03A
:1095B00050E00E9494EDCA01B9010E94BC2A8AE0E1
:1095C0000E94EC400E9459C50E9465BC6093FC0556
:1095D0007093FD058093FE059093FF052091551132
:1095E00030915611409157115091581129833A8367
:1095F0004B835C83C501B4010E9483EE9F774114C5
:1096000051046104710409F00BCF20E030E040E820
:109610005FE30E9466E787FF10C03A89412C512C16
:109620003201332331F085E0482E8DE0582E612C35
:10963000712C4C0C5D1C6E1C7F1C0023C1F18D81B4
:109640009E81AF81B885892B8A2B8B2B61F0D70146
:10965000C6012D813E814F815885821B930BA40B3F
:10966000B50BB7FD24C029813A814B815C816D85A2
:109670007E858F8598890E9483EE20E030E040EC63
:109680005FE30E9466E787FDB5CED701C601805A29
:109690009541AF4FBF4F8D839E83AF83B88729819C
:1096A0003A814B815C812D873E874F87588B809113
:1096B0006201882309F49ECE4114510461047104AF
:1096C00061F030E1C31A37E2D30AE108F108C418A7
:1096D000D508E608F708F7FE8DCE1A8A0ECFA5E268
:1096E000B0E0E5E7FBE40C944CEE83E50E944A1CF5
:1096F000182F882309F446C10E942F218D83809161
:109700006D0190916E01A0916F01B09170018AA3DB
:109710009BA3ACA3BDA32091710130917201409134
:109720007301509174012E8F3F8F48A359A38091EC
:10973000750190917601A0917701B09178018E8B9F
:109740009F8BA88FB98F112331F09D81911103C098
:1097500080E00E947E2C8091930390919403A091CD
:109760009503B091960325E1B695A79597958795B2
:109770002A95D1F79C01AD01217033274427552745
:109780002A8B3B8B4C8B5D8B0E946B2D882309F4BD
:10979000FDC083E40E944A1C882309F4CEC00E94C5
:1097A0005E216A8F7B8F8C8F9D8F83E6282E84E0CD
:1097B000382E810180E090E0A8ECB2EC8A879B878C
:1097C000AC87BD8720E030E048EC52E42E833F8335
:1097D00048875987D8014D905D906D907C90139784
:1097E00014962D913D914D915C9117972E873F874F
:1097F000488B598B18968D909D90AD90BC901B977F
:1098000069017A01A3019201C701B6010E9466E7CE
:10981000181614F473016201A5019401C701B60181
:109820000E9466E7181614F475016401A7019601F9
:109830006E817F81888599850E9466E7181624F4D9
:10984000CE82DF82E886F986CE84DF84E888F988D4
:10985000A3019201C701B6010E94E7EF87FF02C092
:1098600073016201A5019401C701B6010E94E7EFEF
:1098700087FF02C075016401A70196016A857B8597
:109880008C859D850E94E7EF87FF04C0CA86DB8632
:10989000EC86FD86045F1F4FE7E8F4E0E017F10770
:1098A00009F098CF2A853B854C855D856E817F8147
:1098B000888599850E9484EE20E030E040E05FE3F7
:1098C0000E94CBE72A8D3B8D4C8D5D8D0E9484EEEE
:1098D0004B015C012DEB37E346E855EB0E9466E750
:1098E00087FD0AC02DEB37E346E855E3C501B40117
:1098F0000E94E7EF18160CF580E00E947E2C13E022
:10990000710103E0D7016D917D918D919D917D0154
:109910006D01B4E0CB1AD108A50194010E9483EE39
:10992000F6016083718382839383015059F711504C
:10993000FCE02F0E311C1111E3CF2A893B894C89A1
:109940005D89232B242B252B49F00E946B2D882326
:1099500029F08EEA92E00E940D41FCDB8AE50E942C
:109960004A1C882359F00E945E2169837A838B8385
:109970009C8360E0CE0101960E949E2C8D810E9406
:109980007E2C14C020915E042D83B9CE2D8121112F
:1099900008C08A899B89AC89BD89892B8A2B8B2B2E
:1099A000E9F250DC84EC92E00E940D413D813323CA
:1099B00049F080915E04811105C040DC8FE892E09F
:1099C0000E940D413FDC81E892E00E940D418091B0
:1099D0005E0428DC37DC84E792E00E940D41C090F1
:1099E0005F04D0906004E0906104F090620420E095
:1099F00030E0A901C701B6010E94E7EF18160CF08C
:109A000040C042E0C701B6010E9482B38DE00E94CF
:109A1000EC408AE00E94EC402AA13BA14CA15DA150
:109A200060916D0170916E0180916F019091700154
:109A30000E9466E781111FC02E8D3F8D48A159A15C
:109A40006091710170917201809173019091740124
:109A50000E9466E781110FC0209175013091760157
:109A600040917701509178016E897F89888D998D19
:109A70000E9466E781110E9401A1A596E2E10C9483
:109A800068EE8FE692E00E940D41C6CFCF93DF9340
:109A9000EB010E940D41BE01DD0F880B990B0E9466
:109AA00038B1DF91CF910895EC018B01F42E0E9423
:109AB000CF83209709F47AC0C5DBCE010E940D4107
:109AC0008AE00E94EC400115110511F400E11EE24C
:109AD0000E94F7241F930F93DF93CF9383E092E0CC
:109AE0009F938F9381E08F930E9424240E94562F8E
:109AF000C091FD11C695C69588EF91E10E949B2704
:109B0000DC2FDD0F1D2F1C0F8DB79EB707960FB6EC
:109B1000F8949EBF0FBE8DBF83E00E94622646EE82
:109B20005EE06C2F80E00E94B62A10923312D09330
:109B300034126FEF7FEF84EF91E00E94CE271092F6
:109B40003312109334126FEF7FEF87EE91E00E9493
:109B5000CE278CEF91E10E9420BF8111DDCF6EDB1B
:109B600083E192E00E940D4189EE93E0019739F084
:109B700000C00000EEE5F9E03197F0F7F7CFF89478
:109B800089EE93E0019739F000C00000E6EEF3E0C3
:109B90003197F0F7F7CF0E94CF83FF2021F00E948A
:109BA000E889A895FECF0E94A389FBCF0115110576
:109BB00011F400E11EE2CAE0D2E08ACF8091330CBA
:109BC0009091340C2FEF3FEF981751F0E92FF0E010
:109BD000ED5CF34F228130E09F5F9F779093340CD0
:109BE000C90108951F920F920FB60F9211240F9082
:109BF0000FBE0F901F9018951F920F920FB60F92E5
:109C000011240BB60F922F938F939F93EF93FF9393
:109C10009091C6002091340CE091330C81E08E0FBE
:109C20008F77281729F0F0E0ED5CF34F9283E82F4F
:109C3000E093330CFF91EF919F918F912F910F90B3
:109C40000BBE0F900FBE0F901F9018958EBD0DB4D8
:109C500007FEFDCF08958FEF8EBD0DB407FEFDCF3B
:109C60008EB50895909164009B7F90936400982F27
:109C7000906A96959CBD80FD03C091E0863009F402
:109C800090E09DBD0895ADE2B0E0E9E4FEE40C94FF
:109C90004CEE8DA72091EF0528A721E02093EF053A
:109CA00080919B038D3409F46FC5843511F40C94B5
:109CB0008162873489F48091990390919A038C3161
:109CC000910509F4FCC1A8F48430910509F4BEC1E2
:109CD00030F4029708F421C10E94D6B602C045971D
:109CE000D9F7EDA5E1110C94635B0E94C3B60C9407
:109CF000635B8A35910509F439C508F0BDC08D3123
:109D0000910509F45CC38A9739F780910A0683307C
:109D100040F389E40E94C11C082F10E0882319F049
:109D20000E944F21182F8AE40E94C11CF82E88231C
:109D300009F40BC50E944F2101110BC5833008F0B7
:109D40000CC590E1EDE6F1E0A5E4B4E001900D92E0
:109D50009A95E1F7002391F034E01302F001112409
:109D6000EE5BFD4E408151816281738140934504D9
:109D7000509346046093470470934804FF2091F089
:109D800094E08902F0011124EA5CFD4E808191810A
:109D9000A281B3818093490490934A04A0934B0419
:109DA000B0934C0486E40E94C11C882309F4DAC4F1
:109DB0000E945E216B017C0120E030E0A9010E943D
:109DC000E7EF87FF03C0C12CD12C760129E838E8E2
:109DD00048E85CE3C701B6010E94CBE76B017C0158
:109DE00080901D0190901E01A0901F01B090200155
:109DF00020E030E0A9010E9466E7882341F0C0928C
:109E00001D01D0921E01E0921F01F09220010091ED
:109E100021011091220184E690E090932201809329
:109E20002101C0906701D0906801E0906901F09035
:109E30006A0180E090E0A0E8BFE38093670190931F
:109E40006801A0936901B0936A010E94469C8092C8
:109E50001D0190921E01A0921F01B092200110934B
:109E6000220100932101C0926701D0926801E09223
:109E70006901F0926A0135CF8B35910509F479C4F7
:109E80008C35910509F028CF3DE7C32E31E0D32E64
:109E90004DE6E42E41E0F42E212C312C10E0D601C9
:109EA0008D916D010E94C11C082F882351F10E94E1
:109EB0005E214B015C01F701208131814281538198
:109EC0000E9483EE2B013C012DEB37E346E855EB76
:109ED0000E9466E787FD0AC02DEB37E346E855E3AD
:109EE000C301B2010E94E7EF18165CF4133011F0C1
:109EF000202E032DD7018D929D92AD92BC92139787
:109F0000302E1F5FB4E0EB0EF11C143041F622201E
:109F100009F433C40E9404A001C480910A0683306E
:109F200008F4DFCE65E4C62E64E0D62E7DE6E72E8B
:109F300071E0F72E10E088E5810F0E94C11C882394
:109F400009F468C00E945E214B015C01812F0E94D0
:109F5000231C882359F0D7012D913D914D915C919F
:109F6000C501B4010E9484EE4B015C01F6018082C0
:109F70009182A282B3821F5FF4E0CF0ED11C24E055
:109F8000E20EF11C1330B9F685E40E94C11C88234F
:109F900009F44BC00E945E216B017C0183E00E94AA
:109FA000231C882371F02091790130917A0140912E
:109FB0007B0150917C01C701B6010E9484EE6B01C8
:109FC0007C01C0925104D0925204E0925304F0926A
:109FD000540486E40E94C11C8823C9F00E945E21BB
:109FE00020E030E0A9010E94E7EF181684F40E94F7
:109FF0005E2129E838E848E85CE30E94CBE76093FB
:10A000001D0170931E0180931F01909320010E94F7
:10A01000469C67CEF70180819181A281B381F601D0
:10A0200080839183A283B383A6CF8091790190919D
:10A030007A01A0917B01B0917C01809351049093AF
:10A040005204A0935304B0935404C3CF80E50E94FC
:10A05000C11CC12CD12C7601882321F00E94FE2046
:10A060006B017C0183E50E94C11C882361F00E9482
:10A070005E2120E030E04AE754E40E94CBE70E94F2
:10A0800068EF6B017C010E941A8D8091E60E8111B0
:10A0900005C060E087E494E00E9441240E9465BC12
:10A0A000C60ED71EE81EF91E0E9465BC6C197D09FC
:10A0B0008E099F0997FF15CE0E9459C5F5CF87E0FD
:10A0C0000E942B9C811111C0809193039091940365
:10A0D000A0919503B09196035EE0B695A7959795EC
:10A0E00087955A95D1F780FDFCCD0E941A8D10926C
:10A0F000280160915E048CE40E943E21A82E80E03D
:10A100000E947E2C0E9465BC6093FC057093FD0547
:10A110008093FE059093FF0580911D0190911E0193
:10A12000A0911F01B0912001809374039093750357
:10A13000A0937603B093770380912101909122013F
:10A14000909373038093720384E690E090932201CE
:10A150008093210181E080934A050E940FA58091A0
:10A16000930390919403A0919503B0919603A7FB5C
:10A17000112710F92B2F2170B1FB882780F91213BA
:10A1800003C0811709F410C1B22E982E82E50E94F7
:10A19000C11C412C512C40EA642E40E4742E8823CB
:10A1A00059F00E945E212B013C0120E030E0A90122
:10A1B0000E9466E78823D1F1111103C0BB2009F486
:10A1C000C5C0C0907501D0907601E0907701F09005
:10A1D0007801A3019201C701B6010E94E7EF87FF52
:10A1E00002C07301620180E090E0A0E8B0E48C8FCF
:10A1F0009D8FAE8FBF8F20E030E04AE753E4C70168
:10A20000B6010E9466E7181634F4C12CD12C3AE747
:10A21000E32E33E4F32EC982DA82EB82FC82BE01A4
:10A22000645E7F4FCE0101960E94E69F112309F4E0
:10A2300088C0BB2009F482C010926D0110926E019B
:10A2400010926F01109270011092710110927201C0
:10A2500010927301109274010E9404A0EEE2FAE1E0
:10A26000C590D590E590F490E2E3FAE145905590E1
:10A2700065907490A7019601C301B2010E9466E740
:10A2800087FF98C0A7019601C301B2010E94FBEEAF
:10A290009B01AC010E94CBE720E030E040E85FE3A7
:10A2A0000E9484EE0E9420F021E030E048E452E475
:10A2B0000E94CBE769837A838B839C8380917501AD
:10A2C00090917601A0917701B091780188A399A32C
:10A2D000AAA3BBA320E030E040EC5FE3C301B201DE
:10A2E0000E94CBE72B013C0177FA709477F87094C9
:10A2F00020E030E040EC5FE3C701B6010E94CBE70D
:10A300009058DE0111966D01E8A0F9A00AA11BA1E9
:10A31000A30192010E945C9F0E9416A610926D01FB
:10A3200010926E0110926F011092700110927101E3
:10A3300010927201109273011092740180E00E94D9
:10A3400006A0BB2019F081E00E9406A0992019F018
:10A3500082E00E9406A00E9404A08091490580939B
:10A360004A05AA2019F081E00E947E2C8091740396
:10A3700090917503A0917603B091770380931D01AE
:10A3800090931E01A0931F01B0932001809172034E
:10A3900090917303909322018093210183E0809335
:10A3A00057010E9401A19DCC11E0BB24B3949924D4
:10A3B0009394ECCEA3019201C701B60167CF83E568
:10A3C0000E94C11C882381F10E941E21863028F042
:10A3D0008FE295E00E940D4184CC182F833009F460
:10A3E00053C1B8F4813039F1823009F449C08CE1AD
:10A3F00095E00E940D410E946B2D8823B9F0809159
:10A400005E040E9412490E94AA48123009F086C1D7
:10A41000ABC0843009F489C1853049F780E00E94DF
:10A420007E2C0E946E2C7AC110E0E1CF8EE095E088
:10A430000E940D41EACF0E946E2C109209011092E9
:10A4400008018091340481111BC080919303909185
:10A450009403A0919503B09196032DE0B695A7952E
:10A46000979587952A95D1F780FF07C082E095E000
:10A4700090934E0580934D0534CC8CEF94E0F8CF4B
:10A48000809108019091090197FF05C083ED94E048
:10A490000E940D4126CC009709F097C019821A82BC
:10A4A0001B821C828EEC9CECACE4BEE38C8F9D8FF7
:10A4B000AE8FBF8FBE016F5F7F4FCE014C960E9463
:10A4C000E69F8091080190910901893091050CF077
:10A4D000A6C021E0209328019C012F5F3F4F3093BD
:10A4E00009012093080163E00E94DBED382F80FF13
:10A4F00003C022E0291B922FB4E09B02F00111243B
:10A50000EE5BFD4E608171818281938124E0320295
:10A51000F0011124EA5CFD4E20813181428153819A
:10A52000BDECCB2EBCECDB2EBCE4EB2EBEE3FB2E55
:10A53000CC8EDD8EEE8EFF8E19821A821B821C82DB
:10A54000DE0111966D01E12CF12C00EA10E40E946D
:10A550005C9F19821A821B821C82B601CE014C9626
:10A560000E94E69F10923404E0900801F0900901E7
:10A570008701E9E0EE16F10414F009E010E0B801FB
:10A580008CE694E083DA69E070E087E694E07EDAB6
:10A590008AE00E94EC401E141F040CF0BFC01F9202
:10A5A00089E08F931F930F9380E594E09F938F939F
:10A5B0008EE594E09F938F931F920E9424240FB600
:10A5C000F894DEBF0FBECDBFA9C0815063E00E94EA
:10A5D000DBED80FF03C022E0291B922F292F990F6A
:10A5E000330BF901EE0FFF1FE20FF31FE80FF11D10
:10A5F00087FDFA95EE0FFF1FEE0FFF1FED59FB4F82
:10A600008091750190917601A0917701B0917801C8
:10A6100080839183A283B3831092280152CF80E07C
:10A6200090E0A0EAB0E48093750190937601A09346
:10A630007701B09378018DE191E00E94549F0E94D0
:10A640001A8D8FEF9FEF90930901809308018FEB94
:10A6500094E00E940D4160E08DEA94E00E94412464
:10A6600063E972E084E690E00E947FAC6AEB72E0FE
:10A6700084E690E00E947FAC87EA94E00E94BC628E
:10A6800081E00E947E2C6ECF89E40E94C11C882349
:10A6900079F00E944F218C01833070F062E070E00D
:10A6A00084E994E0F3D981E994E00E940D4119CB4B
:10A6B0008AE40E94A64815CB8AE40E94C11C882324
:10A6C000B9F30E944F217C01B2E0B81750F462E068
:10A6D00070E08EE794E0DAD98BE794E00E940D41B8
:10A6E00000CB8AE50E94C11C8823D9F00E945E211C
:10A6F000002E000C110BF801EE0FFF1FE00FF11FF1
:10A70000EE0DF11DE7FCFA95EE0FFF1FEE0FFF1F98
:10A71000ED59FB4F60837183828393830E9401A173
:10A72000E0CA8AE50E94A648DCCA8AE50E94C11CEC
:10A730008823B9F30E945E21609387047093880494
:10A740008093890490938A04E9CF80E0002309F480
:10A75000F8CA133010F40C94AE6286E495E00E94BF
:10A760000D41BFCA60E070E0CB0124CB10927803AA
:10A77000B8CA8FE080937803B4CA332079F289E7AE
:10A7800091E00E94069BCACF8091990390919A0311
:10A790008237910511F40C94975D08F082C18B34D7
:10A7A000910509F46BC708F0F6C08831910509F4EA
:10A7B0007BC508F0BBC08231910511F40C94665C36
:10A7C00008F06EC08230910508F4DBC4419709F0AF
:10A7D00083CA0E94391C882309F42FC50E94981C43
:10A7E00000918C04102F1095182309F47ACAF12CCB
:10A7F000E12CD12CA12EB12CC5010E2C02C09595B7
:10A8000087950A94E2F780FF08C08E2D0E94EF8999
:10A81000F701EA5DFD4F8081D82A3FEFE31AF30A82
:10A8200083E0E816F10441F713FF05C00E94B189E7
:10A830009D2D9360D92E102B10951D2109F451CA1E
:10A8400088E20E94EC40F12CE12CC12ED12CC601F3
:10A850000E2C02C0959587950A94E2F780FF09C0F7
:10A86000F701E358FE4F80810E94EC4080E20E9495
:10A87000EC40AFEFEA1AFA0AB3E0EB16F10439F74D
:10A8800013FF09C085E40E94EC4080E30E94EC4085
:10A8900080E20E94EC4082E795E00E940D4121CACF
:10A8A0008531910509F4E3C458F5449709F014CAB9
:10A8B0008091651384FFD3C483EA95E00E940D4123
:10A8C0008091651384FF17C080EA91E10E9498800F
:10A8D0008BE1E0EAF1E1DE01119601900D928A959B
:10A8E000E1F770E060E0CE0101960E946CC2CE01FB
:10A8F00001960E94668284E995E00E940D41F1C9AB
:10A900008631910509F4B7C4479709F0E5C98091EC
:10A91000970390919803FC012191222309F4BDC46F
:10A920002032D1F7DF0111971C92F6CF8D319105BE
:10A9300009F451C5A0F48A31910509F4D0C408F492
:10A94000BFC48B31910509F4E9C44C9709F0C4C91F
:10A9500080919703909198030E94EEC0C2C98F31F5
:10A96000910509F4E5C508F43DC58032910509F467
:10A970009AC58934910509F0AFC980E50E94C11CD0
:10A98000882309F4AEC90E941E21853608F084E6AA
:10A9900080932104A6C98836910509F47BC608F086
:10A9A0004CC08235910509F481C7F0F48D349105CE
:10A9B00009F46CC608F466C68135910509F08CC9A6
:10A9C0000E942A8D109227060E94CF830E94A8A67B
:10A9D00068EE73E080E090E00E949B2D60E081E8EB
:10A9E00096E00E9441247DC98435910509F46EC723
:10A9F00008F464C78535910511F40C94005D8C351D
:10AA0000910509F069C90E94604987FD6AC9809172
:10AA1000930384FF02C00C94255D8091950387FF0A
:10AA200002C00C94255D80919603837011F00C9404
:10AA3000255D81E00E940BB754C98D36910509F45C
:10AA40002EC698F48A36910509F444C608F42CC63B
:10AA50008B36910509F47BC68C36910509F03CC90B
:10AA60001092F505109262013CC98F36910509F4E8
:10AA700090C608F47BC68037910509F4C6C68137B5
:10AA8000910509F029C983E50E94C11C882309F4B6
:10AA9000CCC60E941E218D3308F0C2C68093560199
:10AAA00020C98232E1E09E0711F40C946C6008F03A
:10AAB0009DC18A39910509F4D2C608F0E0C08737F4
:10AAC000910511F40C94E85D08F0BCC08537910540
:10AAD00011F40C949F5D10F00C94AF5D83379105D9
:10AAE00009F0FAC88DE498E00E940D4160E08DE322
:10AAF00098E00E94D54260E088E298E00E94D5424A
:10AB000061E081E298E00E94D54260E086E198E051
:10AB10000E94D54261E087E098E00E94D54261E062
:10AB200087EF97E00E94D54260E08EEE97E00E94AA
:10AB3000D54261E084EE97E00E94D54260E08AED64
:10AB400097E00E94D54260E083ED97E00E94D542F5
:10AB500060E08BEC97E00E94D54261E08DEB97E0DE
:10AB60000E94D54261E08FEA97E00E94D54260E002
:10AB700080EA97E00E94D54260E082E997E00E9477
:10AB8000D54260E08CE797E00E94D54260E08BE61A
:10AB900097E00E94D54260E086E597E00E94D542AA
:10ABA00060E087E497E00E94D54261E080E497E0AE
:10ABB0000E94D54260E089E397E00E94D54261E0BF
:10ABC00080E397E00E94D54260E08BE197E00E942D
:10ABD000D54260E08DE097E00E94D54260E080E0E1
:10ABE00097E00E94D54261E08DEE96E00E94D5424A
:10ABF00060E080EE96E00E94D54260E08BED96E04A
:10AC00000E94D54261E08EEC96E00E94D54260E061
:10AC10008AEB96E00E94D54260E087EA96E00E94C7
:10AC2000D54260E086E491E10E94201C682F6170AB
:10AC30008EE996E00E94D54260E080E996E00E94AD
:10AC4000D5424FC88937910509F4CFC708F4C4C766
:10AC50008C38910509F4F9C58139910509F03CC892
:10AC600070E060E083E50E945221823008F4C5C79D
:10AC70000E941E4987E199E00E940D4132C88C3C38
:10AC8000910511F40C94C55E08F04FC08E3B910500
:10AC900009F4E0C550F58B39910509F01DC883E52D
:10ACA0000E94C11C882309F41CC80E941E21182F71
:10ACB0008C3308F08CE3809309060E9465BC6B011D
:10ACC0007C01212F30E0A8EEB3E00E94C0EDC60E5B
:10ACD000D71EE81EF91EC0920506D0920606E09225
:10ACE0000706F09208060C94714E893C910509F410
:10ACF000EEC78B3C910511F00C946C4E8091930340
:10AD000084FF02C00C94A25E80919503887811F0B4
:10AD10000C94A25E80919603837011F00C94A25E55
:10AD200081E00E9448480C94714E833D910511F4D6
:10AD30000C94765FE0F48D3C910511F00C946C4E10
:10AD40008091930381FF02C00C941A5F8091940359
:10AD500081FF02C00C941A5F809195038C7011F0F2
:10AD60000C941A5F81E00E94F4470C94714E8C3D64
:10AD7000910511F40C940F608D3D910511F00C9428
:10AD80006C4E0E946049082F87FF02C00C94714EE0
:10AD900083E50E94C11C002E000C110B7801EE0C03
:10ADA000FF1C882311F40C9452600E944F21F7017C
:10ADB000EF5BFE4F91838083000F111F000F111F67
:10ADC00009591E4FBC01990F880B990B0E946CE723
:10ADD0002AE037ED43E25CE30E94CBE7D8016D93B4
:10ADE0007D938D939C9313970C94714E853A31E02B
:10ADF000930711F40C949E6108F05EC08F32B1E0AD
:10AE00009B0711F40C94966160F58D32F1E09F0779
:10AE100011F40C94C96010F00C9450618C32914084
:10AE200011F00C946C4E83E50E94C11C04E011E00B
:10AE3000882319F00E940E218B0180E50E94C11C1D
:10AE4000882311F40C94C5600E940E21CB0169384F
:10AE5000734110F088E893E1B8010E947FAC0C9434
:10AE6000714E8039A1E09A0711F40C949A61B0F404
:10AE70008033914011F00C946C4E8091930383FFCA
:10AE800002C00C94136180919403817811F00C94AA
:10AE9000136181E00E94C4470C94714E8A39F1E03D
:10AEA0009F0709F4B9C4843A914011F00C946C4E98
:10AEB0000E946F4B0C94714E883F31E0930711F460
:10AEC0000C94576208F011C1853FB1E09B0711F463
:10AED0000C944C6248F4843F914011F00C946C4EF9
:10AEE0000E94048A0C94714E863F21E0920711F46F
:10AEF0000C945062873F914011F00C946C4E61E0CD
:10AF000083E50E943E2111E0182764EB7AE0812F4F
:10AF10000E94ECB6812F0E9426498CEA9AE00E949A
:10AF20000D4189E09AE00E940D418AE00E94EC40C8
:10AF30006AE97AE0812F0E94ECB6812F0E942649AF
:10AF40008DE79AE00E940D41812F0E940BB7812F5F
:10AF50000E944848812F0E946F48812F0E942848F4
:10AF6000812F0E94F44765E27AE0812F0E9403B7A7
:10AF700000915E048CE19AE00E940D41602F70E028
:10AF800090E080E00E9438B140915F0450916004ED
:10AF9000609161047091620487EA9EE20E94EA4235
:10AFA0008FE09AE00E940D4180915E040E94124958
:10AFB0000E946B2D882309F449C093E6C92E94E0C2
:10AFC000D92E00E05601F12C812F0E94264982E7FC
:10AFD0009AE00E940D418F2D0E94F8208FE69AE0A2
:10AFE0000E940D41802F0E94F82087EA9EE20E9475
:10AFF0000D41D5016D917D918D919C9145E00E940F
:10B0000082B38AE00E94EC40F394BCE0AB0EB11C2A
:10B01000E3E0FE12D9CF0F5FF4E0CF0ED11C033076
:10B0200089F6812F0E94264984E69AE00E940D410C
:10B0300060918704709188048091890490918A04BA
:10B0400045E00E9482B38AE00E94EC4069E47AE025
:10B05000812F0E94ECB687EAE82E85E0F82E00E00A
:10B06000812F0E94264980E49AE00E940D41802FA2
:10B070000E94F820D7016D917C91072E000C880B5F
:10B08000990B0E946CE7AB01BC018DE39AE00E9432
:10B09000EA42F70162817381072E000C880B990B3D
:10B0A0000E946CE7AB01BC018AE39AE00E94EA428D
:10B0B000D7011496CD90DC9087E39AE00E940D4171
:10B0C000C6010E94C02D8AE00E94EC40B6E0EB0E63
:10B0D000F11C013011F00C945462812F0E942A4916
:10B0E000812F0E94C4470C94714E803AA3E09A07C6
:10B0F00009F410C2B8F48C30924011F00C946C4EEC
:10B100001091651312FD02C00C94696217FF02C012
:10B110000C9469620E948F3A80FB17F910936513B3
:10B120000C94714E873EF3E09F0711F40C9471620A
:10B13000893E934011F00C946C4E0E941A8D8091C0
:10B140006513877F8B7F809365130E9424A66D33E0
:10B1500071058105910520F088EE9AE00E94BC629D
:10B1600084EE9AE00E94BC6284EE8093210480ED1C
:10B170009AE00E940D418CEC9AE00E94BC620C9413
:10B18000714E80E50E94C11CC12CD12C7601882310
:10B1900021F00E94FE206B017C0183E50E94C11C0E
:10B1A000882361F00E945E2120E030E04AE754E409
:10B1B0000E94CBE70E9468EF6B017C010E941A8D10
:10B1C0008091970390919803009709F10E9454B4DD
:10B1D0001091EF0583E08093EF0581E08093F50502
:10B1E000C114D104E104F10431F00E9465BCC60E23
:10B1F000D71EE81EF91E8091F5058823B1F0C11411
:10B20000D104E104F10449F40E9459C5F4CF60E08F
:10B210008FE595E00E944124DBCF0E9465BC6C194C
:10B220007D098E099F0997FDEFCF1092F5051093C8
:10B23000EF050E9438B70C94714E60E081E895E00C
:10B240000E94412480E00E94EF8981E00E94EF8902
:10B2500082E00E94EF890E94B1890C94714E0E9495
:10B2600022498AE895E00E940D410C94714E0E949B
:10B27000F1C40C94714E8091651382FF04C087FD68
:10B2800002C00C94714E0E946DC0809165138F7E38
:10B290008064809365130C94714E60E00E943AC103
:10B2A000109221040C94714E0E948F3A882321F051
:10B2B0000E947BC00E9471A60E9438B70C94714E08
:10B2C0008091651382FF05C087FD03C08B7F80934B
:10B2D00065130E9493A60E9438B70C94714E80911A
:10B2E000651384FD02C00C94714E83E50E94C11C5D
:10B2F000882311F40C94714E0E940E21AB01BC0105
:10B3000040936113509362136093631370936413BB
:10B310008AE691E10E94B37D0C94714E8091930373
:10B3200090919403A0919503B091960322E0B69575
:10B33000A795979587952A95D1F780FF1DC081EE37
:10B3400095E00E940D4180916D11882381F0BE012E
:10B350006F5F7F4F8AE691E10E948C7FCE0101965C
:10B360000E94F3408AE00E94EC400C94714E84EB02
:10B3700095E00E940D41F6CF8091651382FF25C0B4
:10B38000C0906113D0906213E0906313F090641347
:10B390008FEC95E00E940D41C701B6010E94DBB021
:10B3A0008FE20E94EC4060915D1370915E1380917A
:10B3B0005F13909160130E94DBB08DE00E94EC401F
:10B3C0008AE00E94EC400C94714E8EEB95E00E9456
:10B3D0000D410C94714E809165138E7F809365139F
:10B3E0000C94714E8091651384FD02C00C94714ED3
:10B3F0000E94CFDB8091651384FD02C00C94714ED6
:10B400004091970350919803BE01645E7F4F80E0A6
:10B410000E9421B58C01009711F40C94714E6C8D33
:10B420007D8D19821C8222E0AC01CE0101960E9422
:10B430006B82811116C0F12CCE0101960E946682AA
:10B44000FF2021F1B8018BE096E00E945FC01092CE
:10B4500061131092621310926313109264130C9490
:10B46000714ECE0101960E9457DB882321F361E0E3
:10B47000CE0101960E94727F0097E9F225EEFC0151
:10B4800020831C820E9418C3F82ED6CF83EF95E04C
:10B490000E940D41C8010E94F34080EF95E00E9498
:10B4A0000D410C94714E8091651382FF03C087FF9C
:10B4B0000E941A8D8091651384FD02C00C94714E18
:10B4C00060E080E50E943E21182F682F809197034D
:10B4D000909198030E943AC183E50E94C11C882381
:10B4E00081F00E940E21AB01BC0140936113509387
:10B4F000621360936313709364138AE691E10E9470
:10B50000B37D0E947BC011110C94714E0E9471A6F4
:10B510000C94714E2091970330919803909165138C
:10B52000926090936513C9010E94EEC00C94714E15
:10B530000E9424A66B017C0120E831E541E050E047
:10B540000E9494EDC9016DE671E00E94E8ED4B01A7
:10B550005C01C701B60120E13EE040E050E00E94FE
:10B5600094EDCA01B90128E130E040E050E00E94CA
:10B5700094ED2B013C011B01C701B6012CE330E027
:10B5800040E050E00E9494ED6B017C01CA01B901DA
:10B590002CE330E040E050E00E9494ED8E010F5F1C
:10B5A0001F4F8114910419F1DF92CF927F936F9313
:10B5B0005F924F92BF92AF929F928F9281E496E0FA
:10B5C0009F938F931F930F930E94FFE60FB6F894FB
:10B5D000DEBF0FBECDBFC8010E9454B40E942249F5
:10B5E000B80185E596E00E945FC00C94714EA114ED
:10B5F000B10489F0DF92CF927F936F935F924F9265
:10B60000BF92AF9281E396E09F938F931F930F9326
:10B610000E94FFE6DBCF4114510479F0DF92CF9214
:10B620007F936F935F924F9285E296E09F938F9303
:10B630001F930F930E94FFE6C9CF6115710569F052
:10B64000DF92CF927F936F938DE196E09F938F93DC
:10B650001F930F930E94FFE6B9CFDF92CF9289E14B
:10B6600096E09F938F931F930F930E94FFE60F9096
:10B670000F900F900F900F900F90ADCF0E9471A67A
:10B680000C94714E0E9493A60C94714E0E94A8A631
:10B690000C94714E80E00E9488490C94714E81E0B8
:10B6A0000E9488490C94714E0E946049182F87FDB2
:10B6B0000AC082E696E00E940D41812F0E942483F9
:10B6C0008AE00E94EC40F8A5F093EF05AD96E2E128
:10B6D0000C9468EE80E50E94C11C811132C08091FB
:10B6E000930390919403A0919503B09196030FEF6B
:10B6F00010E080FF04C060912706062F10E089E467
:10B700000E94C11C882309F41FC70E941E2190E0DB
:10B710001816190614F481E090E026E0289FF00145
:10B72000299FF00D1124E955FA4F048115810F3F2F
:10B73000110519F010F00FEF10E0009327060C949C
:10B74000714E0E941E2181110C94714EC8CF80E56C
:10B750000E94C11C811104C0109227060C94714EE6
:10B760000E941E2181110C94714EF6CF8EE40E942E
:10B77000C11C882311F40C94714E0E940E21609319
:10B78000B50C7093B60C8093B70C9093B80C0C94D6
:10B79000714E83E50E94C11C882321F00E941E2166
:10B7A0008093E80B0E94224983E796E00E940D41B6
:10B7B0008091E80B882331F110E000E020E08091D7
:10B7C000E80B90E0002E02C0959587950A94E2F769
:10B7D00080FF12C0FF24F394F20E222319F08CE2B2
:10B7E0000E94EC40F801EE0FFF1FE759F94F8591D9
:10B7F00094910E940D412F2D0F5F1F4F05301105B1
:10B80000F1F6B0CD85E696E0B4CD41E070E060E0C1
:10B8100080E59FE20E94544D0E94DDA00C94714E81
:10B820008CE3809356010C94714E0E942249109132
:10B8300056018AE796E00E940D41812F0E94F82070
:10B840008AE00E94EC400C94714E80E00E941A4104
:10B850000C94714E81E00E941A410C94714E83E564
:10B860000E94C11C882311F40C94714E0E941E2169
:10B87000182F8C3308F08CE3809304060E9465BC7B
:10B880006B017C01212F30E0A8EEB3E00E94C0EDF7
:10B89000C60ED71EE81EF91EC0920006D092010601
:10B8A000E0920206F09203060C94714E80917803A8
:10B8B0008F7D8061809378030C94714E8091780322
:10B8C0008F7E8062809378030C94714E83E50E9492
:10B8D000C11C8823F1F00E9465BC6093FC05709345
:10B8E000FD058093FE059093FF050E945E2120E0F8
:10B8F00030E04AE754E40E94CBE70E9468EF60938F
:10B9000063017093640180936501909366010C94C8
:10B91000714E0E94391C882309F46EC00E941A8D52
:10B920000E94981C082F10918C04182311F40C9479
:10B93000714EF12CE12CC82ED12CAA24A394B12C49
:10B94000C6010E2C02C0959587950A94E2F780FFF8
:10B9500012C08E2D0E94B889882369F0F701EA5D34
:10B96000FD4F808195010E2C01C0220F0A94EAF749
:10B97000822B809518232FEFE21AF20A33E0E316A8
:10B98000F104F1F603FF04C00E94A3898111147F22
:10B99000F12CE12CC12ED12CC6010E2C02C09595A4
:10B9A00087950A94E2F780FF0FC0F701E358FE4F36
:10B9B00080810E94EC40F701EA5DFD4F908180910B
:10B9C0008C0489230E94E5DB8FEFE81AF80A93E0E4
:10B9D000E916F10409F713FD02C00C94714E85E4D9
:10B9E0000E94EC4080E30E94EC4080918C048370C4
:10B9F0000E94E5DB0C94714E0E942A8D0C94714ECE
:10BA000083E50E944A1C882311F40C94714E0E9415
:10BA100065BC6093FC057093FD058093FE059093D3
:10BA2000FF050E945E2120E030E04AE754E40E94D6
:10BA3000CBE70E9468EF6093F8057093F905809357
:10BA4000FA059093FB050C94714EFDE7CF2EF1E0C3
:10BA5000DF2EA9EEEA2EABE0FA2E10E0D6018D9192
:10BA60006D010E94C11C882349F0133089F00E94A7
:10BA70005E21F701648B758B868B978B1F5FF4E0DB
:10BA8000EF0EF11C143051F70E94F68C0C94714E9D
:10BA90000E945E214B015C0120E030E040EA51E46D
:10BAA0000E9466E787FF3AC0A50194016091090CE6
:10BAB00070910A0C80910B0C90910C0C0E94FBEE83
:10BAC0002B013C01AC019B016091190C70911A0C87
:10BAD00080911B0C90911C0C0E94CBE76093190C79
:10BAE00070931A0C80931B0C90931C0C60911B0696
:10BAF00070911C0680911D0690911E060E946AE7B7
:10BB0000A30192010E94CBE70E9468EF60931B069D
:10BB100070931C0680931D0690931E068092090C5C
:10BB200090920A0CA0920B0CB0920C0CA7CF0E9422
:10BB3000EFB382ED91E10E94E9880C94714E8091FF
:10BB4000970390919803009709F4B6CBDC012C91F0
:10BB5000222309F4B1CB0E9454B40C94714E00918D
:10BB600097031091980394E0F12C40E09150F9F084
:10BB7000F8018081282F2B7F213499F421812133F2
:10BB8000B1F4813411F1853409F441E098012E5F5C
:10BB90003F4F89012F5F3F4FF80180818032C9F309
:10BBA000E5CF803521F4818180538A3078F34111CB
:10BBB0000E942249FF2021F084E199E00E940D417A
:10BBC000C8010E94FE400C94714EFF24F394DECF16
:10BBD0000E94F4A40C94714E81E080934A058093F6
:10BBE00049050E940FA50C94714E10924A051092BF
:10BBF00049050E940FA50C94714E8C01112788E411
:10BC00000E94C11C8823C1F00E944F218A3A9105ED
:10BC10000CF44BC00E944F21863F91050CF048C0A8
:10BC20000E944F2126E0209FF001219FF00D11245A
:10BC3000E955FA4F9183808382E40E94C11C8823D6
:10BC4000A9F00E944F210597B4F10E944F2184373B
:10BC50009105A4F50E944F2126E0209FF001219F2D
:10BC6000F00D1124E955FA4F9383828386E40E94F4
:10BC7000C11C882311F40C94714E0E944F2197FD32
:10BC800020C00E944F218F3F910509F0ECF40E94E3
:10BC90004F2126E0209FF001219FF00D1124E9554E
:10BCA000FA4F958384830C94714E8AEA90E0BACF60
:10BCB00085EF90E0B7CF85E090E0CECF83E790E0CE
:10BCC000CBCF90E080E0E5CF8FEF90E0E2CF8091A6
:10BCD000930384FD0DC080919503887849F4809189
:10BCE0009603837029F481E00E946F480C94714E92
:10BCF0000E94604987FF02C00C94714E0DE711E06D
:10BD000079EEE72E7BE0F72EE1E8CE2EE1E0DE2EA5
:10BD1000D8018D918D010E94C11C882359F00E9489
:10BD20005E210E9468EFF7016083718382839383B1
:10BD30000E94B28CF4E0EF0EF11CC016D10641F760
:10BD40000C94714E0E94604987FF02C00C94714EA2
:10BD50006DE7E62E61E0F62E10E000E0D7018D9150
:10BD60007D010E94C11C882349F00E945E21F801D8
:10BD7000E751F44F64A375A386A397A30C5F1F4FED
:10BD80000031110559F70C94714E8091940387FD91
:10BD900009C0809195038E7029F481E00E942848A3
:10BDA0000C94714E83E50E94C11C882391F00E947F
:10BDB0005E2160931D0C70931E0C80931F0C90935A
:10BDC000200C6093250C7093260C8093270C909385
:10BDD000280C80E50E94C11C882351F00E945E213E
:10BDE00060931D0C70931E0C80931F0C9093200C7D
:10BDF00082E50E94C11C882351F00E945E2160935D
:10BE0000210C7093220C8093230C9093240C84E5D6
:10BE10000E94C11C882311F40C94714E0E945E2173
:10BE20006093250C7093260C8093270C9093280C1C
:10BE30000C94714E82E40E94C11C882351F00E9430
:10BE4000FE206093F90B7093FA0B8093FB0B909399
:10BE5000FC0B83E50E94C11C882351F00E945E21E7
:10BE60006093290C70932A0C80932B0C90932C0CCC
:10BE700084E50E94C11C882351F00E945E216093DA
:10BE80002D0C70932E0C80932F0C9093300C8AE421
:10BE90000E94C11C882311F40C94714E0E945E21F3
:10BEA0006B017C012AE037ED43E25CE30E94E7EF9F
:10BEB00087FD14C02AE939E949E95EE3C701B60103
:10BEC0000E9466E7181654F0C0920B06D0920C063A
:10BED000E0920D06F0920E060C94714E0E941E49DF
:10BEE00089E399E00E940D410C94714E83E50E9414
:10BEF0004A1C882331F00E942F21809327010C9443
:10BF0000714E6AE779E081E00E9403B71091270142
:10BF1000105D81E799E00E940D41812F0E94EC4065
:10BF20008DE699E00E940D41809127010E941249FF
:10BF30008091290190912A01A0912B01B0912C01AF
:10BF400088A399A3AAA3BBA340902D0150902E01D2
:10BF500060902F01709030018090310190903201FB
:10BF6000A0903301B0903401C0903501D0903601DB
:10BF7000E0903701F09038018091390190913A01B9
:10BF8000A0913B01B0913C018CA39DA3AEA3BFA3A4
:10BF900080913D0190913E01A0913F01B0914001FF
:10BFA00089A79AA7ABA7BCA785E699E00E940D4197
:10BFB00048A159A16AA17BA188E599E00E94EA42C3
:10BFC000B301A2018AEA9EE20E94EA42B501A401FD
:10BFD00087EA9EE20E94EA4283E699E00E940D41D0
:10BFE0008BE599E00E940D41B701A60188E599E033
:10BFF0000E94EA424CA15DA16EA17FA18AEA9EE265
:10C000000E94EA4249A55AA56BA57CA587EA9EE253
:10C010000E94EA428AE00E94EC400C94714E82E455
:10C020000E944A1C882341F08091210190912201B5
:10C0300090930B0180930A0182E50E944A1C882399
:10C0400041F080910A0190910B019093220180931D
:10C05000210183E50E94C11C882331F00E944F21F9
:10C0600090932201809321018091930390919403F6
:10C07000A0919503B0919603892B8A2B8B2B11F0FD
:10C080000C94714E609121017091220188E899E031
:10C090000E94464D85E20E94EC408AE00E94EC40FE
:10C0A0000C94714E0E94224985E40E94EC4080E38A
:10C0B000800F0E94EC40F701EF5BFE4F60817181C1
:10C0C0008CE899E00E94464D85E20E94EC408AE0AF
:10C0D0000E94EC400C94714E8AE50E94C11C88239A
:10C0E000F1F00E945E2120E030E040E050EC0E9440
:10C0F000E7EF87FF31C060E070E080E090EC2091D6
:10C10000050C3091060C4091070C5091080C0E94D0
:10C11000CBE70E9463EFCB010E945BB705C083E5CC
:10C120000E94C11C8111DDCF8091950387FD26C03F
:10C1300080919603837011F50E94224940918704F3
:10C14000509188046091890470918A0484E999E08F
:10C150000E94FB420C94714E0E945E2120E030E070
:10C1600040E050E40E9466E718161CF00E945E2131
:10C17000C6CF60E070E080E090E4C1CF82E50E942D
:10C180004A1C8111D9CF0C94714E88EE93E00C9427
:10C190002C578091930383FD09C08091940381788B
:10C1A00029F481E00E942A490C94714E80E50E9496
:10C1B000C11C882351F00E945E2160935C11709332
:10C1C0005D1180935E1190935F1189E40E94C11C00
:10C1D000882381F00E945E212CEA35EC47E25EE381
:10C1E0000E94CBE76093601170936111809362119C
:10C1F0009093631184E40E94C11C882311F40C9471
:10C20000714E0E945E2120E030E543EC50E40E9434
:10C21000CBE76093641170936511809366119093DE
:10C2200067110C94714E80E50E944A1C882351F0DE
:10C230000E945E2160939B0570939C0580939D05F1
:10C2400090939E0589E40E944A1C882381F00E94F5
:10C250005E212CEA35EC47E25EE30E94CBE7609377
:10C260009F057093A0058093A1059093A20584E497
:10C270000E944A1C882311F40C94714E0E945E2186
:10C2800020E030E543EC50E40E94CBE76093A30547
:10C290007093A4058093A5059093A6050C94714E08
:10C2A00083E50E944A1C182F882369F00E944F21C1
:10C2B0009C0190936C0180936B0191E0232B09F01A
:10C2C00090E09093431180E50E944A1C882361F01E
:10C2D00020916B0130916C01232B11F00E942F21D2
:10C2E000809343110C94714E11110C94714E0E9465
:10C2F00022498DEB99E00E940D41809143118823E2
:10C3000091F085EA99E00E940D4160916B01709176
:10C310006C018CEA99E00E94464D88EA99E00E94FF
:10C320000D410C94714E81EA99E0EDCF0E94FE42DE
:10C330000C94714E0E941A8D0C94714E88E50E94E7
:10C340004A1CC82E89E40E944A1CA82E8823A1F109
:10C350000E944F21182F89E50E944A1CF82E8AE47A
:10C360000E944A1CE82E882309F43FC00E944F21F6
:10C37000082F8AE50E944A1CD82EB12C811104C0D6
:10C3800081E50E944A1CB82EA11001C0E12C8E2D1F
:10C3900090E0C11001C0F12C8F0D911D019721F487
:10C3A000D1103CC0B1103AC00E941E4989EE99E0FC
:10C3B0000E940D410C94714EC11002C01FEFCBCFF3
:10C3C0000E945E2120E030E040E252E40E9484EED0
:10C3D0002AE037ED43E25CE30E94CBE70E9463EF83
:10C3E000162F633008F4B7CFE9CFF11002C00FEF7A
:10C3F000C0CF0E945E2120E030E040E252E40E9483
:10C4000084EE2AE037ED43E25CE30E94CBE70E9432
:10C4100063EF062F633008F4ACCFE9CF17FD02C0FD
:10C4200007FF08C00E941E4980ED99E00E940D415F
:10C430000C94714E0E945E21E12E110FFF08E02F37
:10C44000000FFF0B8701000F111F20E030E0A90152
:10C45000BB2079F0D801AE0DBF1DAE0FBF1FAA0FD4
:10C46000BB1FAA0FBB1FAD59BB4F2D913D914D91E5
:10C470005C910E0D1F1D0E0F1F1F000F111F000FCF
:10C48000111F0D591B4F0E9484EEF80160837183C8
:10C49000828393830C94714E0E940AA60C94714E71
:10C4A0000E941AA50C94714E01E00C943058209310
:10C4B0008B040E94BBA110928B04882311F40C946E
:10C4C000714E0E94224981EC9AE00E940D410C9429
:10C4D000714E14FD02C00C94714E0E94CFDB0C947F
:10C4E000714E83E080930A0610923B0F60E083E573
:10C4F0000E943E2181110C94714E0E9450B60C9402
:10C50000714E0091990310919A030E9465BC60934B
:10C51000FC057093FD058093FE059093FF050023B5
:10C5200011F40C94714E0E94224984E50E94EC4063
:10C53000802F0E94F82080E20E94EC408CEE9AE06E
:10C540000E940D410C94714E83E50E94C11C88230A
:10C5500009F4EDC80E940E218B01E9C8F1100C947A
:10C560009E4E90E1EDE6F1E0A5E4B4E001900D927D
:10C570009A95E1F70C94AC4EB0E0A0E0E2ECF2E664
:10C580000C944EEE7C014DB65EB66090F605709050
:10C59000F7058DB69EB66AE070E0C7010E94A3E67B
:10C5A0006C018C010E191F09892B21F4C7010E940F
:10C5B000B5E68C01C80101962DB73EB7281B390B93
:10C5C0000FB6F8943EBF0FBE2DBF8DB79EB7019634
:10C5D0005C01A801B7010E94D6E6F501E00FF11F4A
:10C5E0001082C5010E94122B81E00E94434EC114AB
:10C5F000D10451F076019FEFE91AF90A0FB6F894C9
:10C600009EBE0FBE8DBEC5CF0FB6F8949EBE0FBEA8
:10C610008DBEC3010E94122B0FB6F8945EBE0FBEF2
:10C620004DBEE0E10C946AEECF93DF93C0911D0DF7
:10C6300081E6C89FE0011124C15ED24F8091E80BD2
:10C6400080FF05C00E942249CE010E94FE40CE011B
:10C650000E94122B80E00E94434EDF91CF910895FB
:10C66000A0E1B0E0E6E3F3E60C945AEE8C01DC01C5
:10C67000ED91FC910280F381E02DBE016F5F7F4F51
:10C680000995882309F45DC08981807C91F56F81CB
:10C69000637070E0762F6627770F770F8885B4E098
:10C6A0008B9FC0011124682B792B898582958695F3
:10C6B00086958370682B6F5F7F4F90E080E02A85BE
:10C6C0002370220F3B8537FB332730F9232B3E8124
:10C6D0003F70230F3327331F2750310904C0660FE3
:10C6E000771F881F991F2A95D2F76096E4E00C9473
:10C6F00076EE803419F568856695669570E090E071
:10C7000080E0CB01772766272A85622B098510E018
:10C71000102F0027012E000C220B330B602B712BE6
:10C72000822B932B6F5F7F4F8F4F9F4F4AE0660F97
:10C73000771F881F991F4A95D1F7D7CF8BE0F80153
:10C74000848360E070E0CB01D0CF0895FC0182814A
:10C7500008954F925F926F927F928F929F92AF92C5
:10C76000BF92CF92DF92EF92FF92CF93DF93CDB73C
:10C77000DEB728970FB6F894DEBF0FBECDBF60912D
:10C780009805709199056115710511F180919405D5
:10C7900090919505A0919605B091970589839A830C
:10C7A000AB83BC83072E000C880B990B0E946CE7AF
:10C7B00029813A814B815C810E9483EE4B015C01AF
:10C7C00020E030E040E251EC0E9466E787FF07C0BE
:10C7D00081E080934701C12CD12C760113C020E069
:10C7E00030E040E251E4C501B4010E94E7EF1816C1
:10C7F00004F581E080934701C12CD12C9FE7E92EFD
:10C8000093E4F92EC701B60128960FB6F894DEBF5F
:10C810000FBECDBFDF91CF91FF90EF90DF90CF9013
:10C82000BF90AF909F908F907F906F905F904F9050
:10C83000089580919F059091A005A091A105B091C8
:10C84000A2058D839E83AF83B8878091470188239B
:10C8500091F010923505109236051092370510921E
:10C86000380510923105109232051092330510925E
:10C8700034051092470120913505309136054091DD
:10C88000370550913805C501B4010E9484EE2B0193
:10C890003C0120E030E0A9010E94E7EFC12CD12C3F
:10C8A000760187FD14C02D813E814F81588560E05F
:10C8B00070E08FE793E40E94FBEE6B017C01A30123
:10C8C00092010E9466E7181614F473016201C09287
:10C8D0003505D0923605E0923705F0923805209163
:10C8E0009B0530919C0540919D0550919E05C50189
:10C8F000B4010E94CBE74B015C0180922905909224
:10C900002A05A0922B05B0922C05A70196016D81F6
:10C910007E818F8198850E94CBE76B017C01C0925C
:10C920002D05D0922E05E0922F05F0923005409013
:10C93000310550903205609033057090340529819F
:10C940003A814B815C81609125057091260580912B
:10C950002705909128050E9483EE2091A305309130
:10C96000A4054091A5055091A6050E94CBE7A3011F
:10C9700092010E9483EE20ED3CEC4CE45DE30E94CA
:10C98000CBE7A30192010E9484EE9B01AC012093AE
:10C990003105309332054093330550933405898136
:10C9A0009A81AB81BC818093250590932605A09345
:10C9B0002705B0932805C501B4010E9484EEA701A4
:10C9C00096010E9484EE6B017C0120E030E04FE78D
:10C9D00053E40E9466E7181634F4C12CD12C8FE77B
:10C9E000E82E83E4F82E20E030E0A901C701B6016B
:10C9F0000E94E7EF87FF06CFEECE6091940570911D
:10CA0000950580919605909197050895FC0190E118
:10CA1000A4E1B5E001900D929A95E1F70895EF92A7
:10CA2000FF920F931F93E0928D04F0928E04009377
:10CA30008F0410939004B62F172F022FF32E242F5C
:10CA4000582FB093910410939204509393046FEF76
:10CA5000FF27B01B1F09520B30F450951095B1956C
:10CA6000160B560B662760936C02A6E0BA9F0092E5
:10CA70006002712DEE271A9F700DE11D5A9FE00D87
:10CA800070936102E0936202AFE0BA9F0092640289
:10CA9000712DEE271A9F700DE11D5A9FE00D7093C6
:10CAA0006502E0936602AAE0BA9F00926802712DC7
:10CAB000EE271A9F700DE11D5A9FE00D70936902D9
:10CAC000E0936A021F910F91FF90EF900895A5E007
:10CAD000B0E0EDE6F5E60C9453EE6F367105810596
:10CAE000910578F4FB01EE0FFF1FEE0FFF1FEA5BCD
:10CAF000F44E65917591859194912596EBE00C9497
:10CB00006FEEF62EE72E282FE6E4FAE10027BB278A
:10CB10005F2D8E2D922F992341F4982F852FB85F8A
:10CB2000992319F4982F8827B85F903138F48295AB
:10CB30009295582F5F70807F952BBC5F903428F4BE
:10CB4000880F991F880F991FBE5F903818F4880FBF
:10CB5000991FB395880F991FE90FF01F549181E039
:10CB60009927B85079F1C0F0B0FF02C0550F881F67
:10CB7000B1FF04C0550F881F550F881FB2FF06C0B4
:10CB800082955295152F1F70507F812BB3FF1AC0CD
:10CB9000982F852F552716C0B195B0FF02C08595F7
:10CBA0005795B1FF04C08595579585955795B2FF68
:10CBB00005C08295507F5295582B8F70B3FF02C0ED
:10CBC000582F8827BB247727AA27B2E0F59EB018F4
:10CBD0007109A00BB00BE59E7019A109B00B259F40
:10CBE000A019B109F89E7019A109B00BE89EA0190F
:10CBF000B109289FB019F99EA019B109E99EB01991
:10CC00005B9DA12C99244427662733278B9DA00C7C
:10CC1000911C401F601F301F9B9D900C411D601F89
:10CC2000301F579FA00C911C401F601F301F879F13
:10CC3000900C411D601F301F979F400D611D301FDC
:10CC40005A9F900C411D601F301F8A9F400D611D2F
:10CC5000301F9A9F600D311D5B9F400D611D301F7D
:10CC60008B9F600D311D9B9F300DB1E0AA27772768
:10CC7000BB24F49EB0187109A00BB00BE49E701990
:10CC8000A109B00B249FA019B109F69E7019A10942
:10CC9000B00BE69EA019B109269FB019F39EA0190A
:10CCA000B109E39EB019BF187E09A20B20F0B1E0D4
:10CCB0004B0F601F301F1124762F642F90E0832FBD
:10CCC0001CCFA2E1B0E0E7E6F6E60C944CEE788BE0
:10CCD0006F87DC018D909D90AD90BC90139714965A
:10CCE0002D913D914D915C9117972D833E834F83FC
:10CCF000588720E030E040E251E4C501B4010E94D1
:10CD000083EE2AE037ED43E25CE30E94CBE70E942A
:10CD100063EF16160CF010C161E0E62E660FFF08F7
:10CD2000F701EE0FFF1FEE0FFF1FEE5BFD4E408081
:10CD300051806280738087010F5F1F4F20E030E0D9
:10CD400040E251E46D817E818F8198850E9483EE5F
:10CD50002AE037ED43E25CE30E94CBE70E9463EFF9
:10CD6000698316160CF0ECC0E1E0E9832981022EFC
:10CD7000000C330B3A8B298BF901EE0FFF1FEE0FDE
:10CD8000FF1FEE5BFD4E80819181A281B38189837B
:10CD90009A83AB83BC8319019FEF291A390AB70123
:10CDA000660F771FDB01AE0DBF1DBA87A987FD0196
:10CDB000E20FF31FEE0FFF1FEE0FFF1FED59FB4FAA
:10CDC000C080D180E280F380F801EE0FFF1FEE0FEC
:10CDD000FF1FEE5BFD4EA301920160817181828194
:10CDE00093810E9483EE6B877C878D879E87A3014A
:10CDF0009201C501B4010E9483EE2B013C01C801E0
:10CE0000880F991F080F191FE989FA89E00FF11F90
:10CE1000EE0FFF1FEE0FFF1FED59FB4FA70196010D
:10CE200060817181828193810E9483EE2B853C8594
:10CE30004D855E850E94FBEEA30192010E94CBE727
:10CE4000A70196010E9484EE6B017C01E985FA85B9
:10CE5000E20DF31DEE0FFF1FEE0FFF1FED59FB4F0D
:10CE600080809180A280B380020D131DF801EE0F27
:10CE7000FF1FEE0FFF1FED59FB4FA50194016081CD
:10CE80007181828193810E9483EE2B853C854D8543
:10CE90005E850E94FBEEA30192010E94CBE7A501F3
:10CEA00094010E9484EEA70196010E9483EE4B013B
:10CEB0005C01F101EE0FFF1FEE0FFF1FEE5BFD4E59
:10CEC00029813A814B815C8160817181828193816A
:10CED0000E9483EE9B01AC01C501B4010E94FBEEF0
:10CEE0004B015C0129813A814B815C816D817E819E
:10CEF0008F8198850E9483EE9B01AC01C501B4012E
:10CF00000E94CBE7A70196010E9484EEAF85B88905
:10CF10002D913D914D915C910E94CBE7209187042A
:10CF2000309188044091890450918A040E9484EED3
:10CF30006296E2E10C9468EE67FFEFCE60E0EDCE22
:10CF4000F981F7FF13CF198211CF8F929F92AF9281
:10CF5000BF92CF92DF92EF92FF92CF93DF93EC01DB
:10CF600080905F0490906004A0906104B09062048F
:10CF700020E030E0A901C501B4010E9466E78823E2
:10CF800009F454C0C880D980EA80FB80A7019601CB
:10CF9000C501B4010E9466E718160CF04CC0209140
:10CFA0005A0430915B0440915C0450915D04C701C8
:10CFB000B6010E9466E7882331F1C0925A04D092EC
:10CFC0005B04E0925C04F0925D0420915604309181
:10CFD00057044091580450915904688179818A819D
:10CFE0009B810E94CBE79B01AC0160E070E080E890
:10CFF0009FE30E9483EE609323017093240180934A
:10D000002501909326016091230170912401809164
:10D01000250190912601DF91CF91FF90EF90DF9055
:10D02000CF90BF90AF909F908F90089560E070E098
:10D0300080E89FE3F0CF60E070E0CB01ECCFFC0133
:10D040007081472F50E0062E02C0559547950A94EF
:10D05000E2F740FF14C04091550450E0062E02C094
:10D06000559547950A94E2F740FF09C021E030E06A
:10D0700001C0220F6A95EAF720952723208308959F
:10D08000282F81E3243609F080E28093400490E267
:10D090002A3040F03AE0822F632F0E94CFED0E94A9
:10D0A000CFED905D90934104822F6AE00E94CFED16
:10D0B000905D9093420485E28093430480E494E081
:10D0C00008956091410170914201072E000C880B78
:10D0D000990B0E946CE72AE037ED43E25CE30E9483
:10D0E000CBE7609367017093680180936901909327
:10D0F0006A010895CF93DF93EC01CB01BA010E943E
:10D100006CE723E333E343E250E40E94CBE720E003
:10D1100030E040E05FE30E9484EE0E9468EF6883A5
:10D12000DF91CF9108950E946CE723E333E343E25C
:10D1300050E40E94CBE720E030E040E05FE30E9453
:10D1400084EE0E9468EF24E6629FC001112481589A
:10D150009F4F6FEF70E00E94FCED862F91CF809182
:10D16000D905811104C08091390480932706089560
:10D1700080915C138823C1F0815080935C13E0EAB6
:10D18000F1E1882351F08150990B2BE1289FF001A8
:10D19000299FF00D1124E25BFD4E8BE1A5E8B1E182
:10D1A00001900D928A95E1F720915C13211105C041
:10D1B0008091651380648093651381E090E0A0E026
:10D1C000B0E0211103C080E090E0DC018093C00555
:10D1D0009093C105A093C205B093C3051092BA0500
:10D1E00081E08093D00583E0809357010895CF9329
:10D1F000DF93EC01CB01BA010E946CE7688379836D
:10D200008A839B83DF91CF910895CF93DF93EC01C5
:10D21000CB01BA010E946CE72FE632E143E85AE302
:10D220000E94CBE7688379838A839B83DF91CF91C8
:10D230000895CF93DF93EC01CB01BA010E946CE714
:10D240000E9468EF6883DF91CF910895CF93DF93B9
:10D25000EC018D810E94324E60E08B810E947DBB8B
:10D26000DF91CF910895CF92DF92EF92FF920F93CB
:10D270001F93CF938C01C62F69017A01E7DF0E94CB
:10D28000F9BC8C2F80640E94264E8F2D0E94264E62
:10D290008E2D0E94264E8D2D0E94264E8C2D0E9492
:10D2A000264E87E8C11101C085E90E94264ECC3088
:10D2B00011F40E942B4EC0E00E942B4EF801868391
:10D2C00087FF04C0CF3F11F0CF5FF6CFCF911F9102
:10D2D0000F91FF90EF90DF90CF90089561E0FC01F7
:10D2E00083810E947DBB8FEF0C94264E0F931F937A
:10D2F000CF938C01ABDF0E94F9BCC82F882369F063
:10D300008DEF0E94264E0E94F9BCC82FC801E6DFAF
:10D310008C2FCF911F910F91089582E1F8018483A2
:10D32000F5CFB0E0A0E0E7E9F9E60C9452EEEC01AD
:10D330006A017B014801590120E030E0A90167E35F
:10D3400092DFA501980167E1CE018DDF81111DC03B
:10D350008F81833039F089E0CC0CDD1CEE1CFF1C82
:10D360008A95D1F7A701960169E1CE017CDF11E032
:10D37000882319F010E087E08C83CE01AFDF812F86
:10D38000CDB7DEB7ECE00C946EEE89E08C8310E054
:10D39000F4CFCF93DF93EC016EBDFA01CA019E5F1B
:10D3A0000DB407FEFDCF20812EBD0DB407FEFDCFCD
:10D3B00021812EBD3296E817F90791F70DB407FECB
:10D3C000FDCF8FEF0E94264E8FEF0E94264E0E94C7
:10D3D0002B4E8E838F71853041F083E18C83CE019B
:10D3E0007DDF80E0DF91CF91089581E0FBCF0F9347
:10D3F0001F93CF93DF93EC018B0128DF0E94F9BCD0
:10D4000081110BC085E18C8310E0CE0167DF812F95
:10D41000DF91CF911F910F910895A8016CEFCE017C
:10D42000B8DF182F882371F3F0CF0F931F93CF939A
:10D43000DF93EC0189018F81833039F089E0440F5B
:10D44000551F661F771F8A95D1F79A01AB0168E1D6
:10D45000CE0109DF811127C0A8016EEFCE0199DF4F
:10D46000182F8823A9F00E94F9BC182F8823C1F037
:10D4700020E030E0A9016DE0CE01F5DE882321F047
:10D4800086E18C8310E004C00E942B4E8111F8CFFE
:10D49000CE0124DF812FDF91CF911F910F9108954D
:10D4A00087E18C83F5CF86E0ECCF1F93CF93DF939A
:10D4B000EC01CCDE20E030E0A9016CE0CE01D3DE4F
:10D4C00011E0882319F010E083E08C83CE0106DFA1
:10D4D000812FDF91CF911F9108951F93CF93DF93F9
:10D4E000EC018F81833039F089E0440F551F661FAE
:10D4F000771F8A95D1F79A01AB0162E1CE01B3DEC5
:10D5000011E0882319F010E085E08C83CE01E6DE7F
:10D51000812FDF91CF911F9108958F929F92AF92AB
:10D52000BF92EF92FF920F931F93CF93DF938C01E3
:10D53000EB017A010E9465BC4B015C012CE2820E7A
:10D5400021E0921EA11CB11C0E942B4EF801868383
:10D550008F3F69F40E9465BC681979098A099B09A3
:10D5600097FDF2CF81E1F8018483C0E021C08E3FB6
:10D5700069F5F1E0EF1AF1088FEF8EBDFE012FEF94
:10D580000DB407FEFDCF8EB581932EBDCF018C1B50
:10D590009D0B8E159F05A0F30DB407FEFDCF8EB534
:10D5A000CE0DDF1D88830E942B4E0E942B4EC1E0C2
:10D5B000C80194DE8C2FDF91CF911F910F91FF90C6
:10D5C000EF90BF90AF909F908F9008958FE0CBCF5A
:10D5D0000F931F93CF93DF93EC018B0137DE40E075
:10D5E00052E0B801CE0199DFDF91CF911F910F91E9
:10D5F00008950F931F93CF93DF93EC0189018F81DF
:10D60000833039F089E0440F551F661F771F8A95D4
:10D61000D1F79A01AB0161E1CE0125DE882351F0FB
:10D6200084E08C83CE015ADE80E0DF91CF911F91A0
:10D630000F91089540E052E0B801CE016EDFF5CFC2
:10D64000B0E0A0E0E6E2FBE60C9452EEEC01162F0F
:10D650001F821C824B830E9465BC6B017C0120ED04
:10D66000C20E27E0D21EE11CF11CA89561E08B815F
:10D670000E947DBB8B810E9463B3249A2C9A279AC7
:10D680002698259A81E00E94324E85E08D830E9483
:10D69000324E0AE08FEF0E94264E0150D9F7A8952E
:10D6A00020E030E0A90160E0CE01DDDD8E83813035
:10D6B00079F00E9465BC6C197D098E099F0997FD60
:10D6C000EFCF81E08C83CE0109DE1A8280E065C055
:10D6D000A8952AEA31E040E050E068E0CE01C3DDE1
:10D6E000853031F581E08F83A8958F81812C912C35
:10D6F0005401823029F4812C912CA12C80E4B82E85
:10D7000020E030E0A90167E3CE01ADDDA501940181
:10D7100069E2CE01A8DD8E838823F1F00E9465BC0A
:10D720006C197D098E099F0997FDEACF8AE0CACF5F
:10D7300004E00E942B4E8E830150D9F78A3A11F4EF
:10D7400082E0D1CF0E9465BC6C197D098E099F09CA
:10D7500097FDBFCF82E0B6CF8F818230B9F420E051
:10D7600030E0A9016AE3CE017EDD882311F088E074
:10D77000A9CF0E942B4E807C803C11F483E08F83E4
:10D780000E942B4E0E942B4E0E942B4ECE01A6DDF6
:10D7900081E08A83173030F41D83CDB7DEB7ECE02B
:10D7A0000C946EEE88E18C8391CF0F931F93CF93EF
:10D7B000DF93EC018B0120E030E0A90169E053DD4B
:10D7C000882351F080E18C83CE0188DD80E0DF91F9
:10D7D000CF911F910F91089540E150E0B801CE0123
:10D7E0009CDEF5CFCF93C82FCB010E940D4184E979
:10D7F00099E10E940D4185E899E1CC2311F08AE876
:10D8000099E10E940D418AE00E94EC40CF91089579
:10D81000EF92FF920F931F93CF937B018A01C2E493
:10D820008F3F09F0C4E580E20E94EC408C2F0E94FB
:10D83000EC408AE30E94EC40F701608171818281B3
:10D84000938142E00E9482B38BE296E20E940D41F6
:10D85000F801608171818281938142E00E9482B3EC
:10D8600062E070E080E090E00E94D9BBCF911F9110
:10D870000F91FF90EF9008950C9471BC40918B0430
:10D8800021E042276CE070E00C9437B340918B04A8
:10D8900021E0422764E070E00C9437B340918B04A0
:10D8A00021E0422761E070E00C9437B340918B0493
:10D8B00021E0422761E070E00C9437B340918B0483
:10D8C00021E0422768E070E00C9437B340918B046C
:10D8D00021E042276CE070E00C9437B341E061E056
:10D8E00070E00C9437B340918B0421E042270C94F4
:10D8F00037B36CE070E00C940CBC61E070E00C9409
:10D900000CBC6CE070E00C940CBC64E070E00C9417
:10D910000CBC61E089E394E00C949E2CA4E0B0E0A0
:10D92000E4E9FCE60C945CEE0E946CE72FE632E141
:10D9300043E85AE30E94CBE769837A838B839C8315
:10D94000CE0101960E9486212496E2E00C9478EEA6
:10D95000B0E0A0E0EEEAFCE60C9451EE61E081E07C
:10D960000E949C23C091BA05EC2E85E0982E9C0E57
:10D970009EEAC92E98E1D92ED7E0DC1BBB24B394D4
:10D9800016E01C1B22E0A22E05E00C1B84E0F82E02
:10D99000FC1A8A2C8C1A7B2C7C1AC1112CC0809109
:10D9A000B9058823B9F080915701882361F06E2D65
:10D9B000619581E09091B905911180E024E043EEFA
:10D9C00058E10E947AB7CF5FC911E7CF88E0809312
:10D9D000B3050CC08091B4051092B405882319F3E7
:10D9E0000E94C22F8091D0058823E9F2CDB7DEB71F
:10D9F000EDE00C946DEEC13011F58091B9058130E8
:10DA000079F0809157018823F1F281E09091B90576
:10DA1000913009F080E023E049E35EE2672DD1CF49
:10DA20008091B4051092B405882359F387E09EE6EF
:10DA30000E94A9B88091D005882319F3D7CFC230AE
:10DA400009F0C5C09091B905923071F080915701ED
:10DA5000882309F4B8CF81E0923009F080E020E219
:10DA600045ED58E1682DADCF8091B4051092B40515
:10DA7000882361F32FED38E130934E0520934D0557
:10DA80008091D005882311F3B1CF1092D9059091E0
:10DA9000B905933079F080915701882309F493CF29
:10DAA00063E06E1981E0933009F080E020E249ECF8
:10DAB00058E187CF8091B4051092B405882359F3BB
:10DAC00020ED38E130934E0520934D058091D0052F
:10DAD000882309F38BCFB092D9059091B905943082
:10DAE00071F080915701882309F46DCF81E0943063
:10DAF00009F080E020E249EC58E16F2D62CF80917F
:10DB0000B4051092B405882361F324EC38E1309316
:10DB10004E0520934D058091D005882311F366CFE3
:10DB2000A092D9059091B905953071F08091570177
:10DB3000882309F448CF81E0953009F080E020E2A5
:10DB400049EC58E1602F3DCF8091B4051092B405A7
:10DB5000882361F32FEB38E130934E0520934D0578
:10DB60008091D005882311F341CF8091B90586308B
:10DB700081F080915701882309F425CF81E09091AD
:10DB8000B905963009F080E023E042EB58E1612FBF
:10DB900018CF8091B4051092B405882351F38EE913
:10DBA00094E70E94A9B88091D005882311F31ECF75
:10DBB0008091B4051092B4058823D9F0D0924E0517
:10DBC000C0924D058091D005882399F00FCFC330C6
:10DBD00009F45BCFC43009F47ECFC53009F4A0CF7F
:10DBE000C63019F2C73009F0EECE9091B9059730E2
:10DBF000F9F280915701882309F4E5CE81E097304E
:10DC000009F080E020E24DE958E16D2FDACEB0E076
:10DC1000A0E0EDE0FEE60C9457EE61E081E00E94AA
:10DC20009C23C091BA0585E0E82EEC0ED4E0DC1B05
:10DC300013E01C1B02E00C1B81E0F82EFC1ADC2E0A
:10DC4000D194C1112BC08091B9058823B1F0809186
:10DC50005701882359F081E09091B905911180E036
:10DC600024E046E958E16D2D0E947AB7CF5FEC12AF
:10DC7000E8CF85E08093B3050CC08091B405109285
:10DC8000B405882321F30E94C22F8091D0058823F8
:10DC9000F1F2CDB7DEB7E7E00C9473EEC13011F5C9
:10DCA0008091B905813079F0809157018823F1F294
:10DCB00081E09091B905913009F080E023E04FE5D3
:10DCC0005EE26F2DD1CF8091B4051092B405882308
:10DCD00059F38BE197E70E94A9B88091D00588237A
:10DCE00019F3D7CFC23009F055C08091B905823001
:10DCF00081F080915701882309F4B8CF81E0909199
:10DD0000B905923009F080E023E048E55EE2602F3B
:10DD1000ABCF8091B4051092B405882351F386E10E
:10DD200097E70E94A9B88091D005882311F3B1CF5D
:10DD30008091B905833081F080915701882309F4DF
:10DD400095CF81E09091B905933009F080E023E010
:10DD500041E55EE2612F88CF8091B4051092B40551
:10DD6000882351F381E197E70E94A9B88091D005FB
:10DD7000882311F38ECF8091B4051092B4058823C7
:10DD800091F085E192E70E94A9B88091D00588239F
:10DD900051F07FCFC33061F2C43009F067CF80917A
:10DDA000B905843041F380915701882309F45ECF8F
:10DDB00081E09091B905943009F080E023E043E4DC
:10DDC0005EE26D2F51CFEF92FF920F931F93CF938F
:10DDD000DF9361E081E00E949C23C091BA0585E059
:10DDE000F82EFC0ED3E0DC1B12E01C1B01E00C1B28
:10DDF000EC2EE194C1112BC08091B9058823B1F0BC
:10DE000080915701882359F081E09091B9059111D3
:10DE100080E024E04EE757E16E2D0E947AB7CF5F95
:10DE2000FC12E8CF84E08093B3050CC08091B40568
:10DE30001092B405882321F30E94C22F8091D0054F
:10DE40008823F1F2CDB7DEB7E6E00C9474EEC13072
:10DE500011F58091B905813079F0809157018823BF
:10DE6000F1F281E09091B905913009F080E023E072
:10DE700041E757E1602FD1CF8091B4051092B405EE
:10DE8000882359F381EC9BE70E94A9B88091D005C3
:10DE9000882319F3D7CFC23091F58091B90582302C
:10DEA00081F080915701882309F4B9CF81E09091E6
:10DEB000B905923009F080E023E046E657E1612F92
:10DEC000ACCF8091B4051092B405882351F38FE450
:10DED0009CE70E94A9B88091D005882311F3B2CFA6
:10DEE0008091B4051092B405882381F087ED9CE7FA
:10DEF0000E94A9B88091D005882341F0A3CFC330F8
:10DF000009F08DCF8091B905833051F3809157018D
:10DF1000882309F484CF81E09091B905933009F00A
:10DF200080E023E04AE557E16D2F77CFA7E0B0E02E
:10DF3000ECE9FFE60C944CEE61E081E00E949C234A
:10DF40007090BA05272C25E0270D2D8387E08719CF
:10DF50008E8386E087198F8385E0682E671884E0BA
:10DF6000582E571882E0482E471881E0382E37186F
:10DF700071105DC08091B905882309F446C0809175
:10DF80005701882361F0622D619581E09091B90578
:10DF9000911180E024E042E759E10E947AB7809134
:10DFA00027068093390485E0781277C11092D9054D
:10DFB0008091B905853009F435C1809157018823D6
:10DFC000E1F011E08091B905853009F010E0809111
:10DFD000390424E6829FC001112481589F4F6FEFBE
:10DFE00070E00E94FCED862F4BD800E09C0141E5DB
:10DFF00059E1662D812F0E94192A73948D81871112
:10E00000B7CF88E08093B3050EC08091B40510921D
:10E01000B405882309F4B3CF0E94C22F8091D005A4
:10E02000882309F4ACCF2796E2E10C9468EE81E0F6
:10E03000781241C08091B905813031F1809157014A
:10E04000882309F4ACCF11E08091B905813009F043
:10E0500010E06091210170912201072E000C880BC5
:10E06000990B0E946CE769837A838B839C83CE0132
:10E0700001960E94782300E09C014CE659E1632D53
:10E08000812F0E94192A8BCF8091B4051092B4057C
:10E090008823A1F210E000E027EE33E04AE050E0F0
:10E0A00061E271E08CE699E10E94EAB88091D005C6
:10E0B000882321F2B8CF22E0721258C18091B905AD
:10E0C0008230D9F080915701882391F011E080913E
:10E0D000B905823009F010E087E894E00E948621BB
:10E0E00000E09C0146E659E1642D812F0E94192A27
:10E0F000809127068093390480CF8091B4051092D7
:10E10000B4058823F9F220E030E04AE754E4609156
:10E110008704709188048091890490918A040E94F8
:10E12000CBE720E030E04AE754E40E9484EE0E940E
:10E1300068EF912C812C3BEEA32E31E7B32E6B01BF
:10E1400010EDE12E17E0F12E00E010E028E13CEFA9
:10E150004FEF5FEF67E874E086E699E10E945CB8F4
:10E160008091D005882309F4ADCF5DCF8091B905AA
:10E17000833021F180915701882309F4B9CF11E050
:10E180008091B905833009F010E0609159117091C8
:10E190005A11072E000C880B990B0E946CE76983BB
:10E1A0007A838B839C83CE0101960E94782363E05F
:10E1B000621900E09C014FE559E162CF8091B405FE
:10E1C0001092B4058823B1F20E9450B80CE31CE60B
:10E1D00025EF30E050E040E069E571E18FE599E13D
:10E1E0000E94EAB88091D005882321F21CCF80914B
:10E1F000B4051092B405882309F4C4C00E9450B835
:10E200000EEA1DE123E730E050E040E068E975E008
:10E210008BE599E10E94EAB88091D005882309F442
:10E22000B1C001CF8091B4051092B405882309F4E0
:10E23000C4CE0E9450B86091390470E090E080E054
:10E240000E946AE729EC38EC48EC5EE30E94CBE7D9
:10E2500020E030E040E05FE30E9484EE0E9468EF3F
:10E260008FEA882E88E6982E95EEA92E91E7B92E92
:10E270006B0114E6E12EF12C00E010E020E030E02C
:10E28000A90169E374E081E599E10E945CB880919D
:10E29000D005882309F491CEC6CE86E078123EC020
:10E2A0008091B905863019F180915701882309F4CE
:10E2B000A4CE11E08091B905863009F010E060919C
:10E2C000410170914201072E000C880B990B0E94AE
:10E2D0006CE769837A838B839C83CE0101960E94CD
:10E2E000782300E09C014CE459E16F8183CE80915A
:10E2F000B4051092B4058823B9F201E618E627EEBA
:10E3000033E04AE050E061E471E08CE499E10E947E
:10E31000EAB88091D005882339F285CE27E07212C1
:10E320006CCE8091B905873091F080915701882398
:10E3300009F463CE81E09091B905973009F080E04F
:10E3400023E041E459E16E810E947AB756CE809174
:10E35000B4051092B405882341F38DEF91E70E9434
:10E36000A9B88091D005882301F35DCE23E0721611
:10E3700009F4FCCE84E0781212CE8091B905843085
:10E3800009F435CF80915701882309F4B1CE11E00B
:10E390008091B905843009F010E060919805709182
:10E3A0009905072E000C880B990B0E946CE7698376
:10E3B0007A838B839C83CE0101960E94782300E0B0
:10E3C0009C014BE559E1652D5BCE6AE778E683E970
:10E3D00098E60C94A93665E079E68EE89CE60C9404
:10E3E000A93667EF78E68AE894E70C94A93669E1E4
:10E3F00079E689ED9AEA0C94A93620E040E070E0D5
:10E4000060E086EA92E70E94E22D81E08093380482
:10E410001092DF051092DE05089520E040E070E0E4
:10E4200060E080E297E70C94E22D0E9430B48823EC
:10E4300041F020E040E070E060E085E297E70C9476
:10E44000E22DEBCF21E020933804FC018081918103
:10E45000A281B3818093190190931A01A0931B01AB
:10E46000B0931C0120E040E070E060E08091BB05CB
:10E470009091BC050C94E22DA4E0B0E0E2E4F2E758
:10E480000C945CEE8DEC9CECACECBCE389839A8341
:10E49000AB83BC83CE010196D5DF2496E2E00C94D9
:10E4A00078EEA4E0B0E0E7E5F2E70C945CEE8DECEA
:10E4B0009CECACECBDE389839A83AB83BC83CE0137
:10E4C0000196C0DF2496E2E00C9478EEA4E0B0E080
:10E4D000ECE6F2E70C945CEE80E090E0A0E8BFE3AD
:10E4E00089839A83AB83BC83CE010196ABDF2496EC
:10E4F000E2E00C9478EEA4E0B0E0E1E8F2E70C94FE
:10E500005CEE80E090E0A0E2B1E489839A83AB8383
:10E51000BC83CE01019696DF2496E2E00C9478EE5F
:10E5200081E08093380410924B051092550420E04E
:10E5300040E070E060E083EA9DE70E94E22D8FED0D
:10E5400098E190934E0580934D0508958F929F9288
:10E55000AF92BF92CF92DF92EF92FF928091B4057B
:10E560001092B405882359F00E945A37FF90EF901B
:10E57000DF90CF90BF90AF909F908F900895809143
:10E58000C0059091C105A091C205B091C305009747
:10E59000A105B10589F01092C0051092C105109235
:10E5A000C2051092C30521E020935701880F991FDF
:10E5B000880F991F0E945BB7809157018823B1F2A1
:10E5C0006091DE057091DF05072E000C880B990B1A
:10E5D0000E946CE72091300630913106409132065E
:10E5E000509133060E94CBE76B017C0120E030E4C0
:10E5F0004CE156E40E94CBE74B015C0120E030E0A7
:10E60000A901C701B6010E9466E720E030E040EAB8
:10E6100050E487FF04C020E030E040EA50ECC50140
:10E62000B4010E9484EE2DEC3CEC4CEC5DE30E94C6
:10E63000CBE70E9463EF6B017C018BE2F7FE09C020
:10E64000F094E094D094C094C11CD11CE11CF11C46
:10E650008DE280933D04C701B60120E137E240E03E
:10E6600050E00E940FEE8AE0882E912CA12CB12C54
:10E67000CA01B901A50194010E940FEE605D60938B
:10E680003E04C701B60128EE33E040E050E00E94AE
:10E690000FEECA01B901A50194010E940FEE605D61
:10E6A00060933F048EE280934004C701B60124E6E4
:10E6B00030E040E050E00E940FEECA01B901A50130
:10E6C00094010E940FEE605D60934104C701B601A2
:10E6D000A50194010E940FEE6B01CA01B901A501C9
:10E6E00094010E940FEE605D6093420480E3C80EC7
:10E6F000C09243046DE374E081E499E10E94B32980
:10E7000035CF8091390490913A040C94A6BC609165
:10E7100039048FEF0C94B0BC80913904682F0C94AD
:10E72000B0BC6FEF809139040C94B0BCB0E0A0E0B5
:10E73000ECE9F3E70C944EEE0091390461E081E0DE
:10E740000E949C23C091BA0510E0000F111F005FCA
:10E75000164E95E0592E5C0E28EEE22E28E1F22EA0
:10E76000D3E0DC1B31E9C32E33E7D32E46EFA42ED2
:10E7700048E1B42E82E0782E7C1A5DE1852E59E1C5
:10E78000952E81E0682E6C1A4C2E4194C1112BC03D
:10E790008091B9058823B1F080915701882359F001
:10E7A00081E09091B905911180E024E044E059E1C5
:10E7B000642D0E947AB7CF5FC511E8CF84E08093C3
:10E7C000B3050CC08091B4051092B405882321F3E1
:10E7D0000E94C22F8091D0058823F1F2CDB7DEB719
:10E7E000E0E10C946AEEC13059F5F80185919491FD
:10E7F0009093DB058093DA058091B905813081F033
:10E80000809157018823B9F21F929F928F926F9245
:10E8100081E09091B905913009F473C080E071C036
:10E820008091B4051092B405882351F38091390486
:10E83000682F0E94B0BC8091D005882309F3CECF09
:10E84000C23009F041C0F801859194919093DB05A5
:10E850008093DA058091B9058230D1F0809157011B
:10E86000882309F4A8CFDF92CF92BF92AF927F9214
:10E8700081E09091B905923009F080E08F930E9479
:10E88000FD210F900F900F900F900F900F9093CF4E
:10E890008091B4051092B405882301F342DF809182
:10E8A000D0058823D9F29ACF8091B4051092B4058F
:10E8B0008823C1F0609139048FEF0E94B0BC809131
:10E8C000D005882379F08ACFC33009F074CFF801DE
:10E8D000859194919093DB058093DA058091B90539
:10E8E000833011F380915701882309F464CF1F927C
:10E8F000FF92EF92DF9381E09091B905933009F098
:10E900008DCF8F930E94FD210F900F900F900F904D
:10E910000F9051CFA4E0B0E0E0E9F4E70C945CEE96
:10E920000E946CE769837A838B839C83CE01019676
:10E930000E94BF212496E2E00C9478EEA8E0B0E0BB
:10E94000E4EAF4E70C944CEE80914B0587708983E0
:10E950000E946B2D682E61E081E00E949C23209133
:10E96000BA052F83722E2B5F2A8383E087198B834E
:10E9700082E087198C8381E087198D83972D91958B
:10E980009E835BEE452E5DE1552E64EE262E6DE1F5
:10E99000362E2F8121112BC08091B9058823B9F023
:10E9A00080915701882359F081E09091B905911128
:10E9B00080E024E04BE256E16E810E947AB7662047
:10E9C000E9F18981873009F478C093E038C08091FB
:10E9D000B4051092B405882319F30E94C22F8091C8
:10E9E000D0058823E9F22896E2E10C9468EE8F8145
:10E9F000813011F58091B905813079F0809157010E
:10EA00008823E9F281E09091B905913009F080E026
:10EA100023E041E256E16D81D0CF8091B4051092A0
:10EA2000B405882359F380E992E70E94A9B8809140
:10EA3000D005882319F3D7CF611003C092E09887DF
:10EA400042C02F81223009F0BCCF8091B9058230BD
:10EA500029F180915701882361F081E09091B905F7
:10EA6000923009F080E023E047E156E16C810E949A
:10EA70007AB78981873029F180915F049091600491
:10EA8000A0916104B09162048093390490933A0498
:10EA9000A0933B04B0933C0423E022C18091B405D1
:10EAA0001092B4058823A9F28FED9AEA0E94A9B8C2
:10EAB0008091D005882369F296CF9F81933009F425
:10EAC000C8C024E0288780915F0490916004A091E1
:10EAD0006104B09162048093390490933A04A09346
:10EAE0003B04B0933C0488859F8189131EC08091AC
:10EAF000B9052885821709F4F5C08091570188234C
:10EB0000A1F0FF80F71811E08091B9059F8189136A
:10EB100010E089E394E00E94BF2100E09C0147EFF0
:10EB200055E16F2D812F0E94192A88858F5F2F81D3
:10EB300082131DC08091B905821709F403C1809129
:10EB400057018823A1F0FF80F71811E08091B905E3
:10EB50009F81891310E087E894E00E940D2200E075
:10EB60009C0141EF55E16F2D812F0E94192A888564
:10EB70008E5F2F81821316C08091B905821709F428
:10EB80001BC180915701882369F06F81671981E06B
:10EB90009091B9052F81921380E023E044EE55E176
:10EBA0000E947AB788858D5F9F81891321C08091EB
:10EBB000B905891709F411C1809157018823C1F063
:10EBC0005F924F9286ED95E19F938F938F81871986
:10EBD0008F9381E09091B9052F81921380E08F93FC
:10EBE0000E94FD210F900F900F900F900F900F90AB
:10EBF00088858C5F9F81891321C08091B905891711
:10EC000009F4FDC0809157018823C1F03F922F92F3
:10EC100087EC95E19F938F938F8187198F9381E084
:10EC20009091B9052F81921380E08F930E94FD216E
:10EC30000F900F900F900F900F900F908F818F5F1C
:10EC40008F839A818913A5CE28852B5F2093B305E6
:10EC5000CACE80915E0488878091B9058330B9F46B
:10EC60008091B4051092B405882389F0988521E03D
:10EC7000922798878F818093570189E99CE2892B9D
:10EC800011F00E94992C8091D0058111ACCE809119
:10EC90005701882309F415CF81E09091B90593308D
:10ECA00009F080E0988527E036E1911102C023E069
:10ECB00036E101E04AE056E16B810E94192A809119
:10ECC0005F0490916004A0916104B091620480930C
:10ECD000390490933A04A0933B04B0933C0424E09D
:10ECE000288723CF8091B4051092B405882309F4B6
:10ECF00004CF0E9450B86091390470913A04809119
:10ED00003B0490913C040E9468EF29E8822E2CE697
:10ED1000922E31EFA32E31E7B32E6B0114E6E12ED4
:10ED2000F12C00E010E020E030E0A90169E374E09C
:10ED300087EF95E10E945CB88091D005882309F4A3
:10ED4000DCCE51CE8091B4051092B405882309F42D
:10ED5000F6CE20E030E048EC52E4609187047091F8
:10ED600088048091890490918A040E94CBE720E076
:10ED700030E04AEF54E40E9484EE0E9468EF912C48
:10ED8000812C80E5A82E87E3B82E6B0110EAE12ED6
:10ED90001FE0F12E00E010E020E338EF4FEF5FEFCF
:10EDA00067E874E081EF95E10E945CB88091D0053E
:10EDB000882309F4C4CE17CE8091B4051092B4050F
:10EDC000882309F4DECE82E29FE20E94A9B88091F6
:10EDD000D005882309F4D5CE06CE8091B4051092D3
:10EDE000B405882309F4E8CE4114510411F00E94BF
:10EDF000EB1D8091D005882309F4DECEF4CD8091FF
:10EE0000B4051092B405882309F4FCCE2114310412
:10EE100011F00E94E41D8091D005882309F4F2CE00
:10EE2000E2CD67EF79EA82E00C9490B96BEF79EA72
:10EE300081E00C9490B96FEF79EA80E00C9490B97E
:10EE400061EE77EA83E00C9490B9CF92DF92EF9273
:10EE5000FF920F931F9387E7C82E88E1D82EF12CDD
:10EE6000E12C09E718E130E020E04DE052E769E8E5
:10EE700078E18EE898E10E949E351F910F91FF90F6
:10EE8000EF90DF90CF900895CF92DF92EF92FF92B4
:10EE90000F931F9383E8C82E87E1D82EF12CE12C25
:10EEA00004E018E130E020E04FEB5AE365E877E159
:10EEB0008AE897E10E949E351F910F91FF90EF9095
:10EEC000DF90CF9008951092BA050C94F1C4B0E091
:10EED000A0E0EDE6F7E70C9454EEADB6BEB6809137
:10EEE000A30E60EE75E0882311F063EA7EE0FB017B
:10EEF00001900020E9F7CF01861B970B01962DB7F3
:10EF00003EB7281B390B0FB6F8943EBF0FBE2DBF7E
:10EF10008DB79EB701967C0180E2EDB7FEB7818385
:10EF2000C70101960E94A8F083E3C82E88E1D82E7D
:10EF300005E318E130E020E047EE57E761E478E1CF
:10EF400088E498E10E949E350FB6F894BEBE0FBECD
:10EF5000ADBEEAE00C9470EEAAE0B0E0E2EBF7E7B9
:10EF60000C945AEE809157018823F1F01F9289E0AA
:10EF70008F938091350490E001969F938F938CE856
:10EF800095E19F938F938E010F5F1F4F1F930F93F8
:10EF90000E94FFE6B80181E895E10E94B3290FB60F
:10EFA000F894DEBF0FBECDBF84E0809357018091FF
:10EFB0003404811108C020E040E070E060E085E6A4
:10EFC0009EE20E94E22D2A96E4E00C9476EEB0E0F8
:10EFD000A0E0EDEEF7E70C9456EECDB6DEB6E0EE2F
:10EFE000F5E0DF010D900020E9F7CD01885D954047
:10EFF0002DB73EB7281B390B0FB6F8943EBF0FBE96
:10F000002DBF0DB71EB70F5F1F4FFF93EF938CE21D
:10F0100098E19F938F931F930F930E94FFE67801CF
:10F0200034E0E30EF11C0F900F900F900F900F90B3
:10F030000F90D7018D917D01882349F0082E000C97
:10F04000990B0E9465F0F70131978083F2CF67E258
:10F0500078E1C8010E9498E6C8010E9495230FB686
:10F06000F894DEBE0FBECDBE0E94562F0E9438B768
:10F07000E8E00C9472EE8FE897E10C949523B0E0F1
:10F08000A0E0E5E4F8E70C944CEE0E94D82DD82FD0
:10F0900061E081E00E949C23C091BA052C2E85E09E
:10F0A000382E3C0E07EE1DE192E3A92E96E1B92E13
:10F0B00084E0782E7C1A2BEEE22E2DE1F22E33E442
:10F0C000832E36E1932E83E0682E6C1A44EEC42E14
:10F0D0004DE1D42E82E0582E5C1A81E0482E4C1A65
:10F0E000C11129C08091B9058823A1F080915701F1
:10F0F000882361F0622D619581E09091B9059111AD
:10F1000080E024E042E756E10E947AB7DD2309F46B
:10F11000A8C0C4C08091B4051092B405882331F30F
:10F120000E94C22F8091D005882301F3CDB7DEB7AE
:10F13000E2E10C9468EEC13019F58091B905813097
:10F1400081F080915701882309F4A6C081E0909155
:10F15000B905913009F080E023E040E656E1642DE6
:10F16000D3CF8091B4051092B405882351F384EC79
:10F170009FE20E94A9B88091D005882311F3D6CFD1
:10F18000C23009F070C08091B9058230E1F0809101
:10F190005701882309F480C0DF92CF9281E596E180
:10F1A0009F938F935F9281E09091B905923009F01F
:10F1B00080E08F930E94FD210F900F900F900F9091
:10F1C0000F900F90A3CF8091B4051092B4058823BF
:10F1D000F1F2C114D10411F00E94E41D8091D00518
:10F1E0008823A9F2A3CF8091B4051092B405882397
:10F1F00009F442C0E114F10411F00E94EB1D80916A
:10F20000D0058823C9F192CF8091B4051092B4053E
:10F21000882381F00115110511F00E94E71D8091EE
:10F22000D005882339F082CFC430D9F48091B90554
:10F23000843051F380915701882399F01F930F93E5
:10F24000BF92AF927F9281E09091B905943011F511
:10F250008F930E94FD210F900F900F900F900F90B1
:10F260000F9085E01CC0D11119C0C330E9F6809120
:10F27000B905833009F4B7CF80915701882389F30A
:10F28000FF92EF929F928F926F9281E09091B905D9
:10F290009330F1F280E0DCCFDD2331F283E0CF5F09
:10F2A0003C121ECF8093B30541CFA5E0B0E0EBE563
:10F2B000F9E70C944CEE0E94C52D282E8091651321
:10F2C00084FB222720F92983312C84FF03C00E946C
:10F2D0008F3A382E61E081E00E949C237090BA053D
:10F2E000572C85E0870D8A8380E042EFE42E47E1CA
:10F2F000F42E91E0492E4718972D91959B8302E6B5
:10F300001AE35FE0C52E58E1D52E92E097199C8351
:10F3100093E097199D8360EA862E67E1962E75EB40
:10F32000A72E77E1B72E2A81721609F427C277201B
:10F3300031F1211064C00E949D3A882309F48FC1E5
:10F3400081E0781609F457C192E0692E761074C1F5
:10F350008091B905781609F485C1809157018823F9
:10F3600009F46AC1672D651981E09091B90597117B
:10F3700080E023E04BEE57E10E947AB75DC18091B7
:10F38000B905882361F180915701882391F281E0CA
:10F390009091B905911180E024E04BE158E16B8137
:10F3A0000E947AB7222039F234E0632E76104AC0E8
:10F3B0008091B905781609F466C1809157018823B8
:10F3C00009F440C0672D651981E09091B905971146
:10F3D00080E023E04FED57E10E947AB733C080917F
:10F3E000B4051092B405882371F20E94C22F809157
:10F3F000D005882341F22596E2E10C9468EE81E085
:10F40000781609F494C092E0791609F4BEC023E09E
:10F410007212CACF8091B905833009F4DBC08091A4
:10F420005701882309F4C0CF81E09091B90593304A
:10F4300009F080E023E04FEF57E16D810E947AB739
:10F4400024E0622E81E0860D781215C08091B90506
:10F45000781609F429C180915701882361F0672D3E
:10F46000651981E09091B905971180E023E041EDA5
:10F4700057E10E947AB782E0860D781215C080911C
:10F48000B905781609F421C180915701882361F0EC
:10F49000672D651981E09091B905971180E023E00F
:10F4A00043EC57E10E947AB783E0860D9981992356
:10F4B00009F43FC1311039C078121CC08091B905E0
:10F4C000781609F413C180915701882399F01F928F
:10F4D000BF92AF92872D85198F9381E09091B905E6
:10F4E000971180E08F930E94FD210F900F900F9055
:10F4F0000F900F9084E0860D781215C08091B905A9
:10F50000781609F405C180915701882361F0672DB1
:10F51000651981E09091B905971180E023E044EAF4
:10F5200057E10E947AB785E0860D7394FCCE8091F6
:10F53000B9058130D1F080915701882309F434CF87
:10F540001F930F93DF92CF924F9281E09091B90574
:10F55000913009F080E08F930E94FD210F900F9071
:10F560000F900F900F900F901FCF8091B4051092C5
:10F57000B405882301F30115110511F00E94623AC8
:10F580008091D0058823B9F236CF8091B9058230B9
:10F5900091F080915701882309F406CF81E0909182
:10F5A000B905923009F080E023E044E058E16C8135
:10F5B0000E947AB7F9CE8091B4051092B4058823E1
:10F5C00041F384E497E70E94A9B88091D00588238D
:10F5D00001F311CF8091B4051092B405882309F48A
:10F5E0001ECF86E99FE60E94A9B88091D0058823A6
:10F5F00009F415CF00CF8091B9058130F9F08091E1
:10F600005701882309F4A0CE8EEA9AE39F938F9343
:10F61000FF92EF924F9281E09091B905913009F0FD
:10F6200080E08F930E94FD210F900F900F900F901C
:10F630000F900F9082E0682E6394B8CE8091B4054D
:10F640001092B4058823D9F28EEA9AE3892B11F03F
:10F650000E94AE3A8091D005882389F2CCCE6624F0
:10F66000639474CE8091B4051092B405882309F494
:10F6700074CE88EA9CE60E94A9B88091D0058823C0
:10F6800009F46BCEB8CE8091B4051092B4058823EE
:10F6900009F493CE8BEE93E80E94A9B88091D0052F
:10F6A000882309F48ACEA7CE8091B4051092B405C0
:10F6B000882309F4D0CE8FE398E70E94A9B88091FF
:10F6C000D005882309F4C7CE96CE8091B405109258
:10F6D000B405882309F4D8CE83EE9EE60E94A9B82B
:10F6E0008091D005882309F4CFCE85CE8091B405D2
:10F6F0001092B405882309F4E6CE8FE897E10E94C2
:10F7000095238091D005882309F4DDCE872D0DCF78
:10F710008091B4051092B405882309F4F4CE8AEDE3
:10F720009CEA0E94A9B88091D005882309F4EBCE09
:10F73000EDCF781212C09091B905791681F08091C1
:10F740005701882351F0672D651981E0791280E017
:10F7500020E243E957E10E947AB784E0E5CE809148
:10F76000B4051092B405882351F390924E0580920F
:10F770004D058091D005882311F3C8CF8093B30540
:10F780003ACEA5E1B0E0E7ECFBE70C9458EE8091AF
:10F79000B4051092B405882331F00E94C22F6596FB
:10F7A000E6E00C9474EE60E085E00E949C230091FA
:10F7B000BA0510E08AE3F82E90E2E92E011130C07C
:10F7C00080915701882341F030E020E043E063E579
:10F7D00077E1812F0E942329F982EA8242E150E0F9
:10F7E00064E177E1CE0103960E94D6E68C8987FD1D
:10F7F0001C8A0530C1F580915701882349F09E018C
:10F800002F5F3F4F41E06AE077E1812F0E9423297B
:10F810000F5F1F5F153091F687E08093B305BFCF70
:10F82000013051F4809157018823B1F230E020E09B
:10F8300041E066E477E1CDCF023009F580915701D0
:10F84000882351F230E020E041E06BE377E1C1CF63
:10F8500080915701882309F4BFCF30E020E043E0D6
:10F8600061E377E1B6CF063099F68091570188239E
:10F8700079F230E020E041E06CEF76E1C6CF033072
:10F8800039F3043009F0A8CF80915701882309F497
:10F89000A3CF30E020E041E066E177E19ACFA5E137
:10F8A000B0E0E5E5FCE70C9458EE8091B4051092C9
:10F8B000B405882331F00E94C22F6596E6E00C94CF
:10F8C00074EE60E085E00E949C230091BA0510E090
:10F8D0008AE3F82E90E2E92E01110CC080915701C5
:10F8E000882341F030E020E043E06BEE76E1812FA9
:10F8F0000E942329F982EA8242E150E064EE76E137
:10F90000CE0103960E94D6E68C8987FD1C8A0130C1
:10F9100069F480915701882349F09E012F5F3F4F82
:10F9200041E06FED76E1812F0E942329F982EA827E
:10F9300042E150E06BED76E1CE0103960E94D6E6FF
:10F940008C8987FD1C8A023069F4809157018823D5
:10F9500049F09E012F5F3F4F41E062ED76E1812F3C
:10F960000E942329F982EA8242E150E06AEC76E1C2
:10F97000CE0103960E94D6E68C8987FD1C8A03304F
:10F9800069F480915701882349F09E012F5F3F4F12
:10F9900041E066EC76E1812F0E9423290F5F1F5F13
:10F9A000153009F099CF84E08093B30586CFA5E1A7
:10F9B000B0E0EDEDFCE70C9458EE8091B4051092A8
:10F9C000B405882331F00E94C22F6596E6E00C94BE
:10F9D00074EE60E085E00E949C230091BA0510E07F
:10F9E0008AE3F82E90E2E92E01110CC080915701B4
:10F9F000882341F030E020E042E067EB76E1812FA0
:10FA00000E942329F982EA8242E150E065EB76E127
:10FA1000CE0103960E94D6E68C8987FD1C8A0130B0
:10FA200069F480915701882349F09E012F5F3F4F71
:10FA300040E06CEA76E1812F0E942329F982EA8274
:10FA400042E150E068EA76E1CE0103960E94D6E6F4
:10FA50008C8987FD1C8A023009F04EC080915701C5
:10FA6000882349F09E012F5F3F4F40E06FE976E128
:10FA7000812F0E942329F982EA8242E150E06BE75C
:10FA800076E1CE0103960E94D6E68C8987FD1C8A1A
:10FA9000053069F480915701882349F09E012F5F5A
:10FAA0003F4F40E06CEA76E1812F0E942329F982E2
:10FAB000EA8242E150E067E776E1CE0103960E94D8
:10FAC000D6E68C8987FD1C8A063089F5809157011E
:10FAD000882349F09E012F5F3F4F40E06FE976E1B8
:10FAE000812F0E9423290F5F1F5F153009F07CCF03
:10FAF00088E08093B30569CF033059F480915701B2
:10FB0000882309F4B8CF30E020E040E06DE876E1EA
:10FB1000AFCF043009F0AFCF80915701882309F4AB
:10FB2000AACF30E020E042E06DE776E1A1CF0730D8
:10FB3000D1F6809157018823B1F230E020E040E017
:10FB40006DE876E1CDCF0E949629809155048770AB
:10FB5000873041F420E040E070E060E084EC9CEA13
:10FB60000C94E22D0895B0E0A0E0E9EBFDE70C94E1
:10FB700052EEEC018B81811106C080E0CDB7DEB77B
:10FB8000ECE00C946EEE09891A892B893C890417E4
:10FB900015072607370788F34A015B01823031F4E5
:10FBA00088869986AA86BB8681E0E8CF8114910475
:10FBB000A104B10449F4188619861A861B861C8292
:10FBC0001D821E821F82F0CF088519852A853B85FC
:10FBD000E98DFA8D858590E00996B901A80141501B
:10FBE000510961097109082E04C0769567955795EA
:10FBF00047950A94D2F775016401E1E0CE1AD10865
:10FC0000E108F10804C0F694E794D794C7948A9564
:10FC1000D2F7C416D506E606F70620F0012B022B14
:10FC2000032B11F58D899E89AF89B88D8C839D83B7
:10FC3000AE83BF838E010C5F1F4FC114D104E1045A
:10FC4000F10409F4ADCF4C815D816E817F81980113
:10FC5000898D9A8D0E943DDA91E0C91AD108E10898
:10FC6000F1088111EACF89CFC41AD50AE60AF70A4A
:10FC7000E1CFB0E0A0E0EFE3FEE70C944CEEEC0146
:10FC80004B018A018B81811107C08FEF9FEFCDB7A8
:10FC9000DEB7E2E10C9468EE898180FFF6CF8989B6
:10FCA0009A89AB89BC89488559856A857B85841B7F
:10FCB000950BA60BB70BA80170E060E084179507C1
:10FCC000A607B70708F48C0168011E0124E0220E84
:10FCD000311CC114D10409F4AAC0488559856A852C
:10FCE0007B855A0181E0B822898D9A8D2A013B01DA
:10FCF00039E076946794579447943A95D1F72B81DD
:10FD0000FC01223089F5628D738D848D958D640D93
:10FD1000751D861D971DE12C22E0F22EEA18FB08C6
:10FD2000CE14DF0408F47601E114E2E0FE0671F47B
:10FD300040903C1150903D1160903E1170903F11E9
:10FD4000641575058605970509F04EC040E00E94D0
:10FD500061C3882309F499CFB501645C704FA70192
:10FD6000C4010E947AF052C0F480FA94F420A114E5
:10FD7000B10471F4F1100CC0452B462B472B51F503
:10FD80008D899E89AF89B88D8C839D83AE83BF8317
:10FD9000E98DFA8D4C805D806E807F8022E0421A72
:10FDA000510861087108858504C0440C551C661C07
:10FDB000771C8A95D2F786859785A089B189480EE8
:10FDC000591E6A1E7B1EC301B2016F0D711D811D7C
:10FDD000911DA1CF4C815D816E817F8191010E9437
:10FDE0003DDA8111D5CF51CFA0914111B09142118F
:10FDF000ED91FC9111970088F189E02D9401AB0100
:10FE0000BC01CD010995882309F43FCF8E0C9F1CBE
:10FE100088859985AA85BB858E0D9F1DA11DB11D65
:10FE200088879987AA87BB87CE18DF0852CFC80179
:10FE30002ECF0F931F93CF93DF93FC0123812223B7
:10FE400031F080E0DF91CF911F910F9108958B01E8
:10FE5000EC01FB018789803139F582E08B831D8AB3
:10FE60001E8A1F8A188E808D918DB0E0A0E025E05B
:10FE7000880F991FAA1FBB1F2A95D1F7898B9A8BD0
:10FE8000AB8BBC8B1A8F098F81E08983188619860A
:10FE90001A861B861C821D821E821F82188A1C865F
:10FEA0001D861E861F86CECF803259F683E08B8357
:10FEB000428D538D648D758D4D8B5E8B6F8B788FDE
:10FEC0009E012F5E3F4FC8010E94BADA8111DACF3E
:10FED000B8CFCF93DF93EC010E9423DB1B82DF912D
:10FEE000CF910895CF93DF93EC01462F41706C853D
:10FEF0007D858E859F850E9461C3882351F0888906
:10FF000020E2829FC0011124845C904FDF91CF9149
:10FF1000089590E080E0FACFCF93DF93EB01FC01EE
:10FF20002381211104C080E0DF91CF9108952250F8
:10FF3000223028F48FE28883198281E0F5CF60E0D7
:10FF4000D1DF009781F3DC0160E080E09EE22D913B
:10FF5000203299F0883031F49E01260F311DF901CD
:10FF600090836F5F9E01260F311DAD0141505109F5
:10FF7000FA014081F90140836F5F8F5F8B3039F761
:10FF8000FE01E60FF11D1082D8CFACE0B0E0EBEC43
:10FF9000FFE70C944DEE5C01DC0159968D909C902E
:10FFA000F40181859285A385B4859C01AD012F5F05
:10FFB0003F4F4F4F5F4F29873A874B875C87D5016B
:10FFC00014964D905D906D907C901797411451045C
:10FFD0006104710409F459C0BFEF4B1A5B0A6B0A44
:10FFE0007B0A312C730162011D821E821F821886DA
:10FFF000F40181859285A385B4852D813E814F8151
:020000021000EC
:100000005885281739074A075B0708F056C08985C5
:100010009A85AB85BC858C159D05AE05BF0550F452
:1000200082E0C82ED12CE12CF12C92E0492E512CEB
:10003000612C712C9E012F5F3F4FB701A601C401B7
:100040000E943DDA8823C9F189819A81AB81BC8104
:10005000892B8A2B8B2B01F1260137019FEF491A3F
:10006000590A690A790A2D813E814F8158852F5F8F
:100070003F4F4F4F5F4F2D833E834F8358873FEF56
:10008000C31AD30AE30AF30AB3CF408051806280D7
:10009000738033243394A6CFC414D504E604F70444
:1000A00011F70FEF1FEF2FEF3FE0B701A601C401DB
:1000B0000E94C2D9782E811106C0712C872D2C96F2
:1000C000E1E10C9469EEF501448155816681778107
:1000D000411551056105710539F097018601C4018B
:1000E0000E94C2D9882349F3D5011496CD92DD929E
:1000F000ED92FC921797332051F0D701C60101967B
:10010000A11DB11DF40180839183A283B383F50106
:1001100085899689A789B08D892B8A2B8B2B71F6BF
:10012000C58AD68AE78AF08E818180688183C6CFAE
:1001300040E050E0BA0117CD4F925F926F927F92EC
:10014000AF92BF92CF92DF92EF92FF920F931F93E5
:10015000CF93DF931F92CDB7DEB78C017B015A019D
:10016000C22EDB0159968D919C91F801928F818F5F
:10017000CB01DEDF712CF70180859185A285B385E7
:10018000418952896389748984179507A607B7073F
:1001900008F051C055E0B695A795979587955A9563
:1001A000D1F7F82FFF70DF2ED70113968C91823094
:1001B00010F480E0D9C041E050E0BE016F5F7F4F96
:1001C000C70157DD0197A9F7F70180859185A285C1
:1001D000B3854F96A11DB11D80879187A287B387F4
:1001E000F0E2DF9EB0011124645C704F611571056F
:1001F00001F3DB018C91882341F0853E09F04BC06F
:10020000772029F077247394B6CF71100EC08091B7
:100210003C1190913D11A0913E11B0913F11F80118
:1002200084879587A687B787D08ADB018C91811157
:10023000E9CF772473948C2D8274823409F0B9CF7E
:10024000772009F4A1C0F801D08861E0C8014ADE36
:10025000009709F4AECF20E2DC011D922A95E9F760
:100260002BE0F501DC0101900D922A95E1F721E2E6
:1002700038E2FC01318B208B40E058E057874687FD
:10028000338B228B318F208F578B468B0E9418C364
:10029000811109C08ECF4BE050E0C5010E946DF086
:1002A000892B09F068CFF0E2DF9ED00111249D0177
:1002B000245C304FF9018385817121F08C2D82718E
:1002C00009F000C1F801818D928D40913C1150914F
:1002D0003D1160913E1170913F11448755876687AB
:1002E0007787D08AFD01E45CF04F44885588712CF3
:1002F000612C320155244424D80155964D925D92CB
:100300006D927C925897428D538D70E060E0442945
:1003100055296629772955964D935D936D937C9366
:100320005897D9011B962C91287109F0BDC0848D76
:10033000958DA68DB78DF801818B928BA38BB48B95
:1003400081E083838C2D8F70F80181831482158264
:1003500016821782108611861286138681E0C4FEEB
:1003600003C0C8010E9457DB0F90DF91CF911F910E
:100370000F91FF90EF90DF90CF90BF90AF907F9064
:100380006F905F904F900895D70113968C911397BB
:10039000823009F40ECF51968D919D910D90BC91B4
:1003A000A02D803E9F4FAF41B10508F002CFC7019D
:1003B000ECDD882309F4FDCE0E9418C3882309F4DC
:1003C000F8CED7015996ED91FC915A9714964D901D
:1003D0005D906D907C901797B2E04B1A51086108C0
:1003E0007108858504C0440C551C661C771C8A95D1
:1003F000D2F786859785A089B189480E591E6A1E55
:100400007B1E81E08093401140923C1150923D113F
:1004100060923E1170923F11ECE3FFE080E092E0C9
:10042000DF019C011D9221503040E1F7DD24D3947F
:10043000D7015996ED91FC918481D816C0F4809132
:10044000411190914211DC01ED91FC910288F389F8
:10045000E02D2CE33FE0B301A2014D0D511D611DC4
:10046000711D0995882309F4A4CED394E1CF258585
:1004700080E092E0A0E0B0E004C0880F991FAA1FBE
:10048000BB1F2A95D2F7F701418952896389748984
:10049000840F951FA61FB71F818B928BA38BB48BE4
:1004A0008CE39FE0D12CD7CE203161F498012F5EF0
:1004B0003F4F0E94BADA882329F084E0D8011396CE
:1004C0008C9340CFD80113961C9273CEFC012381EC
:1004D0002111FFCC0895A1E4B0E0E1E7F2E80C942B
:1004E0004CEE4C015B017A01222E19821C821C8E7B
:1004F0001F8E6115710569F410E0CE014C96E6DFA0
:10050000CE010196E3DF812FCF5BDF4FE2E10C9458
:1005100068EEFC0183818111EFCFFA0180818F3277
:1005200051F18B01CE0101966C012C0180E2382E35
:10053000360122963FAE229721963FAE21973FAEDD
:100540003EAE3DAE3CAE3BAE3AAE39AE38AE3FAA63
:10055000970190E047E0D9018D91882309F446C0C6
:100560008F3209F443C08E3201F54A3029F298E007
:100570004AE09D01F0CFFB0183818250823098F0E8
:10058000618D728DCE014C9654DC882309F4B4CF72
:100590008E01045E1F4FC7017C010196F701208187
:1005A0002F32D1F3BFCF8B01F6CFE7E3F6E22491F0
:1005B000222321F031968213FACF9ECF491708F4F7
:1005C0009BCF813208F498CF8F3709F495CF3FE95C
:1005D000380F3A3108F420EEE7E3F0E0EC0FFD1FAE
:1005E000E90FF11D820F80839F5FC3CF8FA98032F7
:1005F00009F482CF7901F90180812F5F3F4F8F325B
:10060000C9F38823C1F021E0AE01495C5F4FB80116
:10061000C60192DD882309F46FCF0A151B0511F07E
:10062000C80157DCCE014C964C145D0409F0C3019F
:1006300086016C017ECF222DAE01495C5F4FB8016F
:10064000C4017ADD182F59CFEF92FF921F93CF93F9
:10065000DF93CDB7DEB728970FB6F894DEBF0FBE95
:10066000CDBF182F81E5E82E81E1F82EF7016085D6
:100670007185072E000C880B990B0E946CE76D8327
:100680007E838F839887F70184819581A681B781C6
:1006900089839A83AB83BC83AE014B5F5F4FBE01FE
:1006A0006F5F7F4F80E00E94086C90E9E92E95E033
:1006B000F92EF70160857185072E000C880B990BC8
:1006C0000E946CE76D837E838F839887F701848116
:1006D0009581A681B78189839A83AB83BC83AE0160
:1006E0004B5F5F4FBE016F5F7F4F8FEF0E94086CC3
:1006F00087E11802F0011124EF5AFE4E628570E086
:1007000083E396E20E94464DF701628570E08EE237
:1007100096E20E94464D28960FB6F894DEBF0FBEB3
:10072000CDBFDF91CF911F91FF90EF9008950F9370
:100730000FB70F9300916E000B7F00936E007894BB
:100740000F930BB70F930CB70F921F922F933F93FA
:100750004F935F936F937F938F939F93AF93BF93C9
:10076000EF93FF9311240E946190FF91EF91BF914D
:10077000AF919F918F917F916F915F914F913F9139
:100780002F911F900F900CBF0F910BBF0F91046022
:10079000F89400936E000F910FBF0F911895CF93AF
:1007A000DF931092F405C1E5D1E1198618860E9405
:1007B00071BC1A865D98C0E9D5E0198618860E943A
:1007C000AE1D1A865C98DF91CF910895109227068E
:1007D000E6DF0C94562FA9E0B0E0E1EFF3E80C94CB
:1007E0004CEE21E02D838091591190915A11892B63
:1007F00009F41D8261E081E00E949C237090BA059B
:100800007E8285E0870D8F8344244A94512C83E0B7
:100810008719888782E08719898781E0682E6718A1
:10082000272C219486E0382E3718711015C080913E
:10083000B905882309F4DCC080915701882309F4A5
:10084000A3C181E09091B905911180E024E04CE3CF
:1008500059E1622D0E947AB78091591190915A11F5
:1008600090933A048093390491E07912EEC080911C
:10087000B905813009F4CEC080915701882309F46D
:100880004EC011E08091B905813009F010E060910F
:10089000390470913A04072E000C880B990B0E94C2
:1008A0006CE769837A838B839C83CE0101960E94D7
:1008B000782300E09C0145E359E1662D812F0E94D9
:1008C000192A809127068093390483E0781227C083
:1008D0001092D9058091B905833009F4F9C080914F
:1008E00057018823E1F011E08091B905833009F0C8
:1008F00010E08091390424E6829FC00111248158C0
:100900009F4FB2010E94FCED862F0E94406800E0DC
:100910009C0147E259E16885812F0E94192A10E065
:1009200000E034E0F32EE72C8E81E81A00933904BE
:100930007F101FC0F801EE0FFF1FE05FF64E85919C
:1009400094919093DB058093DA058091B905871522
:1009500009F4F9C080915701882359F081E0909102
:10096000B9059F1180E023E04DE159E16E2D0E9411
:100970007AB78F2D0F5F1F4F95E0F92E8530B1F6B6
:100980008091980590919905892B21F49D81992357
:1009900009F4F8C026E0721221C08091B9058630B2
:1009A00009F4E2C0809157018823C1F086EE93E8F4
:1009B0009F938F9384E199E19F938F933F9281E07E
:1009C0009091B905963009F080E08F930E94FD2147
:1009D0000F900F900F900F900F900F9087E091E085
:1009E0009D8373942F81721220CF8093B3050EC024
:1009F0008091B4051092B405882309F41DCF0E949C
:100A0000C22F8091D005882309F416CF2996E2E100
:100A10000C9468EE8091B4051092B405882309F413
:100A20002BCF0E9450B801E813E725EF30E050E0EB
:100A300040E069E374E085E399E10E94EAB88091BF
:100A4000D005882309F418CFE1CF22E0721239CF04
:100A50008091B905823019F180915701882309F4FA
:100A60005ECF11E08091B905823009F010E060910D
:100A7000980570919905072E000C880B990B0E9420
:100A80006CE769837A838B839C83CE0101960E94F5
:100A9000782300E09C0141E359E169850FCF809103
:100AA000B4051092B4058823B9F20E9450B80EEA3A
:100AB0001DE123E730E050E040E068E975E081E3C4
:100AC00099E10E94EAB88091D005882329F29ECF4F
:100AD0008091B4051092B405882309F400CF0E94D8
:100AE00050B86091390470E090E080E00E946AE7BD
:100AF00029EC38EC48EC5EE30E94CBE720E030E0E4
:100B000040E05FE30E9484EE0E9468EF4FEA842E8B
:100B100048E6942E55EEA52E51E7B52E6B0114E64E
:100B2000E12EF12C00E010E020E030E0A90169E3C3
:100B300074E087E299E10E945CB88091D005882337
:100B400009F4CDCE63CF8091B4051092B40588230B
:100B500009F400CF86E993E70E94A9B88091D005F7
:100B6000882309F4F7CE52CF8091B4051092B405D2
:100B7000882309F417CF2ADE8091D005882309F451
:100B800011CF44CF86E02DCF8091591190915A1109
:100B900090933A048093390494CEB0E0A0E0E3ED62
:100BA000F5E80C9452EEB0E4A0E06A2F70E0AB01DF
:100BB0004B0F511D55954795411111C0EAEBFBE2D2
:100BC00065917491072E000C880B990B0E946CE7BD
:100BD000CDB7DEB7ECE00C946EEEB42FE8CFA417DF
:100BE00011F0B41303C0E6EBFCE2EACF9A01215006
:100BF0003109220F331F220F331FF901E854F44D3E
:100C0000E590F490F901E454F44DC591D4918E151A
:100C10009F051CF3A42FC817D9070CF4C6CFF90100
:100C2000E654F44D05911491F901E254F44DC59048
:100C3000D490BC016E197F09072E000C880B990B0C
:100C40000E946CE74B015C01B601601B710B072E23
:100C5000000C880B990B0E946CE79B01AC01C5014D
:100C6000B4010E94CBE74B015C01BE016E197F0904
:100C7000072E000C880B990B0E946CE79B01AC01BE
:100C8000C501B4010E94FBEE6B017C01B801012E8D
:100C9000000C880B990B0E946CE79B01AC01C7010B
:100CA000B6010E9484EE94CFEF92FF920F931F93B0
:100CB000CF93DF93C82F7B018A0180910A0683308E
:100CC00090F00E941E49C7010E940D4181E995E202
:100CD0000E940D41CF3F79F58DE895E20E940D41CC
:100CE0008AE00E94EC405BDDA8958091240581118B
:100CF0003EC081E08093240582E080930A064FDDA8
:100D0000D5E1D150149A49F169E170E080E090E0BA
:100D10000E94D9BBA895149868E270E080E090E04A
:100D20000E94D9BBA89568E270E080E090E00E9444
:100D3000D9BBA895E6CFC7FDD3CF8BE895E20E943B
:100D40000D416C2F0C2E000C770B880B990B0E9419
:100D500038B18AE00E94EC40C3CF64E875E2CF3F2F
:100D600011F068E875E240E0C8010E94544DCDB72B
:100D7000DEB7E6E00C9474EEB0E0A0E0E2ECF6E85A
:100D80000C944EEEEC016B014A01B22EFA01408048
:100D9000518062807380A30192016D817E818F8179
:100DA00098850E9466E78823A1F04D825E826F825B
:100DB0007886AA24A39420E030E0A901F4016081A0
:100DC0007181828193810E94E7EF18160CF0A12CAB
:100DD000AC828C818230A1F0833009F44FC0813025
:100DE000D1F52D813E814F815885F6016081718159
:100DF000828193810E9466E787FD2DC082E08C830B
:100E0000B7010F2C000C880B990B0E946CE79B011B
:100E1000AC016D817E818F8198850E9483EE9B015C
:100E2000AC01F60160817181828193810E94E7EFBC
:100E300087FD16C00E9465BC6B017C019801A8EE7D
:100E4000B3E00E94C0EDC60ED71EE81EF91EC88290
:100E5000D982EA82FB82CDB7DEB7E0E10C946AEE7C
:100E60000E9465BC088119812A813B81601B710B3E
:100E7000820B930B97FDEFCF83E08C834BE056E220
:100E80006BE176E28B2D10DFE6CF4FEA55E26CEB9B
:100E900075E20ACFCF93DF93A8958091531190917B
:100EA00054110E94B0B26093551170935611809303
:100EB00057119093581180919205909193056DDE92
:100EC000609394057093950580939605909397058C
:100ED000C0915311D091541180914F0190915001C4
:100EE000C817D90714F480E0D0DF80915911909190
:100EF0005A11181619066CF480914D0190914E010B
:100F00008C179D0734F44CEE55E269EF75E280E0F2
:100F1000CBDE209192053091930580914705909109
:100F200048052817390714F48FEFAFDF8091980533
:100F300090919905181619068CF42091920530911C
:100F4000930580914B0190914C018217930734F4E3
:100F50004CEE55E269EF75E28FEFA6DEDF91CF919F
:100F60000895A4E0B0E0E7EBF7E80C9452EE80912E
:100F70000A06811106C0A8952496ECE00C946EEE4A
:100F800028C1809139058111F7CF81E0809339051F
:100F900080919B04811107C0109239052496ECE0E2
:100FA0000C946EEE16C176DF10929B040E9465BC15
:100FB0004B015C010E9453B16B017C0160915301B4
:100FC00070915401072E000C880B990B0E946CE75E
:100FD0009B01AC01C701B6010E94E7EF18160CF4A3
:100FE000E7C06091591170915A11072E000C880BBF
:100FF000990B0E946CE769837A838B839C8334E02E
:10100000E32EF12C08E210E020E0AE014F5F5F4FCD
:1010100065E571E18BEB91E1AFDEC0905511D090A9
:101020005611E0905711F090581160915101709154
:101030005201072E000C880B990B0E946CE79B0154
:10104000AC01C701B6010E94E7EF1816CCF460911D
:10105000530170915401072E000C880B990B0E94CC
:101060006CE79B01AC01C701B6010E9466E787FFF0
:1010700007C00E945CB10E9463EF7595679501C03F
:1010800060E060935B1180914D1190914E11A091A1
:101090004F11B09150110097A105B105C1F0A50104
:1010A0009401281B390B4A0B5B0BDA01C901B7FD10
:1010B0000EC00E9453B10E9463EF20914B113091FA
:1010C0004C11621773070CF47DC00E9471BC0E9422
:1010D000FD6420E030E04AEF52E40E94E7EF18168A
:1010E0000CF463C08091970490919804A0919904A6
:1010F000B0919A040097A105B105A1F0881A990A48
:10110000AA0ABB0AB7FC0EC00E94FD640E9463EFEE
:101110002091950430919604621773070CF44BC02C
:101120000E94AE1D6091980570919905072E000CE4
:10113000880B990B0E946CE769837A838B839C836D
:1011400092E0E92EF12C04E110E02FEFAE014F5FA9
:101150005F4F64E975E084EC91E10EDE80909405C8
:1011600090909505A0909605B090970520E030E00E
:1011700040EA50E4C501B4010E94E7EF87FD11C0C9
:1011800020E030E04AEF52E4C501B4010E9466E776
:1011900018163CF00E94A9630E9463EF759567954D
:1011A00001C060E060939A05F7CE8FEF6EDE9ACFB4
:1011B00080E06BDE16CF4EEC55E26DED75E28FEF01
:1011C00073DDB0CF4EEC55E26DED75E280E06CDD85
:1011D0007ECFCF92DF92EF92FF92CF93DF93EC011D
:1011E000C880D980EA80FB808AE795E20E940D41A1
:1011F000C701B6010E94BC2ACC80DD80EE80FF8052
:1012000081EC91E30E940D41C701B6010E94BC2A06
:10121000C884D984EA84FB848DEB91E30E940D415C
:10122000C701B6010E94BC2A8AE00E94EC40DF910F
:10123000CF91FF90EF90DF90CF900895BC01209167
:1012400005053091060540910505509106052417C6
:10125000350731F481E02617370709F080E008955B
:101260009A01F1CF0F930FB70F9300916E000F9378
:101270000B7F00936E0000916F000D7F00936F0055
:101280000F930BB70F930CB70F921F922F933F93AF
:101290004F935F936F937F938F939F93AF93BF937E
:1012A000EF93FF9311240E94CD91FF91EF91BF9195
:1012B000AF919F918F917F916F915F914F913F91EE
:1012C0002F911F900F900CBF0F910BBF0F910260D9
:1012D000F89400936F000F9100936E000F910FBF71
:1012E0000F91189500C000C080914C0580FF1FC071
:1012F000459A8FEF8093BE0480914C0581FF1AC000
:10130000479A8FEF8093BF0480914C0582FF15C0F0
:101310002A988FEF8093C00480914C0583FF10C002
:1013200028988FEF8093C10400C000C008954598AD
:1013300081E0E0CF479881E0E5CF2A9A81E0EACFCB
:10134000289A81E0EFCF80918C04982F977F90931B
:101350008C04982F937081E011F080E008955E9ADC
:1013600008955E9880918C04886080938C04089521
:10137000E82FF0E021E030E0082E02C0220F331FFA
:101380000A94E2F72095309590918C0492239093E3
:101390008C04EA5DFD4F2081922321E019F020E0CA
:1013A000822F0895813079F038F08230C9F7159A8C
:1013B00090914B059B7F04C05E9A90914B059E7F58
:1013C00090934B05EDCF5E9A90914B059D7FF8CFA2
:1013D00080E0CEDF81E0CCDF82E0CADFB4CF8130B5
:1013E00079F070F0823071F021E030E001C0220F1E
:1013F0008A95EAF780918C04822B80938C0408955F
:101400005E98F2CF1598F0CFA6E8B0E0EAE0FAE8EF
:101410000C9456EEC358DF4F188219821A821B8231
:10142000CD57D04080915C0290915D02A0915E0208
:10143000B0915F02CF57DF4F88839983AA83BB8324
:10144000C158D04084E690E09093451180934411B8
:1014500010926911109268111092B90464E070E062
:10146000CE018F579F4F0E940CBC809144119091E8
:101470004511029690934511809344111092691181
:101480001092681181E0CA57DF4F8883C658D04058
:10149000CE018A579F4F0E947D6C68E470E089EE10
:1014A0009BE00E940CBC80E1E1ECF1E08E010F5F5B
:1014B0001F4FD80101900D928A95E1F760E170E02D
:1014C000C8010E940CBC8BE096E00E94856C3CE059
:1014D000D32EF8018D2D11928A95E9F7C8010E944B
:1014E000816C7E019DE6E90EF11C8FEFF701808390
:1014F000C7010E947D6C19821A821B821C82C8015E
:101500000E94856C80915F0490916004A0916104B9
:10151000B091620489839A83AB83BC83C8010E9423
:10152000856C83E08983F701808387E894E00E94DB
:10153000856CC8010E947D6CC7010E947D6C64E2CD
:1015400070E083E694E00E940CBCF8011192DA94FA
:10155000E9F7C8010E94816CC358DF4F18821982D5
:101560001A821B82CD57D0404AE0D42EDA94DD2077
:1015700031F0CE0183589F4F0E94856CF7CF88E0F1
:10158000F701982F11929A95E9F7F80111928A952F
:10159000E9F783E0CB57DF4F8883C558D040EA9600
:1015A0008FAFEA97CE018B579F4F0E947D6CCE0183
:1015B00087589F4F0E947D6C68E070E0C8010E94D0
:1015C0000CBC68E070E0C7010E940CBCC358DF4F40
:1015D000188219821A821B82CD57D0402AE0C22E6F
:1015E000D12CF1E0CF1AD10831F0CE0183589F4FB2
:1015F0000E94856CF6CF1982CC24CA94F701C08270
:10160000C8010E9462BCC7010E947D6C80E1D82E97
:10161000F8018D2D11928A95E9F760E170E0C8011B
:101620000E940CBC1982C8010E9462BC6CE070E090
:1016300087EA95E00E940CBC198A1A8A1B8A1C8AC8
:1016400080E090E0A0E8BFE38D879E87AF87B88BEE
:1016500080915C1190915D11A0915E11B0915F112C
:1016600089839A83AB83BC8320E030E543EC50E46C
:10167000609160117091611180916211909163117C
:101680000E94CBE76D837E838F8398872CEA35ECAD
:1016900047E25EE36091641170916511809166117B
:1016A000909167110E94CBE769877A878B879C8727
:1016B00064E170E0C8010E940CBC84E190E09A8370
:1016C000898362E070E0C8010E940CBC80919B0598
:1016D00090919C05A0919D05B0919E0589839A8368
:1016E000AB83BC8320E030E543EC50E460919F0580
:1016F0007091A0058091A1059091A2050E94CBE771
:101700006D837E838F8398872CEA35EC47E25EE316
:101710006091A3057091A4058091A5059091A605FF
:101720000E94CBE769877A878B879C87C8010E94D4
:10173000796C8CE0E1EDF1E0D80101900D928A9591
:10174000E1F7C8010E94796C1982C8010E947D6C82
:101750008FE78983C8010E947D6CC982C8010E94FD
:101760007D6C85E0EDEDF1E0D80101900D928A9558
:10177000E1F765E070E0C8010E940CBC1982C80165
:101780000E9462BC80E2E2EEF1E0D80101900D928D
:101790008A95E1F760E270E0C8010E940CBCF70195
:1017A0001082C7010E9462BC1982C8010E9462BCFB
:1017B00080E090E0A0EEBFE3C358DF4F88839983B9
:1017C000AA83BB83CD57D040CE0183589F4F0E9440
:1017D000856CC358DF4F188219821A821B82CD573D
:1017E000D040CE0183589F4F0E94856C82E1F80162
:1017F00011928A95E9F762E170E0C8010E940CBC81
:1018000084E2E2E0F2E0D80101900D928A95E1F7DE
:1018100064E270E0C8010E940CBCF8011192DA94F5
:10182000E9F760E170E0C8010E940CBC89E0F801B2
:1018300011928A95E9F769E070E0C8010E940CBC3A
:10184000C358DF4F188219821A821B82CD57D040AD
:10185000CE0183589F4F0E94856C9CE0D92EF801E1
:101860008D2D11928A95E9F76CE070E0C8010E9415
:101870000CBC8CE6F80111928A95E9F76CE670E0F1
:10188000C8010E940CBC8DEA94E00E94796CF701BB
:10189000108211821282138214821582168217829C
:1018A00068E070E0C7010E940CBCF7011192DA9465
:1018B000E9F7CB57DF4F1882C558D04080E090E061
:1018C000A0E4B0E4ED968CAF9DAFAEAFBFAFED97A7
:1018D000C7010E94816CCE018B579F4F0E947D6C87
:1018E000CE0187589F4F0E94856C8091B904811169
:1018F00027C0009144111091451180916811909179
:101900006911F7019183808384E690E090934511FB
:101910008093441164E070E08AE292E00E940CBC83
:1019200062E070E0C7010E940CBC91E00C3DF2E067
:101930001F0709F490E08091B904892B8093B904C2
:101940008091B904811105C060E08AE19DE10E94A7
:1019500041249091B90481E08927CA57DF4FE8E01C
:101960000C9472EEB0E0A0E0E8EBFCE80C9454EECE
:10197000C9EEDBE00FE016E089EFA82E8BE0B82E71
:10198000C12CD12C7601C394699179918991999157
:101990000E946AE7288939894A895B890E94CBE7D6
:1019A0000E9468EFF80161937193819391938F0185
:1019B000C616D706E806F90610F46B017C01AC16D2
:1019C000BD0611F76FEF7FEFCB01A70196010E94D3
:1019D00094ED20931F0630932006409321065093E8
:1019E0002206CDB7DEB7EAE00C9470EE0F931F939A
:1019F000CF93DF930DEF1BE0C8E2D6E0F801219111
:101A00003191419151918F0160E070E080E89FE356
:101A10000E94FBEE6993799389939993F6E0C8331A
:101A2000DF0761F70E94A8B69DDFDF91CF911F917C
:101A30000F9108959091D0118091D111981306C003
:101A40008091310C9091320C892B19F00E9459C56C
:101A5000F1CF08959091D0118091D111981307C0C2
:101A60008091310C9091320C892B09F4B1CC0E94F9
:101A700059C5F0CFA4E0B0E0E0E4FDE80C945AEEE4
:101A800020915E042223E1F08C0108960E94A56754
:101A900069837A838B839C83BE016F5F7F4FC8010C
:101AA0000E9461669B01AC01F801608571858285A9
:101AB00093850E9483EEF801608771878287938700
:101AC0002496E4E00C9476EEA4E0B0E0EAE6FDE8CB
:101AD0000C945AEE20915E042223E1F08C010896CA
:101AE0000E94A56769837A838B839C83BE016F5FA5
:101AF0007F4FC8010E9461669B01AC01F8016085BF
:101B00007185828593850E9484EEF80160877187D4
:101B1000828793872496E4E00C9476EEAEE1B0E001
:101B2000E4E9FDE80C944EEE9E8F8D8F5B018A01F7
:101B3000FC01EA5BFF4F2081318142815381298B77
:101B40003A8B4B8B5C8BCA01B9010E946AE76B012F
:101B50007C01D5012D913D914D915C910E94CBE787
:101B60000E94E8EE2B013C01F80120813181428185
:101B70005381C701B6010E94CBE70E94E8EE4B01FA
:101B80005C01C301B2010E9468EF6D8B7E8B8F8B6D
:101B9000988F683771058105910540F428E730E09A
:101BA00040E050E02D8B3E8B4F8B588FC501B40128
:101BB0000E9468EF698F7A8F8B8F9C8F68377105D1
:101BC0008105910540F488E790E0A0E0B0E0898FBE
:101BD0009A8FAB8FBC8FED8DFE8DEE5AFF4F20811B
:101BE00031814281538129873A874B875C87CA01BB
:101BF000B9010E946CE72B013C016D897E898F89B8
:101C0000988D0E946AE76D837E838F83988720E09A
